:100000000C942F0E0C94570E0C94570E0C94570E04
:100010000C94570E0C94570E0C94570E0C94570ECC
:100020000C94570E0C94570E0C94570E0C94B46607
:100030000C944A6A0C94E1660C94570E0C94D117F8
:100040000C94BF170C94570E0C94570E0C94570E2B
:100050000C94570E0C94570E0C94570E0C94570E8C
:100060000C940A6A0C942D180C944C670C94196823
:100070000C94570E0C94570E0C94570E0C94570E6C
:100080000C94570E0C94570E0C94570E0A6C0E6C71
:10009000166C206C376C516C666C756C8A6CA16C3C
:1000A000AB6CC96CCF6CD46CDA6CE06C3A6D446D9F
:1000B000E96CEF6CF56CFE6C026D076D0F6D216DD8
:1000C000276D2D6D326D126C126D176D1C6D537096
:1000D0006C617368008040000000000000000000B8
:1000E0000000000000000000000000000000000010
:1000F0000000000000000000000000000000000000
:1001000000000000000000000000000000000000EF
:1001100000000000000000000000000000000000DF
:10012000000080C0E0E0F0F8F8FCFCFCF8F8F8F023
:1001300040000000000080808000000000000000FF
:1001400000000000000000000000000080C0C0E0CF
:10015000E0E0F0F0F0E0C00000000000C0F8FFFFB9
:100160009F8783838383838383838383838383833F
:1001700083838383838383830383808383838383D2
:10018000838383838383838383838383838383833F
:100190008383C3E3733F1F0000000080E0F0F8FC9E
:1001A000FEFFFFFFFF7F3F1F1F0F0783C3E1E1E05B
:1001B000E0C0000E1F3F7F7FFFF3E0E08000000003
:1001C0000000000000000080F0FCFEFFFFFFFF7F4A
:1001D0003F0F0301010100000080F0FEFFFFC7C1D7
:1001E000C1C1C1C1C1C1C1C1C1C1C1C1C1C1C1C1FF
:1001F000C1C1C1C1C101C1F0FEFF3F0F070F0D0D0D
:100200000D1D191919193131313171616161E1C166
:10021000C1C18100000080E0F8FCFFFFFFFF2F1745
:100220000F038180C0E0F0F8FCFEFFFFFFFFFFFF3F
:100230007F010000000000000001010307070E1EFF
:100240001C3870E0F0F8FEFFFF7F1F0F0300010075
:10025000000000000000000000000000000000009E
:10026000000000000000000000000000000000008E
:10027000000000000000000000000000000000007E
:10028000000000000000000000000000000000006E
:1002900000000000007EFFFFFFFFFFFFFBF8FCFCFB
:1002A000FEFF7F3F1F0F07C3FFFFFFFFFFFF7F071B
:1002B0000000000000000000000000000000C0E09E
:1002C000F8FEFFFF7F1F0F1F3D7CF8F8F0E0800075
:1002D000000000000000000000000000000000001E
:1002E000000000000000000000000000000000000E
:1002F00000000000000000000000000000000000FE
:1003000000000000000000000000000000000000ED
:1003100000000000000000010101010103070707C0
:100320000301000000E0FCFFFFFFFFFF1F030000D0
:10033000000000000000000000C0F078DE27130974
:100340000E0703000000000000000001030F7FFF04
:10035000FC7878F800000000000000000000008039
:10036000808080808080808000808000808000008D
:1003700000000000008080808080808080808080FD
:1003800080808080808080000000000000000000ED
:10039000000000000000000000000000000000005D
:1003A000000080F0FEFFFFFFFF3F0F010000000094
:1003B00000000000C0E0381E0F0300010000000034
:1003C000000000000000000000000000000000002D
:1003D0000000030301000000000000000000000E08
:1003E0000E02020202020303000F0F000F0F0808A3
:1003F00008080808080F0F08080808080F0F000071
:1004000000000F0F000000000000000000000000CE
:1004100000000000000000000000000000000000DC
:10042000C0F8BFFFFFFF1F7F0100000000000000B9
:1004300000F0FCFF7F7830000000000000000000AA
:1004400000000000000000000000000000000000AC
:10045000000000000000000000000000000000009C
:10046000000000000000000000000000000000008C
:10047000000000000000000000000000000000007C
:10048000000000000000000000000000000000006C
:100490000000000000000000000000000000301C10
:1004A000070E0F0701000000000000000000000020
:1004B000000000000000000000000000000000003C
:1004C000000000000000000000000000000000002C
:1004D00000000000000000001B1E272D36394B4E87
:1004E000636C7278878D939CB1B4C6C9D2D8E1E4AD
:1004F00001020304010302040402030104030201D4
:1005000003010200040506076D656E75537461638F
:100510006B206F766572666C6F77006D656E7553D4
:100520007461636B20756E646572666C6F770070C2
:100530007265737320616E79204B657900414C457B
:100540005254004D455353414745004C4F41444997
:100550004E47002020202020202020202020202066
:1005600020202020202020202000506C6561736511
:1005700020526573657420537769746368657300EE
:100580005377697463686573205761726E696E672B
:1005900000204F6C642056657273696F6E2045456C
:1005A00050524F4D202020434845434B2053455443
:1005B00054494E47532F43414C494200416C6172AC
:1005C0006D732044697361626C6564005265736584
:1005D00074207468726F74746C65005468726F7400
:1005E000746C65206E6F742069646C650050726570
:1005F000737320616E79206B657920746F20736B43
:10060000697000414C45525400454550524F4D20B1
:100610006C6F77206D656D004F46464142535255D1
:1006200073525525454C73454C2554487354482501
:10063000414C73414C2550312050312550322050CF
:1006400032255033205033250054485252554445EA
:100650004C4549443049443149443241494C47456D
:100660004154524E535731535732535733535734E3
:1006700053573553573653573753573853573953C2
:100680005741535742535743004F4646004F4E2061
:10069000002D2D2D004348002D2D2D2000525544B6
:1006A00020454C45205448522041494C20005031AF
:1006B000202050322020503320204D4158204655D4
:1006C0004C4C4359433143594332435943335050BF
:1006D0004D3150504D3250504D3350504D3450509C
:1006E0004D3550504D3650504D3750504D38434891
:1006F0003120434832204348332043483420434884
:100700003520434836204348372043483820434863
:10071000392043483130434831314348313243482E
:100720003133434831344348313543483136002D65
:100730002D2D2D00564552533A2056312E35353049
:10074000312D6572657A00444154453A2031312E8D
:1007500030322E323031320054494D453A2031305A
:100760003A31303A3432002053564E3A20657239CD
:10077000782D7237303800204D4F443A2020202009
:100780000012081200081C0808081C0800000822B3
:1007900000490022080000000000227F2200000023
:1007A000082200490022080000082200490022080F
:1007B000000000227F220000000000082200490003
:1007C00022080000081C0808081C0800DA3013433F
:1007D000F7415E2B4624415423514748E1494A5092
:1007E000864A461D011F371FD71F522154546D00E2
:1007F000457870457846466E654D65644372730072
:10080000544F540053544B1153542500544D45112B
:100810005453570053544154005B4D454E555D2091
:10082000746F207265667265736800537461636BE0
:100830000F6200746D61696E0F6D7300746D7231BB
:10084000204A69747465720F757300746D72314C4F
:100850006174206D696E0F757300746D72314C6137
:1008600074206D61780F7573005354415432004DFC
:100870006F64650042616E6447617000506F74532D
:1008800063726F6C6C00416C61726D205761726EA7
:10089000696E67004D656D6F7279205761726E6980
:1008A0006E67005452453031324147005452453052
:1008B000313241470044656661756C74205377009E
:1008C000537769746368205761726E696E6700546C
:1008D00068726F74746C65205761726E696E670020
:1008E00053706C617368204E616D650053706C616C
:1008F00073682073637265656E004F4646004C69ED
:10090000676874206F6E2053746B204D76004C69BD
:10091000676874206F6666206166746572004C6952
:100920006768742073776974636800466C617368E4
:10093000206F6E2062656570004265657020636F90
:10094000756E74646F776E004D696E7574652062A4
:10095000656570005468726F74746C65207265769A
:10096000657273650053494E474F534D5046494C8D
:10097000540046696C7465722041444300496E61BD
:100980006374697669747920616C61726D0042618B
:100990007474657279207761726E696E6700436F57
:1009A0006E7472617374004861707469632053746B
:1009B00072656E67746800537065616B6572205074
:1009C0006974636800426565706572506953706B45
:1009D0007200536F756E64204D6F646500517569C8
:1009E0006574204E6F4B6579207853686F7274532D
:1009F000686F7274204E6F726D20204C6F6E67208E
:100A000020784C6F6E672000426565706572004FFC
:100A1000776E6572204E616D6500524144494F20EA
:100A200053455455500043616C004D756C746970AA
:100A30006C69657200636831636832636833636848
:100A400034006F6666202B3D203A3D006D6F646573
:100A50000A25207372632020737700536C617665DA
:100A600000545241494E455200000303030300560F
:100A7000455253494F4E005472696D2D202B002072
:100A80004D656E75204578697420446F776E20201F
:100A90002055705269676874204C6566740044493B
:100AA000414700424700414E41005B4D454E555D78
:100AB000205748454E20444F4E45004D4F56452047
:100AC000535449434B532F504F54530053455420D4
:100AD0004D4944504F494E54005B4D454E555D20A5
:100AE000544F2053544152540053544152542043C4
:100AF000414C4942524154494F4E0043414C4942B6
:100B0000524154494F4E0066726565004D4F444551
:100B10004C53454C00434F4C2044697265637469E3
:100B20006F6E0041494C20446972656374696F6E51
:100B300000454C4520446972656374696F6E0053CB
:100B4000776173682052696E6700436F6C6C6563F0
:100B500074697665002D2D2D202020313230202023
:100B600020313230582020313430202020393020BC
:100B70002020200053776173682054797065004805
:100B8000454C49205345545550000044454C45546C
:100B900045204D4F44454C0F5B4D454E555D00542F
:100BA0003254685472696700547261696E657200EC
:100BB000452E204C696D69747300504F534E454764
:100BC0000053686966742053656C004C50342F4C98
:100BD0005035202044534D326F6E6C792044534D74
:100BE000322F44534D580044534D205479706500C2
:100BF00053656E64205278204E756D626572205B7D
:100C00004D454E555D0050504D2046724C656E0D61
:100C10006D536563002052784E756D003443482053
:100C20003643482038434820313043483132434826
:100C3000313443483136434800755300755365637A
:100C40000050504D20202050585820202044534D13
:100C500032202050504D3136200050726F746F009A
:100C600052455441313233004265657020436E7401
:100C7000005472696D20537700457870202020451C
:100C80007846696E6546696E6520204D65646975B4
:100C90006D436F61727365005472696D20496E63B4
:100CA00000542D4578706F00542D5472696D0043C7
:100CB0006F756E7420446F776E436F756E74205538
:100CC0007020200054696D65722000547269676756
:100CD00065720054696D6572004E616D6500534523
:100CE00054555000000901000000000000060200F9
:100CF0004475706C69636174696E67206D6F6465BB
:100D00006C005B4D454E555D20205B455849545D58
:100D1000005945530B4E4F0044454C455445204D1A
:100D20004F44454C004455504C4943415445204D97
:100D30004F44454C00204142434445464748494AB8
:100D40004B4C4D4E4F505152535455565758595A7B
:100D50006162636465666768696A6B6C6D6E6F700B
:100D60007172737475767778797A303132333435BD
:100D7000363738395F2D2E006578702020252020E9
:100D800073773120737732004558504F2F4452000B
:100D9000000344522048696768004452204C6F7732
:100DA000004452204D69640044725377320044720B
:100DB00053773100576569676874004578706F0034
:100DC0004558504F2F445200002B2A52004D49588D
:100DD0004552005072657373205B455849545D203D
:100DE000746F2061626F7274004D6178206D697854
:100DF0006572732072656163683A200044454C4512
:100E00005445204D4958205B4D454E555D00536C6F
:100E10006F772020557000536C6F772020446F77D8
:100E20006E0044656C61792055700044656C617991
:100E300020446F776E0041646420202020204D758F
:100E40006C7469706C795265706C61636520004DDB
:100E5000756C747078004F4646005761726E696E0B
:100E60006700537769746368004375727665730031
:100E70004F4E204F4646005472696D004F46464F14
:100E80004E2000466C4D6F64657472696D004F664C
:100E90006673657400466D5472696D56616C0057D7
:100EA000656967687400536F7572636500454449EE
:100EB00054204D49582000494E53455254204D4925
:100EC0005820002D2D2D2D202020763E6F6673207A
:100ED00020763C6F667320207C767C3E6F66737C48
:100EE000767C3C6F6673414E44202020204F522078
:100EF00020202020584F522020202076313D3D7662
:100F000032207631213D76322076313E76322020F5
:100F100076313C7632202076313E3D763220763175
:100F20003C3D76322000535700435553544F4D20DB
:100F300053574954434845530000025341464554D2
:100F400059205357495443484553000002434C45E8
:100F50004152204D49584553205B4D454E555D004B
:100F60002052455441004368616E6E656C204F729B
:100F70006465720054454D504C4154455300434FF5
:100F80005059205452494D205B4D454E555D002D22
:100F90002D2D494E56004C494D4954530000030332
:100FA00003030303030303030303030303030043D4
:100FB0005600435552564553005052455345540030
:100FC000454449542D3E0043555256450009002DD5
:100FD0002D2D494E56004F46464F4E20002D2D2DAB
:100FE000783E30783C307C787C663E30663C307CA5
:100FF000667C6331206332206333206334206335A1
:101000002063362063372063382063392063313012
:10101000633131633132633133633134633135638A
:10102000313600454550524F4D206F766572666CE3
:101030006F7700454550524F4D206F766572666C54
:101040006F770067656E7772697465206572726F7D
:101050007200454550524F4D20466F726D61747459
:10106000696E670042616420454570726F6D20446F
:10107000617461004D4F44454C2020202020004DDC
:101080004520202020202020200050085000000073
:1010900000000000006F000007000700147F147FAD
:1010A00014242A7F2A1223130864623649552250D9
:1010B0000005030000001C2241000041221C001416
:1010C000083E081408083E080800503000000808D0
:1010D00008080800606000002010080402003E4973
:1010E000453E0000427F4000625149460041494967
:1010F00036001814127F0027454539003E49493211
:1011000000017905030036494936000649291E00C9
:101110000036360000005636000008142241141430
:101120001414144122140800020151090600060992
:1011300009067E0909097E7F494949363E414141F8
:10114000227F4141221C7F494949417F0909090108
:101150003E4149497A7F0808087F00417F410020CD
:1011600040413F017F081422417F404040407F02C0
:101170000C027F7F0408107F3E4141413E7F0909F8
:1011800009063E4151215E7F0919294626494949F0
:101190003201017F01013F4040403F1F2040201F9E
:1011A0003F4030403F63140814630708700807612C
:1011B00051494543007F414100020408102000418D
:1011C000417F00040201020440404040400001020F
:1011D000040020545454787F4844443838444444EC
:1011E00020384444487F3854545418087E0901027A
:1011F0000C5252523E7F0804047800447D40002087
:1012000040443D007F1028440000417F40007C04A2
:101210001804787C0804047838444444387C141456
:101220001408081414187C7C080404084854545406
:1012300020043F4440203C4040207C1C2040201C97
:101240003C4020403C44281028440C5050503C4422
:1012500064544C44000836410000007F0000004107
:101260003608000808221C08081C220808A0608014
:101270000000000000000000000000000000FFFF70
:101280000000000000001F3F00003F1F0000303042
:10129000FFFF3030FFFF30303078CCCCFFFFCCCCBC
:1012A0008C0C060F0F86C0E070381C0C3CFEC7E3A8
:1012B000F33B1E0C00000000333B1F0F000000003A
:1012C0000000F0F81C0E07030000000003070E1CCE
:1012D000F8F000003030E0C0FCFCC0E03030C0C0AE
:1012E000C0C0FCFCC0C0C0C0000000000000000086
:1012F0000000C0C0C0C0C0C0C0C0C0C0000000006E
:1013000000000000000000000080C0E070381C0CED
:10131000000000000000000000000000000038385D
:1013200000000000000000000000000000000303B7
:101330003F3F03033F3F03030C0C0C0C3F3F0C0CDF
:1013400007030C0E07030100183C3C180F1F38312F
:1013500033331E1E33330000000000000000000085
:10136000000003070E1C38300000000030381C0E4F
:1013700007030000030301000F0F00010303000037
:1013800000000F0F000000000000333B1F0F0000A3
:101390000000000000000000000000000000183CF9
:1013A0003C18000000000C0E0703010000000000C4
:1013B0000000FCFE87C3E377FEFC00000C0EFFFF7D
:1013C0000000000000000C0E0783C3E77E3C000015
:1013D0000303C3C3C3E7FE3C0000C0E070381C0E2B
:1013E000FFFF00003F3F33333373E3C30000FCFED5
:1013F000C7C3C3C78E0C00000303C3E3733B1F0FB7
:1014000000003CFEE7C3C3E7FE3C00003C7EE7C3B0
:10141000C3E7FEFC0000183C3C1800000000000080
:10142000183C3C18000000000000C0E0F0381C0E22
:1014300007033030303030303030303003070E1C8E
:1014400038F0E0C000000C0E07030383C3E77E3CC6
:1014500000000F1F3B3130381F0F000030303F3F7E
:101460003030000000003C3E373331303030000077
:101470003030303030391F0F000003030303030303
:101480003F3F00000C1C383030381F0F00000F1F8A
:10149000383030391F0F000000003F3F00000000CF
:1014A00000000F1F393030391F0F000000003038A6
:1014B0001C0E07030000060F0F06000000000000CE
:1014C000333B1F0F000000000000000103070E1C4B
:1014D00038300303030303030303030330381C0EF4
:1014E000070301000000000000003333010000008A
:1014F00000003C7EE7C3C3E77E3CF0F8DCCEC7C704
:10150000CEDCF8F0FFFFC3C3C3C3C3E7FE3CFCFE61
:101510000703030303070E0CFFFF030303070E1C5F
:10152000F8F0FFFFC3C3C3C3C3C30303FFFFC3C3B9
:10153000C3C3C3C30303FCFE0703C3C3C3C7CECCEB
:10154000FFFFC0C0C0C0C0C0FFFF00000303FFFF1B
:1015500003030000000000000303FFFF0303FFFF7D
:10156000C0E0F0381C0E0703FFFF00000000000081
:101570000000FFFF0E1CF8F81C0EFFFFFFFF387085
:10158000E0C08000FFFFFCFE070303030307FEFC2F
:10159000000000000000000000003F3F00000000CD
:1015A00000003F3F3F3F3030303030391F0F0F1FBA
:1015B0003830303030381C0C3F3F303030381C0E63
:1015C00007033F3F30303030303030303F3F000095
:1015D0000000000000000F1F3830303030303F3F37
:1015E0003F3F0000000000003F3F000030303F3F21
:1015F000303000000C1C383030381F0F00003F3FE7
:10160000000103070E1C38303F3F3030303030309F
:1016100030303F3F0000000000003F3F3F3F0000F0
:10162000000103033F3F0F1F3830303030381F0FA9
:10163000FFFFC3C3C3C3C3E77E3CFCFE0703030332
:101640000307FEFCFFFFC3C3C3C3C3E77E3C3C7E6E
:10165000E7C3C3C3C3C78E0C03030303FFFF030326
:101660000303FFFF000000000000FFFFFFFF00007A
:1016700000000000FFFFFFFF000000000000FFFF70
:101680000F1F38F0E0E0F0381F0F3F7FE0C0808090
:10169000C0E07F3F03030383C3E3733B1F0F0000DE
:1016A000FFFF0303030300000C1C3870E0C0800040
:1016B0000000000003030303FFFF000030381C0E8E
:1016C00007070E1C3830000000000000000000007A
:1016D0003F3F00000000000000000F1F383033378C
:1016E0001E1C3F333F3F000003070E1C38300C1C0C
:1016F0003830303030391F0F000000003F3F00000D
:1017000000000F1F3830303030381F0F03070E1C19
:1017100038381C0E07030F1F38381F1F38381F0FAB
:101720003C3E0703010103073E3C000000013F3F30
:10173000010000003C3E37333130303030300000A3
:101740003F3F303030300000000000000001030750
:101750000E0C0000303030303F3F00000000000031
:101760000000000000003030303030303030303099
:10177000000003070E1C383000000000303030300D
:101780003070E0C0FFFFC0E070303070E0C0C0E0FB
:101790007030303030300000C0E070303070E0C069
:1017A000FFFFC0E0703030303070E0C0C0C0FCFEE1
:1017B000C7C303070E0CF0F89C0C0C0C0C0CFCFCC3
:1017C000FFFFC0E070303070E0C000003030F3F355
:1017D00000000000000000003030F3F30000FFFFC5
:1017E0000080C0E07030000000000303FFFF000035
:1017F0000000F0F03070E0E07070E0C0F0F0C0E0A9
:1018000070303070E0C0C0E0703030303070E0C018
:10181000000000000000000000000C1E3F333333C6
:1018200033333F3F3F3F3030303030381F0F0F1FD2
:101830003830303030381C0C0F1F383030303030FA
:101840003F3F0F1F3B3333333333030300003F3F2E
:10185000000000000000000133333333333B1F0F1F
:101860003F3F0000000000003F3F000030303F3F9E
:10187000303000000C1C383030381F0F00003F3F64
:1018800003070F1C38300000000030303F3F30307D
:1018900000003F3F0000030300003F3F3F3F0000C8
:1018A000000000003F3F0F1F3830303030381F0F2E
:1018B000F0F03030303030F0E0C0C0E0F0303030A8
:1018C000E0C0F0F0F0F0C0E070303070E0C0C0E098
:1018D000F0303030303000003030FFFF303000006A
:1018E0000000F0F0000000000000F0F0F0F0000058
:1018F00000000000F0F0F0F0000000000000F0F048
:101900003070E0C08080C0E07030F0F080000000F7
:101910000000F0F03030303030B0F0F070300000C7
:10192000C0E03C3E0703000000000000FFFF000095
:101930000000000003073E3CE0C00000C0C0C0C083
:101940000C1CF8F0E0C0C0E0F0F81C0CC0C0C0C037
:101950003F3F0303030303030100000103030303E9
:1019600003033F3F3F3F0000000000000000303114
:1019700033333333333F1E0C00000F1F3830303801
:101980001C0C0F1F383030381C0C3F3F03070E1C57
:1019900038381C0E07030F1F38381C1C38381F0F2F
:1019A00030381C0F07070F1C383000013333333336
:1019B000333B1F0F30383C3E37333130303000007E
:1019C00000010F1F38300000000000003F3F000002
:1019D0000000000030381F0F010000000000000070
:1019E0000C0E07030100000103070E0C00000000AD
:1019F0004080080420100201081A141A1A1A271A23
:101A00002E1A3B1A461A511A53696D706C652034B0
:101A10002D434800542D43757400537469636B79EA
:101A200020542D43757400562D5461696C00456C2B
:101A300065766F6E5C44656C74610048656C692006
:101A40005365747570004779726F205365747570B3
:101A500000536572766F205465737400000089111D
:101A600012239B322446AD573665BF74488CC19D06
:101A70005AAFD3BE6CCAE5DB7EE9F7F881100801E6
:101A800093331A22A5562C47B7753E64C99C408DE6
:101A9000DBBF52AEEDDA64CBFFF976E802218B3082
:101AA000100299132667AF763444BD554AADC3BCC6
:101AB000588ED19F6EEBE7FA7CC8F5D983310A20A6
:101AC00091121803A7772E66B5543C45CBBD42ACA6
:101AD000D99E508FEFFB66EAFDD874C904428D533E
:101AE00016619F702004A9153227BB364CCEC5DF86
:101AF0005EEDD7FC6888E1997AABF3BA85520C4366
:101B000097711E60A1142805B3373A26CDDE44CF65
:101B1000DFFD56ECE9986089FBBB72AA06638F7201
:101B200014409D512225AB343006B9174EEFC7FE45
:101B30005CCCD5DD6AA9E3B8788AF19B87730E6225
:101B400095501C41A3352A24B1163807CFFF46EE25
:101B5000DDDC54CDEBB962A8F99A708B08848195CD
:101B60001AA793B62CC2A5D33EE1B7F04008C91915
:101B7000522BDB3A644EED5F766DFF7C89940085D5
:101B80009BB712A6ADD224C3BFF136E0C1184809F5
:101B9000D33B5A2AE55E6C4FF77D7E6C0AA583B471
:101BA000188691972EE3A7F23CC0B5D14229CB38D5
:101BB000500AD91B666FEF7E744CFD5D8BB502A495
:101BC00099961087AFF326E2BDD034C1C3394A28B5
:101BD000D11A580BE77F6E6EF55C7C4D0CC685D72D
:101BE0001EE597F42880A1913AA3B3B2444ACD5B95
:101BF0005669DF78600CE91D722FFB3E8DD604C755
:101C00009FF516E4A9902081BBB332A2C55A4C4B74
:101C1000D7795E68E11C680DF33F7A2E0EE787F6F0
:101C20001CC495D52AA1A3B03882B193466BCF7A54
:101C30005448DD59622DEB3C700EF91F8FF706E614
:101C40009DD414C5ABB122A0B9923083C77B4E6A34
:101C5000D5585C49E33D6A2CF11E780FB619112462
:101C60001FBECFEFD0E1DEBFCDBF11E0A0E0B1E0FD
:101C7000EAE7FCED02C005900D92A234B107D9F756
:101C80001EE0A2E4B1E001C01D92A837B107E1F760
:101C90001CE1CEE5DCE104C02297FE010E94F66D56
:101CA000CC35D107C9F70E94E8180C943B6E0C9410
:101CB00000003091B50422B78091B5043817C9F7F8
:101CC000932F80E030E0282B392BC901089529E2B9
:101CD000820290011124359527953595279587FD2A
:101CE000815C86FB880F880B80F9992787FD90958A
:101CF000281B390BC9010895F8942091D50D309116
:101D0000D60D7894C9010895482F50E09A01220F0A
:101D1000331F63E0440F551F6A95E1F7240F351F09
:101D200024543E4FC901089590E09C01220F331FB7
:101D3000220F331F280F391F24503D4FC90108952A
:101D4000AF92BF92CF92DF92EF92FF920F931F93C9
:101D5000CF93DF93C82E162FEA01F22ED02E57FF15
:101D600010C022FF02C08CE101C08FE09C2D981BA7
:101D7000892F612F4DE22F2D0E94A05CD095C19537
:101D8000DF4F2D2D2F218C2D612F4AE30E94A05C67
:101D90008F2D90E0B4E0AB2EB12CA822B922F2FE38
:101DA00002C0E2E001C0E0E0CE016CE370E00E941E
:101DB000A46D9B01442737FD4095542F0F2D0061E2
:101DC0008E2F8C0D612FA2E0EA2E0E94A05EA1143E
:101DD000B10411F0ECE101C0E1E1CE016CE370E08F
:101DE0000E94A46D9C01442737FD4095542F0D2D72
:101DF00000618E2F8C0D612FF2E0EF2E0E94A05E0D
:101E0000DF91CF911F910F91FF90EF90DF90CF90D6
:101E1000BF90AF9008950F931F93062F122F20624B
:101E200050E00E94D65F17FD07C08091A70D602F7C
:101E300046E7212F0E94A05C1F910F910895242F47
:101E4000409108010E940B0F08950F93022F442325
:101E500019F44FE257E020C04530A8F4E091860124
:101E6000F0E0EE0FFF1FEE0FFF1F3197E40FF11DA3
:101E7000E051FB4F449150E0440F551F440F551F54
:101E80004756594F09C0453250F450E0440F551F92
:101E9000440F551F4656594F24E00E94635D0F9131
:101EA0000895FF920F931F93182FF62E022F4423AD
:101EB00021F448E956E024E00EC08A5E4A3008F476
:101EC00085506F2D50E0202F0E94D65F812F6F2DFF
:101ED00045E956E022E00E94635D1F910F91FF905B
:101EE00008950F931F93DF93CF9300D0CDB7DEB744
:101EF000382F162F942F022F442329F0463139F022
:101F00004A3E81F408C08A5F41E956E007C08A5F13
:101F10004DE856E003C08A5F49E856E0202F0E9452
:101F2000935D28C04095441F4427441F81E2841BD1
:101F3000482F832F39839A830E94A05C3981832F95
:101F40008A5F9A81E92FFF27E7FDF095F7FF03C02D
:101F5000F095E195FF4FFF27E7FDF0953197AF0131
:101F6000440F551F4E0F5F1F475B594F612F23E0F2
:101F70000E94635D0F900F90CF91DF911F910F91A1
:101F8000089589E496E00895DF92EF92FF920F930F
:101F90001F93D82EE62EF42E1091AD01E12FFF27CE
:101FA000E7FDF095F7FF03C0F095E195FF4FE031B5
:101FB000A4F483E0E802F0011124E85EF94F8D2DCE
:101FC0006E2DAF0123E00F2D0E94635D1F3F3CF596
:101FD0008D2D86506E2D41E21FC08D2D8650E5322D
:101FE00064F411161CF4412F4F5002C0412F415F81
:101FF0006E2D2F2D0E94710F12C011161CF4412F4F
:10200000445202C0412F4C5D6E2D2F2D0E94710F46
:102010008D2D8E5E6E2D4DE62F2D0E94A05C1F91A2
:102020000F91FF90EF90DF9008958C3038F4E82FF7
:10203000F0E0EE0FFF1FE151FB4F2AC0803198F412
:10204000E82FF0E0DF01AA0FBB1FA457BB4FEE0F34
:10205000FF1FE45AFE4F2D913C9111978081918191
:10206000281B390B0AC0843158F4E82FF0E0EE0F3A
:10207000FF1FE457FB4F20813181220F331F0DC01A
:10208000843248F4E82FF0E0EE0FFF1FEB52FB4FD5
:102090002081318102C020E030E0C9010895AF9273
:1020A000BF92DF92EF92FF920F931F93DF93CF9334
:1020B00000D0CDB7DEB7F82E463008F0DEC088235A
:1020C00009F4DEC0863119F08A3E19F4D6C061E009
:1020D000D7C0992787FD90959C0197FF04C02227C0
:1020E0003327281B390B2A307CF41F144CF02DE0C9
:1020F00030E0A901481B590BCA010E944061BAC0D7
:102100000D960E944061BBC02A50A22EBB249501AF
:10211000220F331F2A0D3B1D2E553E4FF901E85A61
:10212000FD4F5081552309F4A8C0453029F4F5012D
:10213000E058FB4F80819CC0F901EA5AFD4FD080E6
:10214000295A3D4FF901E080553008F4A6C05830B7
:1021500060F08D2D81504A8359830E9415108C01A7
:102160008E2D81500E941510A2C020E030E000E0CA
:1021700010E0583088F4553088F5523009F462C0C8
:10218000533020F4513009F06EC057C05330D1F0B5
:10219000543009F068C01CC05A3009F44EC05B309E
:1021A00038F4583009F43FC0593009F05CC040C0E1
:1021B0005C3009F44CC05C3008F444C05D3009F078
:1021C00052C04AC017FF39C0109501951F4F35C046
:1021D00017FF38C0109501951F4F34C0142F1F5F93
:1021E0008D2D60E0412F0E944F10082F8E2D60E052
:1021F000412F0E944F10F501EE0FFF1FEA0DFB1D4E
:10220000E650FC4F9081953029F4002361F188233A
:1022100041F52AC0963029F4002319F5882319F1D5
:1022200020C0802721C081E002171307E1F41CC001
:1022300081E002171307C1F416C081E020173107AF
:102240009CF011C081E00217130774F00CC081E00C
:10225000021713074CF407C081E02017310724F45C
:1022600002C081E001C080E0F501E058FB4F8083AF
:102270001F142CF061E0682703C060E001C0682FE4
:10228000862F0F900F90CF91DF911F910F91FF90AC
:10229000EF90DF90BF90AF9008958D2D81504A83CD
:1022A00059830E9415108C018E2D0E94670E9C018F
:1022B0004A8159815ECF86B380958E7708950E94BA
:1022C0005B118823E1F70E94AF600895809173014C
:1022D00060E040E00E944F10882331F480919D041B
:1022E00090919E04009711F0C79A0895C798089599
:1022F0000F931F93CF93DF93EC018B010E94365C09
:1023000082E260E043E056E024E00E94935D80E2D8
:10231000BE010E94BA5D88E2B8010E94BA5D80E306
:102320006DEE75E00E94BA5D0E9440608091700180
:102330000E9436600E945F11DF91CF911F910F9133
:1023400008950F93AB0160E123E000E00E94635D1C
:102350000F910895DF92EF92FF920F931F93CF9307
:10236000DF938091850181FD83C080E895E06AE676
:1023700075E00E94781190919D01892F887341F03A
:10238000883131F0883221F0803311F0883329F41C
:10239000892F877C886080939D0100E010E065E1D3
:1023A000E62EF12C08C0C701801B91090E944061F4
:1023B000110F182B0F5F0830B0F3D0909D01D1267C
:1023C00080E060E143E555E026E100E00E94635DC6
:1023D000CD2DD0E0CE0180FF05C082E069E476E03B
:1023E0000E94A111C1FF05C087E16CE476E00E9464
:1023F000A111C2FF05C08CE26FE476E00E94A1113A
:10240000CE01887390700097B1F0012F13FF05C0C3
:1024100081E462E576E00E94A11104FF05C081E439
:1024200065E576E00E94A11105FF05C081E468E53D
:1024300076E00E94A111C6FF05C086E56BE576E057
:102440000E94A111D7FE05C08BE66EE576E00E94E2
:10245000A1110E94406080919D01181749F00E94CF
:102460005B11882329F40E94661100E010E09BCFE5
:10247000DF91CF911F910F91FF90EF90DF90089522
:102480001F93CF93DF930E945B1120E030E011E0B7
:10249000482F50E02F5F3F4FBA01022E02C07595C2
:1024A00067950A94E2F760FD03C01F5F183091F74B
:1024B0001150163030F5812F0E94B156882309F152
:1024C00010936F01812F0E94B55681E00E948457BE
:1024D0000E94365C86E160E04BE455E024E00E9417
:1024E000935DC2EAD1E01AE04991812F68E124E0CE
:1024F0000E94A05C155F1837B9F70E9440600E94E7
:102500005F11DF91CF911F910895CF93DF93EC017D
:102510000E94365C82E260E043E455E024E00E94E1
:10252000935D88E1BE010E94BA5D0E944060809187
:1025300070010E943660DF91CF9108951F93CF9371
:10254000DF93EC01162F0E94365C82E260E04DE3DF
:1025500055E024E00E94935D88E1BE010E94BA5DCF
:102560008CE168E34FE255E00E94C25D0E9440604A
:10257000112319F48091700101C089E10E94366035
:1025800082E10E945E6D0E945F110E945B118823B0
:10259000C9F48091690E833019F4A8951092690EE0
:1025A0008091730160E040E00E944F10882331F475
:1025B00080918A01882311F4112311F0C79AE5CF85
:1025C000C798E3CFDF91CF911F91089580917F0449
:1025D000882351F081E995E060E00E949E1280918D
:1025E0007F048E7F80937F0408958091850187FD0D
:1025F00007C0887329F48CEB95E060E00E949E127E
:1026000008958091850182FD0AC00E94A558883CEA
:10261000910528F489E096E060E00E949E120895FA
:10262000EF92FF92CF93DF93A82FAF70A6509091B7
:10263000B401923074F0292F332727FD30952150B3
:102640003040C1E0D0E002C0CC0FDD1F2A95E2F798
:102650009C2FA83008F09CC06A2F659570E0FB01A4
:10266000EE0FFF1FE050FF4F0190F081E02DB08191
:10267000992379F4CB2FDD27C7FDD095D7FF03C071
:10268000D095C195DF4F9C2FC7FD9D5F9595959582
:102690009F5F4091860150E04170507022E030E031
:1026A000241B350B2617370769F42091B3012F70CF
:1026B00009F473C021E094E03091880130FF03C039
:1026C000919501C020E04B2F552747FD5095C92F0C
:1026D000DD27C7FDD095A0FF03C0C40FD51F04C0E0
:1026E000BA016C1B7D0BEB01209729F07E019F2D19
:1026F0009B2797FF0BC0222349F4BB2339F010829C
:102700000E949F6186E10E945E6D41C0CE018458A7
:102710009F4F893F9105B8F4C08386E00E9484579B
:10272000CE0183589F4F8B3F910588F5D7FF03C09B
:10273000D095C195DF4FD595C795D595C795BE0165
:10274000645C462F1FC01C161D0614F48DE701C0E3
:1027500083E8808386E00E948457CE0183589F4F90
:102760008B3F9105A0F4CE01D7FF03C090958195D2
:102770009F4F64E070E00E94A46D709561957F4F5B
:10278000462F445C87E494E065E10E94EB6B80E0B7
:10279000DF91CF91FF90EF90089520E08DCF8F9241
:1027A0009F92AF92BF92CF92DF92EF92FF920F93E0
:1027B0001F93CF93DF93182FEB015A016901802EED
:1027C00084FF06C01F70106694E0992E05E003C0D8
:1027D00085E0982E04E0802F8066181761F0802F26
:1027E0008064181741F080911E05882369F0133624
:1027F00011F0133449F47E010894E11CF11C83E1CB
:102800000E945E6D892D18C0992D9066191761F090
:10281000992D9064191741F0882309F474C0123679
:1028200019F0123409F06FC07E010894E108F10834
:1028300084E10E945E6D802F90E00E9440618823B9
:1028400051F0EE24FF24EC1AFD0A892D0E949F61AD
:10285000802F0E949F61A114B10491F481E0C816F9
:10286000D10471F4103661F410921E0501E0E02EDF
:10287000F12C209711F0EE24FF2480E60E949F6146
:1028800020919A0430919B04E21AF30ACE14DF04DB
:1028900044F4812F0E949F6183E10E945E6D760166
:1028A0000AC0EA14FB043CF4812F0E949F6184E17A
:1028B0000E945E6D7501EC16FD06A9F0E114F104AD
:1028C00051F4812F0E949061D7FF02C083E101C0C3
:1028D00084E10E945E6D882D83700E94845781E0A0
:1028E0008093970402C010929704C701DF91CF91A3
:1028F0001F910F91FF90EF90DF90CF90BF90AF901E
:102900009F908F9008957E01A6CF0F93772767FD44
:102910007095552747FD5095332727FD30950E9428
:10292000CF130F9108950F93772767FD7095552763
:1029300047FD5095332727FD309502E00E94CF13C5
:102940000F9108950F93772767FD7095552747FDE1
:102950005095332727FD309501E00E94CF130F914A
:102960000895E0919604F0E0EE0FFF1FE257FB4F51
:1029700080819181089590919604992319F4882378
:1029800031F418C0882319F4892F815001C080E0E8
:102990008093960487E10E945E6DE0919604F0E0DA
:1029A000EE0FFF1FE457FB4F0190F081E02D8EEBFF
:1029B000099508958BE195E060E00E949E120895CC
:1029C000FC01A0919604B0E0AA0FBB1FA457BB4F17
:1029D0008D939C938FEB099587E10E945E6D08951E
:1029E000CF93DF93EC0180919604982F9F5F909393
:1029F0009604953040F08093960488E095E060E07E
:102A00000E949E120FC087E10E945E6DE0919604C5
:102A1000F0E0EE0FFF1FE457FB4FD183C0838FEB35
:102A2000FE010995DF91CF91089587E494E00E941B
:102A3000EA6A882311F084E105C08091B6048823F6
:102A400021F081508093B60407C09091630081E02B
:102A500091FF80E08093B7048091B70408951092AD
:102A6000A1041092A3041092A2041092A00408954D
:102A700020919D0430919E042115310531F02150A3
:102A8000304030939E0420939D04882369F0409148
:102A90008A0150E084EF91E0489F9001499F300DFA
:102AA000589F300D112402C020E030E080919F0437
:102AB000882369F06091920170E044EF51E0649FD7
:102AC000C001659F900D749F900D112402C080E09D
:102AD00090E040919D0450919E044217530720F4CA
:102AE00030939E0420939D0420919D0430919E0478
:102AF0002817390720F490939E0480939D040E9428
:102B000066110895E82FF0E0E050FB4FE491F0E00B
:102B1000EE0FFF1FE654FB4F20813181C90108955C
:102B2000CF92DF92EF92FF920F931F93DF93CF9399
:102B30000F92CDB7DEB720E0CC24DD24822F29838D
:102B40000E948215092F10E0C00ED11E29812F5F2F
:102B50002430A1F7C6010F90CF91DF911F910F9103
:102B6000FF90EF90DF90CF9008951F930E947C0E0E
:102B700041E02091ED043091EE048217930709F4AF
:102B800040E040939C040E947C0E9093EE0480935E
:102B9000ED0483E295E060E00E941C3580919C0486
:102BA000882309F4CBC08091A00480FF14C08091D9
:102BB000A104982F9F5F9093A104943660F08356F0
:102BC0008093A1048091A2049091A3040196909314
:102BD000A3048093A20480E00E9492570E94365C76
:102BE0000E94B2600E941013182F0E943815209185
:102BF000FB043091FC048091980490919904821B0D
:102C0000930B60E270E00E94A46D70939B0460934C
:102C10009A046115710591F08091EB049091EC0498
:102C2000821B930B62E070E00E94A46D70939B0482
:102C300060939A0430939904209398043093EC04A1
:102C40002093EB048091880185FF04C010929B04BF
:102C500010929A04E0919604F0E0EE0FFF1FE45703
:102C6000FB4F0190F081E02D812F09950E9440607B
:102C70000E941515882321F0809165008F7E03C086
:102C8000809165008061809365000E947C0E8F7149
:102C900090708230910509F04FC087E00E94821544
:102CA0009C01E4E0220F331FEA95E1F768E070E051
:102CB0000E94A46D40917201552747FD50954A5FCF
:102CC0005F4F649FC001659F900D749F900D11240C
:102CD000820F931F2091880126FD05C06091090194
:102CE00070910A0102C060EF70E02091080130E0AD
:102CF0002F5F3F4F0E94906D260F371F3595279508
:102D0000209308018091EA04805E8093EA0488237E
:102D100099F480917101281778F4223368F081E1E9
:102D20000E945E6D8091880183FF06C082E390E07F
:102D300090939E0480939D0410929F041F91089588
:102D4000AAEBB4E0EAECF4E060E0862F806487B997
:102D5000369A408951898D919C91119796958795C6
:102D6000840F951F8E7F11969C938E9320813181C5
:102D7000C901840F951F96958795918B808B349B05
:102D8000FECF349A84B195B1820F931F96958795A3
:102D9000819391936F5F12966830B9F60895EF9220
:102DA000FF920F931F93CF93DF938091880184FD4F
:102DB00044C00E9466110E94365C80E060E045EDF0
:102DC00050E020E000E00E94415C80918E0184FD93
:102DD00008C080E068E343E951E02AE000E10E9496
:102DE000635D0E944060809170010E9436600E9485
:102DF0005F1100E20E94A0160150E1F70E949015B9
:102E00008C010E947C0EEC01C057DE4F0DC00E9469
:102E1000A0160E9490157C010E945B11882369F422
:102E2000E016F10651F406C00E947C0EC817D907BF
:102E300071F703C00E946611F7CFDF91CF911F9108
:102E40000F91FF90EF900895EAEBF4E040E012C09C
:102E500067B9369A349BFECF349A24B135B1820FCC
:102E6000931F5150A9F796958795819391934F5F42
:102E7000483031F054E080E090E0642F6064E8CFA7
:102E80000895EAEBF4E020E0822F806487B9369A57
:102E9000349BFECF349A84B195B1880F991F8193EA
:102EA00091932F5F283081F70895FF920F931F931E
:102EB000CF93DF938091850180FD3AC08091860198
:102EC00090E08170907002E010E0081B190BF8018F
:102ED000EE0FFF1FEE5BFE4FC181D28160968785AA
:102EE0009089C81BD90B0E944117F02E802F0E9499
:102EF0008215C817D907E4F40E945B118823C1F436
:102F00000DC00E9441178F2D0E948215C817D90746
:102F10007CF40E945B11882341F00AC08BED95E0A0
:102F20006CEC75E00E947811ECCF0E946611E9CF3D
:102F3000DF91CF911F910F91FF9008958EE587B992
:102F4000369A349BFECF349A84B195B10496409161
:102F5000090150910A019A0163E0220F331F6A951B
:102F6000E1F7241B350B820F931F23E0969587957D
:102F70002A95E1F790930A018093090108957894C6
:102F80001F920F920FB60F9211248F938091B50468
:102F90008F5F8093B5048F910F900FBE0F901F909D
:102FA000189578941F920F920FB60F9211242F93B9
:102FB0003F934F935F936F937F938F939F93AF93C1
:102FC000BF93EF93FF93F89487B78D7F87BF789473
:102FD00081B78E5F81BF9091490480914B04882313
:102FE00079F080919101882349F0813051F48091EA
:102FF000770E890F8093770E87FF02C01B9A01C05E
:103000001B9880910B01982F915090930B0188236E
:1030100071F48DE480930B0187E494E00E94FE6AD2
:103020000E94B0618091690E82608093690EF8946D
:1030300087B7826087BF7894FF91EF91BF91AF917E
:103040009F918F917F916F915F914F913F912F91C0
:103050000F900FBE0F901F90189578941F920F92AB
:103060000FB60F9211241F932F933F934F935F93AB
:103070006F937F938F939F93AF93BF93EF93FF9340
:103080002091800030918100F89480917D008F7DA7
:1030900080937D0078948091B8049091B904A9013F
:1030A000481B590BCA01969587953093B904209314
:1030B000B8041091B404212F2150283058F59C01F8
:1030C0002152334055E02737350708F5E12FF0E06E
:1030D000EE0FFF1FEE55FB4FAC014C5D55402091AC
:1030E0008C01332727FD3095265F3F4F429FC0015B
:1030F000439F900D529F900D11246AE070E00E9452
:10310000A46D718360831F5F1093B4040CC0109290
:10311000B40409C0815A9F402EE28F3D920718F4F3
:1031200081E08093B404F89480917D008062809364
:103130007D007894FF91EF91BF91AF919F918F9116
:103140007F916F915F914F913F912F911F910F90C0
:103150000FBE0F901F901895E9E7FEE09F01819147
:103160008535E1F328573E40C9010895CF93DF9399
:103170000E94590EEC0180918901813019F40E945E
:10318000A01607C0823019F40E94241702C00E94C2
:1031900041178EE587B90E94B5150E949E17809150
:1031A000690E833019F4A8951092690E0E94590E89
:1031B0008C1B9D0B2091C5063091C6062817390738
:1031C00020F49093C6068093C506DF91CF910895B1
:1031D0001F938FEF8ABB1BBA91E897BB9EE798BB02
:1031E0009EE394BB91EC95BB11BA82BB88E082B997
:1031F00087EF83B9109261001092620084E180939E
:1032000064008BEF809365000E94006080E487B9C2
:1032100085E886B987E083BF8CE981BF87B7836083
:1032200087BF1FBC8AE08EBD10928B0082E880931E
:103230008A0080917D00806280937D00EDB7FEB7AB
:10324000329785E502C0808331979EE0E837F90721
:1032500009F0C8F778948AEF9EE390938D048093E9
:103260008C0489E10E9436600E943D5710916F01E5
:103270000E944012809170010E94366050918A0134
:1032800040919201451778F4652F70E024EF31E00A
:10329000629FC001639F900D729F900D11249093C7
:1032A0009E0480939D04541770F450E024EF31E0A5
:1032B000429FC001439F900D529F900D1124909307
:1032C0009E0480939D040E9466118091910181303B
:1032D00039F48091880184FD03C087E00E945E6D0F
:1032E0000E94CF160E9401130E9441170E94551799
:1032F0000E94AA110E94F5120E94E6120E945F111C
:1033000080EF90E090930A01809309010E94556933
:103310002DE088E190E00FB6F894A89581BD0FBE2E
:1033200021BD83E295E060E00E941C358AED90E3C8
:103330000E94F01481E00E94BB14809170010E94F1
:10334000366080916F01181729F081E00E94845740
:103350000E94205880ED97E09BBD8ABD80E186BF2A
:1033600087B7806187BF0E94B618FDCF87E494E0DD
:103370000E94E76A089529E282029001112435959E
:1033800027953595279587FD815C86FB880F880BEF
:1033900080F9992787FD9095281B390BC90108955D
:1033A0009C01E5E035952795EA95E1F7AC01440FDE
:1033B000452F441F550B280F391F892F990F990B43
:1033C0008595280F391F241B350BC9010895F894E2
:1033D0002091D50D3091D60D7894C9010895AC0196
:1033E00080E060E021E00E94935D08950F931F93B9
:1033F000CF93DF93182F84E198E00E94EF191136E4
:1034000058F0133628F0133639F481E99AE102C0F6
:103410008AEF9EE30E94E01486E068E04CE058E00A
:103420000E94C25D40913D0650913E068AE268E0EE
:1034300020E000E00E94A00E40913F06509140061F
:103440008EE468E020E00E94A00E86E060E144E0A7
:1034500058E00E94C25D40914106509142068AE2C6
:1034600060E120E00E94A00E409143065091440686
:10347000F4E056954795FA95E1F78EE460E120E097
:103480000E94A00E86E660E040E058E00E94C25D27
:1034900040913B0650913C068EE460E020E00E94A3
:1034A000A00E8091C1069091C2068937910528F03F
:1034B0008091C006C82FD0E002C0C0E0D0E082E01A
:1034C0006CE34EE70E94405E85E06CE143E20E94BF
:1034D000445E1BE0812F6BE343E00E94445E1A5F71
:1034E0001338C1F716E00CE3FE01E85BF94F4081A9
:1034F000602F641B812F0E94445E2196C837D1053E
:1035000010F0C0E0D0E02091C00630E0C217D30731
:1035100019F01F5F1E3741F7DF91CF911F910F9177
:1035200008951F93182F89E698E00E94EF1912362C
:10353000E1F0133628F4103631F01136E9F418C0F2
:103540001336D1F415C08FEF97E090930D0180935F
:103550000C011092C4061092C3061092C606109277
:10356000C50687E10E945E6D07C086EF99E102C043
:103570008AEF9EE30E94E01488E06AE578E00E940A
:10358000BA5D4091C3065091C4065695479584E5AF
:1035900068E00E94E65F80E16BE478E00E94BA5D3B
:1035A00040910C0150910D015695479584E560E1DD
:1035B0000E94E65F88E16CE378E00E94BA5D40918A
:1035C000C3065091C40680910C0190910D01481BD7
:1035D000590B5695479584E568E10E94E65F80E2C5
:1035E00063E378E00E94BA5D2091C5063091C6067B
:1035F00084E690E0289FA001299F500D389F500D30
:103600001124A4E056954795AA95E1F784E560E278
:1036100020E30E94D65F88E26BE278E00E94BA5D08
:103620000E94AC18AC018FE368E20E94C65D82E1A3
:1036300068E349E158E00E94C25D1F9108958DED55
:103640009FE008950F9393E0499FA00111244A52EF
:10365000504F01E0222309F400E023E00E94635D63
:103660000F9108950F9393E0499FA00111244153B6
:10367000504F01E0222309F400E023E00E94635D43
:103680000F910895FF920F931F93F82E062F142F7A
:1036900080E860E0402F50E0212F0E94D65F0A3082
:1036A00010F00FE601C005E7802F60E04FE2212F08
:1036B0000E94A05C4F2D50E04F5F5F4F802F60E075
:1036C000212F0E94D65F1F910F91FF9008956F9256
:1036D0007F928F929F92AF92CF92DF92EF92FF9262
:1036E0000F931F93CF93DF93EC01162FD42E490134
:1036F0006090F7047090F8048091C6089091C70814
:103700008619970920E430E0B9010E94A46D462F84
:1037100060932105E091F904F091FA048091C408C6
:103720009091C5088E1B9F0BB9010E94A46D862F36
:1037300060932205442321F07092C7086092C60866
:10374000882321F0F093C508E093C40880912005F8
:10375000882321F48091880185FF06C010922105FD
:10376000109222051092200560912105662351F4E4
:1037700080912205882331F480919A0490919B04D2
:10378000009781F040918A0150E024EF31E0429FA0
:10379000C001439F900D529F900D112490939E0461
:1037A00080939D048114910409F456C08881882374
:1037B00009F04BC0662331F180911E05882311F575
:1037C000ED2DE61BE7FDE0E0202F30E08E2F99275E
:1037D00087FD90958217930714F0E02FE150FF27A3
:1037E000E7FDF0958D2D90E0E817F90749F0EE0F11
:1037F000FF1FE80DF91D25913491C9010E94E014C5
:1038000010922105153641F4DD2011F0ED2D01C097
:10381000E02FF0E031970FC01436C9F42D2D30E0C1
:10382000802F90E00197281739071CF4ED2DEF5FEA
:1038300001C0E0E0F0E0EE0FFF1FE80DF91D25915B
:103840003491C9010E94E01402C040E001C041E08F
:103850008D2D602F0E94421BE114F10451F09881DC
:103860008C2D9C1508F4892FF701E80FF11D549158
:1038700001C050E080911E05882309F04FC080915F
:103880002205882329F14881481B47FD40E0242F69
:10389000332727FD30958A2D90E0281739070CF043
:1038A0004A2D48838981E114F10459F0C41608F4C3
:1038B0004C2DF701E40FF11DE4918E1718F4E82F59
:1038C00001C0E0E0E98380E68093D70D10922205E5
:1038D0008881882319F1909121059923F9F0498174
:1038E000E114F104B1F0491B47FD40E09C2D8C151B
:1038F00008F4982FF701E90FF11DE491242F3327E5
:1039000027FD30958E2F90E0281739071CF04E2F99
:1039100001C040E0498380E68093D70D103651F115
:10392000113690F4133409F480C0143430F4113299
:1039300079F1123409F09CC06AC0143409F43FC014
:10394000153409F095C04FC01436E9F1153638F436
:10395000123609F45FC0133609F08AC069C0113805
:10396000A1F01F3B21F0153609F082C040C019823A
:10397000188212C0552309F47BC081E090911E0586
:10398000911180E080931E0573C010921E050DC03A
:1039900080911E05882319F010921E0569C0888148
:1039A000882319F08114910421F480E00E94BB1453
:1039B0005FC087E10E945E6D1982188256C08981BE
:1039C000851709F455C0E114F10409F451C0809140
:1039D0001E05882309F04CC08981851710F48F5F7C
:1039E00012C0198242C08981882309F441C0E114C0
:1039F000F10409F43DC080911E058823C9F5898131
:103A0000882319F08150898330C059832EC0888162
:103A10008A1571F180911E05882351F588818A15D8
:103A200010F48F5F0DC018820EC08881882301F1C9
:103A300080911E058823E1F48881882319F0815044
:103A4000888301C0A8828981E114F10461F0988122
:103A50009C1508F4C92EEC0CF11CF7019491891700
:103A600018F4982F01C090E0998380E68093D70DD9
:103A7000DF91CF911F910F91FF90EF90DF90CF904A
:103A8000AF909F908F907F906F9008954F925F922C
:103A90006F927F928F929F92AF92BF92CF92DF925E
:103AA000EF92FF920F931F93DF93CF930F92CDB7B7
:103AB000DEB7D82E81E69AE00E94EF1988E498E0FC
:103AC0006D2D41E020EE37E006E059E6E52E5AE0A4
:103AD000F52E15E0C12EB6E0AB2E0E94671B80903C
:103AE0004808909049088091630081FF07C08AE2EE
:103AF00068E14BE55AE00E94C25D60C182E168E086
:103B00004CE45AE00E94C25D8A9480911E0588238D
:103B100019F0A2E0CA2E02C0CC24C394EE24FF24E4
:103B200010E1A82CBB24A7FCB094F4E06F2E712CFC
:103B30002701440C551C8CE791E0480E591E4E2D70
:103B40004F5F80E0612F20E00E94250FAE14BF047C
:103B500011F491E0911090E0F201218122952695D7
:103B60002695237030E0A901440F551F420F531FC3
:103B70004E5B554F992311F400E001C00C2D88E1F4
:103B8000612F23E099830E94635D99819923C1F09D
:103B900080911E058823A1F0F201618162956695EE
:103BA000669563708D2D40E022E00E94A2148295FC
:103BB000880F880F807CF20191819F73982B9183ED
:103BC000AE14BF0421F401E0F92DF13009F000E05A
:103BD000F2018181880F880F85958595FDE08F0220
:103BE000C0011124B3010E94A46DAB01002311F4A4
:103BF00020E001C02C2D82E4612F0E94D65F0023BB
:103C0000A9F080911E05882389F0F2016181660F79
:103C1000660F659565958D2D41EE2FE10E94A214EA
:103C20008F73F2019181907C982B9183AE14BF0425
:103C300021F491E0F92DF23009F090E0F2012081B9
:103C4000277030E0A901440F551F420F531F4B5CF2
:103C5000554F992311F400E001C00C2D88E4612F29
:103C600023E099830E94635D9981992391F080916B
:103C70001E05882371F0F201608167708D2D40E090
:103C800023E00E94A2148770F2019081987F982B04
:103C90009083AE14BF0421F401E0F92DF33009F054
:103CA00000E0F2014081459545954595002311F4CA
:103CB00020E001C02C2D8AE5612F0E94710F0023A6
:103CC000B1F080911E05882391F0F2016081659525
:103CD000659565958D2D4AEE26E10E94A214880F08
:103CE000880F880FF20190819770982B9083185F4E
:103CF0000894E11CF11C103309F01ACF80E36AE24A
:103D00007AE00E94BA5D40918C01552747FD50959D
:103D1000465F5F4FF82DF43011F421E201C020E23C
:103D20008EE460E30E94D65F282D243049F48D2D67
:103D300060918C0146EF28E20E94A21480938C01CE
:103D4000EE24E394882D853009F0EE2480E068E3CA
:103D500046E25AE02E2D0E94935D44EAA42E44E0F0
:103D6000B42E04E711E090E3F501419151915F0118
:103D7000F801219131918F01421B530B440F551FC4
:103D8000892F68E320E299830E94D65F9981985E2B
:103D9000903951F7EE2091F0FD2DF03679F4A4E73B
:103DA000B1E0E4EAF4E088E001900D928150E1F79F
:103DB00081E00E94845787E10E945E6D0F90CF9151
:103DC000DF911F910F91FF90EF90DF90CF90BF9008
:103DD000AF909F908F907F906F905F904F900895DD
:103DE000AF92CF92EF92FF920F93AE2CEE24FF246E
:103DF000CC240E94671B0F91FF90EF90CF90AF9063
:103E00000895EF920F93DF93CF930F92CDB7DEB764
:103E1000682F8FE69AE069830E94EF198AE498E0A0
:103E2000698142E020EE37E006E0EE240E94F01EB9
:103E300080E167E677E00E94BA5D88E164E377E0BD
:103E40000E94BA5D80E267E477E00E94BA5D88E292
:103E500068E577E00E94BA5D80E367E777E00E945B
:103E6000BA5D0F90CF91DF910F91EF900895CF92AF
:103E7000DF92EF92FF920F931F93DF93CF9300D0C7
:103E8000CDB7DEB7682F8EE99AE069830E94EF19FB
:103E90008CE498E0698143E020EE37E006E0EE2410
:103EA0000E94F01EEEE0CE2ED12C00E010E0143087
:103EB00020F078EFF72EF00E01C0F02EC6010E9420
:103EC0004061E82E1F5F8AE26F2D412F20E00E94A3
:103ED000710F4E2D405D84E46F2D2E2D0E94A05C4D
:103EE000085F0894C11CD11C193009F708E3CC24E1
:103EF000DD2410E0812F90E00E944061F82EA601A1
:103F00004158554F80E0602F25E00E948D5D4F2D78
:103F1000405D80E2602F2F2D0E94A05C1F5F85E036
:103F200090E0C80ED91E0850163021F784E568E1EC
:103F300047E75AE027E00E948D5D66E0E62EF12C0F
:103F400010E230E084E5612F41E857E0232F00E0E4
:103F50003A830E94415CC7010E944061282FC7013B
:103F6000019629830E944061082F2981422F405DDC
:103F70008CE6612F0E94A05C402F405D88E7612F96
:103F8000202F0E94A05C3A813F5F185FE2E0F0E0E2
:103F9000EE0EFF1E3430B1F60F900F90CF91DF91EF
:103FA0001F910F91FF90EF90DF90CF9008958F9227
:103FB0009F92AF92BF92DF92EF92FF920F931F9367
:103FC000CF93DF93D82E86EA9AE00E94EF198EE411
:103FD00098E06D2D44E020EE37E006E0EE24E39417
:103FE0000E94F01EF0904E08CFEED4E010E000E00A
:103FF000812CF4E09F2EA12CB12C88E1612F41E4AB
:104000000E945F5D402F4F5C8EE1612F0E945F5DDB
:10401000802F0E948215AC018AE2612F0E94C65D4A
:104020000730B1F068817981882777FD8095982FD6
:1040300024E630E040E050E00E94656DA501940167
:104040000E94D96D8AE5612FA9010E94E65F0AC02E
:104050008F2D813011F040E201C041E28AE5612FED
:104060000E941F0F0F5F185F2296083031F68CE612
:1040700068E243EA5AE022E00E948D5D4091090126
:1040800050910A0188E760E320E00E94D65F8F2DFF
:10409000813059F4F09220058D2D6091720141E834
:1040A0002FE70E94A21480937201DF91CF911F919C
:1040B0000F91FF90EF90DF90BF90AF909F908F9007
:1040C0000895EF920F93E42E40E020E030E000E00E
:1040D0000E94F01E0F91EF900895AF92BF92CF9281
:1040E000DF92EF92FF920F931F93DF93CF9300D055
:1040F000CDB7DEB78FE161E247E10E94445E8FE118
:1041000067E347E10E94405E85E361E247E10E9488
:10411000445E8FE161E247E10E94405E8BE461E230
:1041200047E10E94445E8BE467E347E10E94405E02
:1041300081E661E247E10E94445E8BE461E247E18F
:104140000E94405E8AE26BE243E00E94445E89E2A4
:104150006CE243E00E94405E86E56BE243E00E9431
:10416000445E85E56CE243E00E94405E8091EF048E
:104170009091F00451E7C52ED12CB6010E94A46D98
:10418000262F8091F1049091F2040FE81FEFB801FF
:104190000E94A46D362F48E2E42EE20E9AE2F92E38
:1041A000F60E8E2D6F2D45E02A8339830E94445EE2
:1041B0003981632F625D8E2D45E00E94405E2A8129
:1041C000822F845D6F2D45E00E94445E8E2D6F2D01
:1041D00045E00E94405E8091F5049091F604B6019E
:1041E0000E94A46D262F8091F3049091F404B801ED
:1041F0000E94A46D062F84E5F82EF20E162F165D90
:104200008F2D612F45E02A830E94445E602F625DFE
:104210008F2D45E00E94405E2A81822F885A612FAF
:1042200045E00E94445E8F2D612F45E00E94405E74
:1042300017EFA12E14E0B12EBAE3FB2E0DE510E02E
:10424000A8E3EA2EF501819191915F0180509C4F86
:10425000B8010E94A46DD62ED394CE2CCD188F2DEC
:104260006C2D4D2D0E94445E8F2D8F5F6C2D4D2D3A
:104270000E94445E8F2D8E5F6C2D4D2D0E94445EFA
:10428000F5E0FF0E8F2D8934E9F60F900F90CF9156
:10429000DF911F910F91FF90EF90DF90CF90BF9033
:1042A000AF9008954F925F926F927F928F929F92FC
:1042B000AF92BF92CF92DF92EF92FF920F931F9334
:1042C000DF93CF930F92CDB7DEB7B82E8BEF9AE086
:1042D0000E94EF198BE798E06B2D45E020EE37E068
:1042E00006E0EE24E3940E94F01E10927B081FE586
:1042F000E12E18E0F12EB1E5CB2EB8E0DB2E8601E1
:10430000470160E0862F69830E948215D4014D9198
:104310005C911197282F392F6981421753070CF4AC
:104320009A01F401219331934F01D8014D915C9191
:104330001197282F392F241735070CF49A01F8010B
:10434000219331938F016F5F6730E1F680915008C0
:1043500080932005FB2DF03219F0FF3B71F40BC068
:104360008F5F80935008833041F487E10E945E6D37
:1043700081E00E948457109250088091500881304B
:10438000B1F0813020F0823009F0A4C03FC08CE051
:1043900060E149EE5AE021E100E00E94635D82E1C4
:1043A00068E149ED5AE02FE00E94635D93C08EE121
:1043B00060E14CEC5AE02CE000E00E94635D82E199
:1043C00068E14AEA5AE020E10E94635DADE68A2E88
:1043D000A8E09A2E20E008E91AE3F8E6AF2EF5EC03
:1043E000BF2ED7010D931D937D01F601A192B192CD
:1043F0006F01822F29830E948215D4018D939D9392
:104400004D0129812F5F273061F764C082E160E1AF
:104410004BEB5AE020E100E00E94635D82E168E13D
:104420004AEA5AE020E10E94635DEDE6AE2EE8E044
:10443000BE2E73E4472E71E0572EF20160E4862E03
:10444000912CD7018D919D917D01D6016D907D902C
:104450006D019C012619370937FF03C0309521955E
:104460003F4F23333105DCF0D5012D913C91318351
:1044700020838901081B190BC801B4010E94A46D97
:10448000061B170B17870687C301821B930B9C0122
:10449000B4010E94A46D261B370B358F248FA2E038
:1044A000B0E0AA0EBB1E3296BDE6EB16B8E0FB06E6
:1044B00041F680E090E0F201219131912F01820FCD
:1044C000931FFBE54F16F1E05F06A9F790936E018D
:1044D00080936D010E946D200F90CF91DF911F910D
:1044E0000F91FF90EF90DF90CF90BF90AF909F9093
:1044F0008F907F906F905F904F900895282F30E0BD
:10450000C901880F991FA90163E0440F551F6A95DF
:10451000E1F7840F951FA9014F5F5F4FBA01660F46
:10452000771FA3E0440F551FAA95E1F7640F751F8D
:1045300064547E4F20953095205E3F4FA901440F73
:10454000551FE3E0220F331FEA95E1F7420F531F97
:1045500084549E4F0E94096E8AE0E2EFF2E0DF0190
:104560001D928A95E9F782E00E9484570E942058A4
:1045700008950F931F93CF93DF93282F30E0E90125
:10458000CC0FDD1FC90113E0880F991F1A95E1F7C1
:10459000C80FD91F8E0104541E4FA9014F5F5F4FF2
:1045A000CA01880F991FA3E0440F551FAA95E1F790
:1045B000840F951F20953095205E3F4FA901440F31
:1045C000551FE3E0220F331FEA95E1F7420F531F17
:1045D00084549E4FB8010E94096E8AE0D8011D9252
:1045E0008A95E9F780919F08CE55DE4F8A8F8B8F91
:1045F00084E68C8F82E00E9484570E942058DF91CD
:10460000CF911F910F910895FF920F931F9385EF04
:10461000E3E4F5E0DF011D928A95E9F78091380621
:10462000ACEBB1E050E021E030E060E07C9177233A
:1046300011F0472F01C040E1641738F5F22E032F27
:10464000162F1F5F802F90E0FC01EE0FFF1FEE0F73
:10465000FF1FE80FF91FED5BFA4F912F9F738081C9
:10466000807C892B80648083F182F39453830F5F75
:10467000141738F3962F9095642F822F8F5F890F30
:10468000390F340F290F240F840F772359F1832F0B
:1046900090E0FC01EE0FFF1FEE0FFF1FE80FF91F68
:1046A000ED5BFA4F4F738081807C5483842B80684C
:1046B000808322832F5F1A968C911A97781719F4AA
:1046C0001182138205C021832F5F852F8F5F838323
:1046D000822F5F5F1A96503219F42093380604C077
:1046E0003F5FA4CF809338061F910F91FF900895EC
:1046F000ECEBF1E080E090819150903108F48F5F15
:104700003A9692E0EC3FF907B1F708951F93182FFE
:1047100080E169EE7DE00E94BA5D0E947823482F17
:1047200088E760E150E020E00E94D65F80E263ED20
:104730007DE00E94BA5D113651F481E60E949F61CE
:1047400081E00E94BB1486E494E20E94F0141F9161
:1047500008950E947823803230F086E893E20E9428
:10476000F01481E0089580E00895EF92FF920F9396
:104770001F93DF93CF9300D0CDB7DEB7182F8132D0
:1047800008F07BC0882319F4442341F476C08032BA
:1047900019F4442331F071C0442319F0012F0F5F45
:1047A00002C0012F0150812F4A8369830E94840E29
:1047B0007C01802F0E94840EFC01D7018C91982FE0
:1047C00091504A816981903108F057C02081213190
:1047D00008F053C06623A1F10E94A923882309F0A1
:1047E0004CC0212F30E0A9014F5F5F4FCA01880FF5
:1047F000991F13E0440F551F1A95E1F7840F951F79
:10480000B901660F771FA901A3E0440F551FAA95B0
:10481000E1F7640F751F64547E4F20953095205E3C
:104820003F4FA901440F551FE3E0220F331FEA95C4
:10483000E1F7420F531F84549E4F0E94096E1DC022
:10484000281759F0442331F08031B8F48F5FF70115
:10485000808313C0D7019C9310C0D701CF010A9663
:1048600004C020813C9131932D93E817F907C9F7D3
:1048700082E00E9484570E9420580F900F90CF91A1
:10488000DF911F910F91FF90EF9008956F927F92AB
:104890008F929F92AF92BF92CF92DF92EF92FF9250
:1048A0000F931F93CF93DF93182F8DEC9DE00E9401
:1048B000EF19E0903806EA9482EA98E0612F44E02C
:1048C0002CEC37E00AE00E94F01EC090A208CC2039
:1048D00011F41092A1081236D9F1133670F4133482
:1048E000A9F1143420F4123409F070C031C010362C
:1048F000C1F0113609F06AC045C0103809F452C041
:10490000113820F4133609F061C020C01E3BB9F104
:104910001F3B09F05BC081E08093A0081092A108C2
:104920002EC01C143CF481E09091A108911180E00C
:104930008093A1088091A1088093A00880919D0890
:10494000882309F443C01092A10840C01092A00827
:104950008091A1088823D1F141E0123609F040E0AE
:1049600080919E086091A0080E94B5238091A008C4
:10497000882319F0133609F4CA941092A0080E94F3
:10498000042324C08091A108882301F180919E080E
:104990000E947E221092A1080E94042381E60E94B8
:1049A0009F6114C01C1494F480919D08882341F0E9
:1049B0000E94A923882321F480919E080E94B92295
:1049C0001092A1088AEF91E50E94F01438E0D32EEE
:1049D00077247A9423E6822E9924BB24BA94662401
:1049E0006394E0901D05E90CFF24F701EE0FFF1F13
:1049F000EE0FFF1FEE0DFF1DED5BFA4F4081842F80
:104A0000807C09F462C146FF06C04F7380E06D2DC3
:104A100020E00E94510F1C14E4F4E701CC0FDD1FCD
:104A2000CC0FDD1FCE0DDF1DCD5BDA4F8981C8169F
:104A300081F46D2D695F80E048E10E94405E8B81CA
:104A400080939E0888818F7380939F0860929D0851
:104A5000B92CF701EE0FFF1FEE0FFF1FEE0DFF1D2C
:104A6000ED5BFA4F808187FF05C19481C92FDD2757
:104A7000C7FDD095AA24A3949281C912AA2486FDC9
:104A80001FC0FE01EE0FFF1FCE01A3E0880F991F8C
:104A9000AA95E1F7E80FF91FED53FE4F40814695C7
:104AA000477050E04753524F8091A108882311F47A
:104AB00000E001C00A2D82E16D2D21E00E94635DBE
:104AC000FE01EE0FFF1FCE0163E0880F991F6A956C
:104AD000E1F7E80FF91FEE55FE4F448D552747FDCE
:104AE00050958DE26D2D2A2D0E94D65F8091A108F0
:104AF000882311F420E001C02A2D8DE26D2D45E2BE
:104B00000E94A05CFE01EE0FFF1FCE0143E0880F64
:104B1000991F4A95E1F7E80FF91FEE55FE4F438DB7
:104B20008091A108882311F420E001C02A2D86E39A
:104B30006D2D0E94250FFE01EE0FFF1FCE0123E019
:104B4000880F991F2A95E1F7E80FF91FEE55FE4FE0
:104B5000458D442359F08091A108882311F420E069
:104B600001C02A2D8EE46D2D0E94710FFE01EE0F03
:104B7000FF1FCE01B3E0880F991FBA95E1F7E80F48
:104B8000F91FEE55FE4F468D442391F023E0429FDE
:104B9000A00111244352504F8091A108882311F4A1
:104BA00000E001C00A2D86E66D2D23E00E94635DC2
:104BB000FE01EE0FFF1FCE0173E0880F991F7A955B
:104BC000E1F7E80FF91FE454FE4F21E085818823C7
:104BD00009F420E0FE01EE0FFF1FCE0153E0880F25
:104BE000991F5A95E1F7E80FF91FE454FE4F8681AB
:104BF000882329F0222309F498C04AE203C0222323
:104C000061F044E480911E05882311F420E001C086
:104C10002A2D89E76D2D0E94A05C8A2D813051F5E7
:104C20005E01AA0CBB1C33E0CC0FDD1F3A95E1F707
:104C3000AC0EBD1EE2EAF1E0AE0EBF1E812FF50103
:104C4000648D43E82DE70E949314F501848FF701EA
:104C5000EE0FFF1FEE0FFF1FEE0DFF1DED5BFA4F76
:104C6000848180939E0880818F7380939F08109227
:104C70009D08B92CF701EE0FFF1FEE0FFF1FEE0D81
:104C8000FF1DED5BFA4F8181882331F088150CF40C
:104C9000882E87150CF0782EF701EE0FFF1FEE0F10
:104CA000FF1FEE0DFF1DED5BFA4F8281882331F06F
:104CB00088150CF4882E87150CF0782E9394F8E064
:104CC000DF0E292D273009F08CCECC20A1F08B2DC2
:104CD0008F3FF9F4C81464F480911D0590E00197AA
:104CE000EFEF8F3F9E0711F480E090E080931D0569
:104CF0007C14ECF414C0FB2DFF3F59F480911D058A
:104D000090E001972FEF8F3F920761F480E090E0F1
:104D100009C08B2D86305CF0992D983040F0809141
:104D20001D058F5F80931D0502C043E56BCFDF91AA
:104D3000CF911F910F91FF90EF90DF90CF90BF9098
:104D4000AF909F908F907F906F9008952F923F9299
:104D50004F925F926F927F928F929F92AF92BF928B
:104D6000CF92DF92EF92FF920F931F935C01CC24BE
:104D7000DD243B018824992464E6262E312C412C25
:104D8000512CC201B1016619770988099909A60158
:104D900095010E94656D7B018C0182E390E0A0E0AB
:104DA000B0E0E80EF91E0A1F1B1FC601B5010E94E4
:104DB000656D0E94656DBC0188279927A401930148
:104DC0000E94656D44E096958795779567954A951D
:104DD000D1F7E60EF71E081F191FC801B701A2017F
:104DE00091010E94B76DC9011F910F91FF90EF9043
:104DF000DF90CF90BF90AF909F908F907F906F90FB
:104E00005F904F903F902F9008951F93CF93DF9323
:104E10009C016115710511F1132F111F1127111F2D
:104E200019F0309521953F4F77FF0EC0C0E0D4E0D8
:104E3000709561957F4FCE01821B930B0E94A62631
:104E40009E01281B390B05C0C9010E94A626282FE8
:104E5000392F112319F0309521953F4FC901DF916A
:104E6000CF911F9108956F927F928F929F92AF92F0
:104E7000BF92CF92DF92EF92FF920F931F93DF9337
:104E8000CF93CDB7DEB7982E962F322F802F6E2D71
:104E9000222359F0442361F440919A0450919B04D9
:104EA0004115510539F421E001C020E0FF2405C07F
:104EB00022E001C021E0FF24F394332311F091118B
:104EC00021E04A2D433679F44C2D50E0440F551F14
:104ED0008A0173E0000F111F7A95E1F7041B150B8F
:104EE000085A1C4F11C0FA2DF236D9F44C2D50E05F
:104EF000440F551F8A0193E0000F111F9A95E1F7A7
:104F0000041B150B075A1C4FF80140810E94710FBA
:104F1000FF2009F463C0F8016081892D4AEE26E183
:104F200059C069887724BB24882051F54C2D50E066
:104F3000440F551F6A01B3E0CC0CDD1CBA95E1F7B4
:104F4000C41AD50AAA0CBB1CAA0CBB1CCA0CDB1CBD
:104F5000C60CD71C4CE453E0C40ED51EF6014081AC
:104F6000552747FD50950E94D65FFF20B9F1F60105
:104F70006081892D4CE924E60E949314F6012DC02E
:104F8000DD24AA0CBB1CA601E3E0440F551FEA95E3
:104F9000E1F74C195D09A40EB51EA80CB11CAA0CB2
:104FA000BB1CF301EA0DFB1DE45BFC4F4081552760
:104FB00047FD50954C595F4F0E94D65FFF2071F01E
:104FC0008501060D171D045B1C4F892DF8016081BA
:104FD0004CE920E00E949314F8018083CF91DF9187
:104FE0001F910F91FF90EF90DF90CF90BF90AF9007
:104FF0009F908F907F906F9008952F923F924F9245
:105000005F926F927F928F929F92AF92BF92CF9258
:10501000DF92EF92FF920F931F93DF93CF93CDB761
:10502000DEB72A970FB6F894DEBF0FBECDBFD82EDD
:1050300080EC9DE00E94EF198BE998E06D2D40E037
:1050400020E030E000E078ECE72E7DE0F72ECC2485
:1050500053E0A52E0E94671B409193084F5F80E3A9
:1050600060E020E00E94250FF0909B08809193085B
:1050700090E0880F991FFC0123E0EE0FFF1F2A9597
:10508000E1F7E81BF90BE85AFC4F808160E040E053
:105090000E944F108823C1F08091930890E0880F00
:1050A000991FFC0113E0EE0FFF1F1A95E1F7E81BB3
:1050B000F90BE75AFC4F808160E040E00E944F10FE
:1050C000882321F411E003C010E001C012E06091D8
:1050D0009308462F50E0FA01EE0FFF1FE151FB4FFE
:1050E000808191818A3191051CF010929A0807C045
:1050F0002FEF873E92071CF481E080939A0820915D
:10510000860130E02170307082E090E0821B930BCA
:105110008417950741F4643030F48091B301807FA7
:1051200011F010929A0880E16BEB7DE00E94BA5D6D
:105130000F92EDB7FEB7319621E0F11020E080919B
:105140009A0880838D2D61E041E006E3A0E1EA2E1C
:10515000C0909308A12E88240E9433270F9088E1E5
:1051600064EB7DE00E94BA5D0F92EDB7FEB7319619
:1051700021E03F2D313009F020E080919A088083B2
:105180008D2D61E041E006E3F8E1EF2EC090930839
:10519000A12E882483940E9433270F9080E26EEA28
:1051A0007DE00E94BA5D0F92EDB7FEB7319621E027
:1051B0008F2D823009F020E010828D2D61E041E0DA
:1051C0000EE1E0E2EE2EC090930873E6A72E88244D
:1051D0000E9433270F9088E268EA7DE00E94BA5D62
:1051E0000F92EDB7FEB7319621E09F2D933009F075
:1051F00020E010828D2D61E041E00EE158E2E52EC5
:10520000C090930832E6A32E88240E9433270F9083
:10521000113019F0123049F404C080E361EA7DE0F6
:1052200007C080E36AE97DE003C080E362E97DE0D6
:105230000E94BA5D00919308402F50E0812F90E0CA
:10524000880F991F880F991FBA01660F771F9B015E
:10525000B3E0220F331FBA95E1F7261B370B820FFD
:10526000931F8E559E4FFC01E655FE4FA081A983EA
:10527000FC01E555FE4FB081BA83FC01E455FE4FB9
:105280009080E4E69E0E83559E4FDC018C908E0E3E
:105290002091860130E02170307082E090E0821B26
:1052A000930B8417950709F062C0043008F05FC0C3
:1052B0008091B301807F09F45AC0EE24FF24870156
:1052C00020E030E0B9816B2E772467FC7094A1E276
:1052D0004A2E512C292C332427FC3094F0E4CF2E75
:1052E000D22ED801C701B595A79597958795B3019B
:1052F00029873A870E940527880F991FB2010E94CB
:10530000A46D629DC001639D900D729D900D11244E
:105310006FE3A62EAD0C64E670E00E94906DEC2D5C
:10532000E61B6E2F8A2D0E94F45D29853A85C901FE
:1053300083709070009761F48A2D6FE30E94F45D92
:105340006D2D6695605E8FE30E94F45D3A85298538
:105350002F5F3F4F81E290E0A0E0B0E0E80EF91E41
:105360000A1F1B1F2E33310509F0BACF7CC0DD2484
:105370009981492E552447FC509401E210E0A92D53
:10538000BB27A7FDB095BC83AB8354E6652E712C7B
:1053900040E2A42EBA812B2E332427FC3094E82D32
:1053A000FF27E7FDF095FE83ED83FD2D21E2F29FBF
:1053B00070011124C701B2010E940527B8010E94A3
:1053C000A46DAB81BC816A9FC0016B9F900D7A9FD9
:1053D000900D11243EE5C32ECD0CB3010E94906DBB
:1053E000BA2DB61B6B2F8C2D0E94F45DED2DF0E0D5
:1053F000E370F070F887EF83309749F48C2D60E20A
:105400000E94F45D6D2D605E8EE50E94F45DC70123
:10541000B1010E940527B8010E94A46D2D813E8133
:10542000629FC001639F900D729F900D11242EE525
:10543000F22EFD18B3010E94906D605E8F2D0E94C8
:10544000F45D8F819885009749F48F2D60E20E946A
:10545000F45D6A2D6D198EE50E94F45DD3949D2D47
:105460009F3109F0A2CFE0919308F0E0EE0FFF1F0B
:10547000E151FB4F408051805201CC24B7FCC094D5
:10548000DC2CC601B50121E230E040E050E00E9492
:10549000D96D822F825A61E04EE30E94445E4091B2
:1054A00093082091860130E02170307082E090E016
:1054B000821B930B242F30E08217930709F050C012
:1054C000443008F04DC08091B301807F09F448C09A
:1054D000C601B50160507C4F8F4F9F4F22E030E0F6
:1054E00040E050E00E94D96DA9816A2F772767FDBF
:1054F0007095C9010E940527BC01660F771F882798
:1055000077FD8095982F292D97FC2D5F2595259562
:10551000332727FD3095432F532F0E94656D29E1D6
:1055200030E040E050E00E94D96D79018A01CA0163
:10553000B9012FED3FEF4FEF5FEF0E94D96D622F62
:10554000605C8FE34EE30E94405EC801B70122E039
:1055500030E040E050E00E94D96D79018A013CC002
:105560001A141B041C041D0414F4698101C06A810F
:10557000772767FD7095C2010E9405279C0144278B
:1055800037FD4095542F1A141B041C041D0414F4F9
:10559000692D01C0682D67FD6D5F6595659577275D
:1055A00067FD7095872F972F0E94656D29E130E088
:1055B00040E050E00E94D96D79018A01CA01B90129
:1055C0002FED3FEF4FEF5FEF0E94D96D622F605ECE
:1055D0008FE34EE30E94405EC601B50129E130E051
:1055E00040E050E00E94656D612CB1E07B2E812C83
:1055F000912CA40193010E94D96D82E760E3A90177
:1056000020E00E94D65FC801B70129E130E040E008
:1056100050E00E94656DA40193010E94D96D84E55C
:1056200068E0A90120E00E94D65F1A141B041C0444
:105630001D0474F4B9816B2F772767FD7095C20143
:1056400044970E940527F701E81BF90BCF010BC017
:10565000FA816F2F772767FD7095C20144960E94EB
:1056600005278E199F099C01220F331F220F331F1C
:10567000280F391F442737FD4095542F84E560E1FA
:1056800000E3F3E0EF2E0E94A05E2A960FB6F89496
:10569000DEBF0FBECDBFCF91DF911F910F91FF9065
:1056A000EF90DF90CF90BF90AF909F908F907F90C2
:1056B0006F905F904F903F902F9008952F923F9260
:1056C0004F925F926F927F928F929F92AF92BF9212
:1056D000CF92DF92EF92FF920F931F93DF93CF93BE
:1056E000CDB7DEB72F970FB6F894DEBF0FBECDBF94
:1056F000982E88E89DE00E94EF1988E998E0692DCE
:1057000043E02CEC37E00AE0F0E9EF2EFDE0FF2E5D
:10571000CC24C394E4E0AE2E0E94671BF09098085E
:10572000FA9430909908292D203841F4F7FC06C0EE
:10573000F09293088DEF97E20E94F01485E168E003
:1057400048E75DE00E94C25D88E593E09C838B831F
:1057500074E9472E78E0572EEFEEF4E0FB87EA87F6
:1057600010E1662477242F2D332727FD30953A83C7
:105770002983C901880F991FFC0153E0EE0FFF1F19
:105780005A95E1F7E81BF90BFE83ED83F62CEB81CC
:10579000FC81808160E040E00E944F10882361F02E
:1057A000EB81FC81818160E040E00E944F10882302
:1057B00029F4BB24B39404C0BB2402C042E0B42E3D
:1057C0002B2D30E038872F83C901880F991F880F50
:1057D000991FA301440F551F9A0103E0220F331FA5
:1057E0000A95E1F7241B350B820F931F8E559E4FB0
:1057F000DC01A355BE4FFC01E455FE4F3C912081D6
:10580000321751F4FC01E555FE4F86559E4F41E09D
:105810002081FC018081281340E0EA85FB8581918D
:105820009191FB87EA879C0197FF04C022273327C9
:10583000281B390B2A3131050CF040E0242E8A3127
:1058400091051CF0F201108207C0FFEF873E9F0711
:105850001CF421E0F20120838091860190E08170A8
:105860009070E2E0F0E0E81BF90BE615F70551F463
:105870008091B301807F31F0F301EC56F74F108235
:10588000222423944F2D4F5F80E0612F20E00E945F
:10589000250F5D864C86F2013081F1E0F9873111E8
:1058A000198680911E05882351F4DD24D3948091BC
:1058B0009A0490919B04009721F4DD2402C0DD241A
:1058C000D39489819A818615970511F421E03110CE
:1058D00020E00F92EDB7FEB73183892D60E04D2DAA
:1058E00007E2E12ECF2CAB2C88240E9433270F90A7
:1058F00029813A812615370509F0D2C0332009F0F5
:10590000CBC0DD2009F4CCC0222009F4C9C08F81AE
:105910009885880F991F880F991FED81FE818E0F42
:105920009F1F8E559E4FF9858F0F911D86559E4F57
:105930009F878E87892DEE85FF8560814CE924E65F
:105940000E949314EE85FF858083AAC021E00F9208
:10595000F2018081EDB7FEB78183892D60E04D2D86
:1059600009E3E12ECF2CAB2C882483940E943327AB
:105970000F9029813A812615370509F097C0332DFC
:10598000313009F08FC0DD2009F490C0222009F4E5
:105990008DC08F819885880F991F880F991FED8181
:1059A000FE818E0F9F1F8E559E4FF9858F0F911D83
:1059B00084559E4F98878F83892DEF81F88560816C
:1059C0004CE920E00E949314EF81F88580836EC03B
:1059D00021E00F92EDB7FEB71182892D60E04D2DC9
:1059E0000FE3E12ECF2CF3E6AF2E88240E9433275D
:1059F0000F9029813A812615370521F421E0332DB6
:105A0000333009F020E00F92EDB7FEB71182892DF7
:105A100060E04D2D07E5E12ECF2CE2E6AE2E882486
:105A20000E9433270894411C511C0F90EC85FD8582
:105A30008081882319F4222031F008C0222031F41B
:105A40008AE34FE705C08BE34EE702C08AE34DE2ED
:105A5000612F0E945F5DFB2DF13019F0F23049F4A7
:105A600004C085E7612F4DE407C085E7612F4CE452
:105A700003C085E7612F48E40E945F5D0894611CC4
:105A8000711C2B813C81225F3F4F3C832B83185F2D
:105A9000103309F07BCE0CC0332D313009F456CFD2
:105AA00020E055CF832D823009F492CF20E091CFB2
:105AB0002F960FB6F894DEBF0FBECDBFCF91DF910A
:105AC0001F910F91FF90EF90DF90CF90BF90AF901C
:105AD0009F908F907F906F905F904F903F902F900E
:105AE000089520E030E0F901EB5CF24FE491E81713
:105AF00011F4822F08952F5F3F4FEE23A1F780E02E
:105B00000895823430F4E82FF0E0EB5CF24F84919A
:105B1000089580E20895EF92FF920F931F93182F3C
:105B2000F62EE22E862FBA010E94BA5D86E66F2D10
:105B3000412F2E2D0E94221BEE2039F0802F612F45
:105B400040E021E00E94A214182F812F1F910F9195
:105B5000FF90EF900895FF920F931F93F82E1091EE
:105B6000AD01212F332727FD309537FF03C0309536
:105B700021953F4F022F25320CF43DC02091420861
:105B8000309143088091400890914108282B392B8F
:105B90008091440890914508282B392B80913F082B
:105BA00090E0282B392B40913C0850E0242B352BDA
:105BB0002115310531F4812F881F8827881F809394
:105BC0003C0811161CF4812F845202C0812F8C5D79
:105BD00060E040E00E944F10882359F090913C080B
:105BE000992339F491E020913F08211190E090939E
:105BF0003F0880933C0820914208309143082F5F72
:105C00003F4F309343082093420820914008309141
:105C100041082F0D311D30934108209340080E9408
:105C20007C0E2091440830914508821B930B8436EA
:105C3000910508F471C12C593F4F309345082093CA
:105C400044082091400830914108E0914208F091C9
:105C50004308C901BF010E94906DF62E462F50E007
:105C60004E9FC0014F9F900D5E9F900D1124281BE9
:105C7000390B30934108209340081092430810924A
:105C8000420800311CF410923F080FC005326CF43A
:105C900011161CF4812F8F5002C0812F815F60E0AC
:105CA00040E00E944F1080933F0880913B06909106
:105CB0003C06019690933C0680933B0640913D063E
:105CC00050913E064F5F5F4F50933E0640933D0616
:105CD000FF2049F0809141069091420601969093F1
:105CE00042068093410680913F08882349F08091C5
:105CF0003F069091400601969093400680933F06A0
:105D0000F69420914306309144062F0D311D3093B7
:105D10004406209343068091AF019091B001909387
:105D20004706809346066091AD01772767FD709521
:105D300077FF03C0709561957F4F662319F4109229
:105D400045061EC0613019F4841B950B15C06031E7
:105D500068F460FF06C0A4E036952795AA95E1F7A0
:105D600009C0209141063091420604C020913F06AF
:105D700030914006821B930B909347068093460612
:105D800080914506813051F0813018F0823049F51C
:105D900014C08091AD01882321F120C08091460676
:105DA0009091470618161906E4F08091AF01909182
:105DB000B0010097B1F082E012C080914606909148
:105DC00047062FEF853C92071CF483E0809345063D
:105DD0008091AF019091B001009719F481E0809318
:105DE0004506809146069091470620913D083091E6
:105DF0003E082817390709F479C02091450621305B
:105E000009F065C02091880122FF45C02091AF01B3
:105E10003091B00121153105F1F18E31910519F460
:105E200089E10E945E6D809146069091470684311B
:105E3000910519F48AE10E945E6D80914606909169
:105E400047068A30910519F48BE10E945E6D8091BE
:105E5000460690914706843091051CF48CE10E941F
:105E60005E6D8091880183FF16C0809146069091F7
:105E700047068E31910549F08431910531F08A3021
:105E8000910519F08430910534F482E390E0909309
:105E90009E0480939D048091880181FF27C080919A
:105EA000AE01209146063091470680FF07C08091E1
:105EB000AF019091B001821B930B01C0C9016CE34B
:105EC00070E00E94906D009789F480E003C022305A
:105ED00069F48CE10E945E6D8091880183FF06C0A9
:105EE00082E390E090939E0480939D042091460667
:105EF0003091470630933E0820933D088091AE01D3
:105F000080FF0AC08091AF019091B001821B930B7A
:105F100090934706809346061F910F91FF90089536
:105F20008091AD01992787FD909597FF03C09095CB
:105F300081959F4F982F823034F1803124F58595DB
:105F40009A3024F40E94C36290E003C0992787FD31
:105F500090950197FC01EE0FFF1FE151FB4F20814F
:105F600031818091AD0187FF05C080E094E0821B04
:105F7000930B03C0C90180509C4F26E096958795EE
:105F80002A95E1F702C080E090E00E94AB2D83E00B
:105F90000E94C362E82FF0E0EE0FFF1FE351FB4FBA
:105FA0008081918180509C4FB6E096958795BA95F7
:105FB000E1F72091AE0122FF0AC08530910538F04B
:105FC0002091A004222319F423E02093A00420911F
:105FD0003808309139082F5F3F4F309339082093AC
:105FE00038082091360830913708280F391F309330
:105FF0003708209336080E947C0E20913A08309191
:106000003B08821B930B23E0883E9207E8F10E9435
:106010007C0E90933B0880933A088091B1018230C6
:1060200051F485E160E040E00E944F10882319F0B0
:1060300087E00E945E6D80913608909137086091EC
:106040003808709139080E94906D109237081092AC
:10605000360810923908109238088091C106909144
:10606000C20601969093C2068093C1068091C00635
:10607000E82FF0E0E85BF94F60838F5F8093C00604
:10608000883710F01092C0060895109245061092BD
:106090003E0610923D061092420610924106109262
:1060A000400610923F06109244061092430608954F
:1060B0000F931F93182F80913906882319F065E2FA
:1060C0007DE002C068E17DE088E00E94BA5D81E089
:1060D00060E142EA51E02AE000E10E94635D82E46F
:1060E00060E14FE30E945F5D82E168E241E15DE0D3
:1060F0000E94C25D82E160E342E05DE00E94C25D19
:10610000113609F44AC01F3B21F0103609F04FC088
:1061100004C080E00E945E6D4AC0809139068823E9
:10612000A9F080EF9CE00E94851280913A060E94BF
:10613000EC56882339F087E10E945E6D82E08093FF
:10614000390629C080E00E945E6D25C080916F01F4
:106150008F5F0E94B05910916F0108C0115011312A
:1061600008F01FE080916F01181739F0812F8F5FC1
:106170000E946359882391F301C010E010936F01CE
:1061800081E00E9484570E94205880916F010E94F4
:10619000B5560E94453080E601C081E60E949F61AD
:1061A00081E00E94BB148AED90E30E94F0141F91DD
:1061B0000F910895AF92BF92DF92EF92FF920F93EB
:1061C0001F93CF93DF93182F8CE09BE00E94EF1971
:1061D00080911E058823A1F4E0912105E7FF10C0FE
:1061E000E195EA3008F0E9E0F0E0EE0FFF1FE4533C
:1061F000F84F25913491C9010E94E01410922105B5
:10620000F0908D088DE898E0612F4FE00E946120AA
:1062100086E360E047E05BE00E94C25D0E94A55813
:10622000AC0186E660E020E00E94D65F80E06AE094
:1062300041E00E94421BD0908D0880913906823047
:1062400021F410928C0810923906163648F4143650
:1062500090F5103609F456C0113609F075C00AC021
:10626000113809F456C01F3B09F465C0103809F015
:106270006BC053C080918C088823E9F010928C0881
:1062800087E10E945E6D81E60E949F610E94205816
:1062900080918D0880936F010E94B5560E94453011
:1062A00081E00E9484570E94205882E00E94845717
:1062B0000E94205849C080916F018D15B9F0812F3F
:1062C0000E949F6180918D0880936F010E942058E9
:1062D00080916F010E94B5560E94453081E00E9476
:1062E00084570E94205881E00E945E6D153619F493
:1062F0008AE490E504C0143639F583E193E40E9402
:10630000E01422C081E080938C0887E10E945E6DDA
:106310001BC081E00E94BB1417C080918C088823A9
:1063200099F081E080933906D0923A0688E590E3AF
:106330000E94F01409C010928C0880916F01809324
:106340008D0881E00E94925780918C08882341F04B
:10635000FD1431F06D2D6F5F8F2D8F5F0E9471598D
:10636000CD2DDD27C7FDD09580911D059E01281BF1
:106370003109C901181619065CF0CE01019797FF83
:1063800002C080E090E080931D0510E1DD240BC089
:1063900025303105D4F3CE0104978B3091059CF361
:1063A0008AE090E0F0CFF0901D05FD0CAF2CBB24EF
:1063B00095012F5F3F4F442737FD4095542FCA1555
:1063C000DB0511F401E101C000E182E1612F72E01F
:1063D000E72E0E94A05E80916F01F81629F481E0FB
:1063E000612F4AE20E945F5D8F2D6DE778E04FE0FC
:1063F0000E946D56CA15DB0531F480918C08882304
:1064000011F001E101C000E188E1612F4DE758E0A2
:106410002FE00E94635DD394185F3D2D363019F64E
:10642000DF91CF911F910F91FF90EF90DF90BF9080
:10643000AF900895AF92BF92CF92DF92EF92FF920A
:106440000F931F93CF93DF935B016C0110E1E12E5B
:10645000F12CC0E0D0E800E010E89E0140E050E000
:10646000CA01B9010E94656DA616B706C806D9060D
:1064700010F4C027D127169507950894E108F10874
:10648000E114F10461F4CE01DF91CF911F910F91DE
:10649000FF90EF90DF90CF90BF90AF900895C02B0A
:1064A000D12BDBCFE1E0683068F4E0E070E09B01E5
:1064B000220F331F220F331F260F371FA901485702
:1064C0005C4F0EC070E0685070409B0153E0220F9B
:1064D000331F5A95E1F7260F371FA90140555C4F2E
:1064E000DA012C9180509C4F97FD0FC0B8E08030AE
:1064F0009B078CF0EE2319F028E030E002C024E086
:1065000030E0240F351FF9012081332727FD309516
:10651000322F222730C0EE2329F0692F9070880F88
:10652000991F03C0692F66959170262F30E0FA01FC
:10653000E20FF31F6181772767FD7095AC015595D8
:106540004795649F9001659F300D749F300D112415
:106550006081772767FD709540E052E0481B590B3A
:1065600055954795649FC001659F900D749F900D50
:106570001124280F391FC90169E170E00E94A46D40
:10658000CB0108952F923F924F925F926F927F922C
:106590009F92AF92BF92CF92DF92EF92FF920F93B2
:1065A0001F93DF93CF9300D00F92CDB7DEB7182F94
:1065B000992493948091A408883008F4992487EC56
:1065C0009FE00E94EF19992011F05AE001C056E0B7
:1065D00082EC98E0612F40E020E030E000E07DECCC
:1065E000E72E7FE0F72ECC24C394A52E0E94671BD4
:1065F0004091A40850E04F5F5F4F84E260E021E0EB
:106600000E94D65F8091A408992079F090E00897C5
:106610007C0103E0EE0CFF1C0A95E1F7E80EF91E81
:1066200020EB33E0E20EF31E0CC090E07C01EE0C98
:10663000FF1CEE0CFF1CE80EF91E88E893E0E80E44
:10664000F91E0091C2080150D090C308113661F0C4
:10665000123628F41434D1F0153471F50EC0143606
:10666000A9F0153649F509C0DD2031F11092C308B3
:1066700081E60E949F61DD241FC080911E05882352
:10668000D9F01D14CCF48D2D815014C080911E05BD
:10669000882391F02D2D332727FD3095992019F06F
:1066A00089E090E002C085E090E02817390724F4E3
:1066B0008D2D8F5F8093C3088091C30880931E0542
:1066C000CE2C4F2C6E2C7F2C90E122243324A02E34
:1066D000BB24A7FCB094F30141913F01552747FD2E
:1066E000509521E0A214B30409F020E088E1692F5D
:1066F00099830E94D65F0894211C311C9981985F70
:10670000983349F7992001F1A5E06A2E712C6E0C9F
:106710007F1C90E1F5E02F2E312CF30141913F01D8
:10672000552747FD509521E0A214B30409F020E05D
:1067300080E3692F99830E94D65F0894211C311C45
:106740009981985F903349F70F3F11F421E0D11000
:1067500020E08CE068E040EC5FE00E94935D9920CF
:1067600019F089E090E002C085E090E021E0A816F1
:10677000B90609F020E08CE068E349EB5FE00E9495
:10678000935D992019F089E090E002C085E090E0E7
:10679000A816B90694F407FD4EC0A02EBB24A7FC92
:1067A000B094AE0CBF1C812FF50160814CE924E64A
:1067B0000E949314F50180833EC01016E4F5812FEA
:1067C0006091C1084CEF24E000E00E9485148093A2
:1067D000C10890919704992371F1992021F050E11B
:1067E00094E049E003C058E092E045E024E68202EC
:1067F00030011124892F90E0909581959F4F869DBF
:106800009001879D300D969D300D1124EC2DF42DB7
:10681000A52E00E0C9016A2D702F0E94A46D61931E
:10682000260D371D8E2F8C198417A0F382E00E944D
:1068300084570E94205880911E05882351F0AA2475
:10684000ECE92E2EEFEF3E2E4D2C552447FC5094B4
:10685000A5C000E01CEFAA24BB2470E2D72EACC078
:10686000C90165E0880F991F6A95E1F7992019F031
:1068700064E070E002C062E070E00E94A46D462F08
:10688000062F055C37016A0C711CF3018081992782
:1068900087FD909555E0880F991F5A95E1F7B10152
:1068A0000E94A46D562F90E2D92ED60E2F5F3F4F37
:1068B0008D2D90E09B838A834216530609F050C0C9
:1068C00082349105ACF48AE3C82EC40E625E8C2D2E
:1068D00045E059830E94405E5981EA81FB81E134A1
:1068E000F10531F0652F615E8C2D45E00E94405E20
:1068F000FD2DF03430F4802F81506D2D45E00E9445
:10690000405E2A813B812F33310594F401506D2D77
:106910006F5F802F45E00E94405E8A819B818E33AD
:10692000910531F06D2D6E5F802F45E00E94405E35
:1069300080919A0490919B04009741F4123631F0B3
:10694000133621F0123411F0133439F5812FF3018D
:1069500060814CE924E60E949314F30180831DC0FA
:106960002A813B81213431052CF4615E802F43E084
:106970000E94405E3D2D303428F4802F6D2D43E081
:106980000E94405E8A819B818F33910534F46D2D86
:106990006F5F802F43E00E94405EA3942A2D30E079
:1069A000992019F089E090E002C085E090E0281776
:1069B00039070CF455CF4DCFC8016091A4080E944F
:1069C0005232BCE3EB2EEA0C9C01A5E036952795EC
:1069D000AA95E1F76D2D621B8E2D0E94F45D950145
:1069E000237030702115310521F48E2D60E20E9454
:1069F000F45D0894A11CB11C005E1F4F90E4A91621
:106A0000B104D1F68CE560E040E40E94445E0F9052
:106A10000F900F90CF91DF911F910F91FF90EF900A
:106A2000DF90CF90BF90AF909F907F906F905F90DE
:106A30004F903F902F9008952F923F924F925F92E8
:106A40006F927F928F929F92AF92BF92CF92DF927E
:106A5000EF92FF920F931F93DF93CF93CDB7DEB7E3
:106A6000A2970FB6F894DEBF0FBECDBF8F8F98A34D
:106A70006A8B80919C04882309F474C080911F055F
:106A8000882319F0815080931F058091C906909149
:106A9000CA062091C7063091C806820F931F209125
:106AA000CB063091CC06820F931F2091CD063091FA
:106AB000CE06820F931F20915207309153072C016D
:106AC000421A530A920157FE03C0309521953F4F59
:106AD00041E0213034073CF09093530780935207F4
:106AE00081E080939F0480918701863FD9F1909146
:106AF00008019233B8F190914F079F5F90934F0731
:106B0000903160F020915007309151072F5F3F4F37
:106B1000309351072093500710924F0790919F0494
:106B2000992321F01092510710925007209150079D
:106B300030915107992787FD90950A9667E771E094
:106B4000869FA001879F500D969F500D11244217DC
:106B5000530740F4237030702130310519F480E17F
:106B60000E945E6D80918601582F51705F5F59873A
:106B700081FF02C01D8602C063E06D876090BA018C
:106B8000662009F44AC08985E82FF0E0EE0FFF1F68
:106B9000E151FB4FA080B180CC24B7FCC094DC2C29
:106BA0009D85E92FF0E0EE0FFF1FE151FB4F2081A3
:106BB0003181442737FD4095542FCA01B9010E9405
:106BC000656D7B018C01C601B501A60195010E948E
:106BD000656DE60EF71E081F191F662D70E080E038
:106BE00090E0EAE0660F771F881F991FEA95D1F7BA
:106BF00024E630E040E050E00E94D96DB901CA01BE
:106C00000E94656D6E157F058007910730F4C801FD
:106C1000B7010E941A324C0102C088249924B401A1
:106C200080E090E024E630E040E050E00E94656DB6
:106C30006B8F7C8F8D8F9E8F62E4662E61E0762E47
:106C4000A7ECB6E0BE8BAD8BFE013196F88FEF8BD3
:106C500050E0252E51E0352E22EA31E03F872E8785
:106C60004FEE54E05A8F498F2901F98BE88BBC8B8A
:106C7000AB8BEE24FF241B865A89517059A3AE2C8E
:106C80008E2D0E9482159C01D30111968D919C91AD
:106C90001297281B390BB901882777FD8095982F0B
:106CA0004AE0660F771F881F991F4A95D1F7121681
:106CB00013062CF45D962D913C915E9703C0F30171
:106CC000278530892436310514F424E630E0442742
:106CD00037FD4095542F0E94D96D8901FCEF21307A
:106CE0003F072CF024E00030120724F405C000E038
:106CF0001CEF02C000E014E08091880180FF0FC00B
:106D00008091860190E08170907042E050E0481BD5
:106D1000590BE416F50619F4109501951F4FA98D2E
:106D2000BA8D0D931D93BA8FA98FC8010F968F311D
:106D30009105F0F4B4E0EB16F1047CF48A2D8F5F3A
:106D40000E94C36290E00197E1E0F0E002C0EE0F24
:106D5000FF1F8A95E2F7CF0108C081E090E00E2C7A
:106D600002C0880F991F0A94E2F7FB85F82BFB8776
:106D70002A2D243008F07AC139A1332309F05FC0ED
:106D80008091AE0181FF5BC06701CC0CDD1C4CE73C
:106D900051E0C40ED51ED60111968C911197807CBE
:106DA00009F44DC08C9185958595859561E040E00D
:106DB0000E944F10882309F442C0D601EC91E7707D
:106DC000F0E0DF01AA0FBB1FAC55BB4FEE0FFF1F5A
:106DD000EC58FE4F8D919C91119720813181821B3F
:106DE000930B62E070E00E94A46DF701EE0FFF1FAD
:106DF000E358FE4F2081422F440F440F459545959F
:106E0000552747FD5095649FC001659F900D749F65
:106E1000900D11246FE170E00E94A46D660F771F42
:106E2000660F771F2295269526952370213019F03D
:106E3000223029F403C0060F171F01C08B018114F3
:106E4000910409F1B985AB1619F0ED85AE16D9F4A8
:106E50006091BA0170E080E090E04AE0660F771F31
:106E6000881F991F4A95D1F79801442737FD40950F
:106E7000542F0E94656D2B8D3C8D4D8D5E8D0E9433
:106E8000D96D022F132FF201EA54FE4F808160E08A
:106E900040E00E944F10882369F0F201E954FE4F50
:106EA000808160E040E00E944F10882329F4CC24C8
:106EB000C39404C0CC2402C032E0C32E809186016A
:106EC00090E08170907022E0A22EB12CA81AB90A2D
:106ED000AE14BF0469F58091B301807F49F1C80108
:106EE00080509C4F62E070E00E94A46D9B01EC2DED
:106EF000F0E0EE0FFF1FEE0FFF1FA701440F551F1D
:106F0000CA01A3E0880F991FAA95E1F7841B950B8E
:106F1000E80FF91FE45BFC4F6081772767FD7095F0
:106F2000C9010E940527AC01440F551F30E028C05D
:106F300031E0101611060CF430E08C2D90E0A70122
:106F4000440F551FFA0163E0EE0FFF1F6A95E1F74A
:106F5000E41BF50B880F991F880F991FE80FF91F85
:106F6000EE55FE4FE30FF11DE655FE4F608177278A
:106F700067FD7095C8013AA30E940527AC013AA1AC
:106F8000EC2DF0E0EE0FFF1FEE0FFF1FB701660FB5
:106F9000771FCB0113E0880F991F1A95E1F7861B25
:106FA000970BE80FF91FEE55FE4FE30FF11DE45567
:106FB000FE4F6081772767FD70956C597F4F88275A
:106FC00077FD8095982FDA019D01442737FD409584
:106FD000542F0E94656D24E630E040E050E00E94AE
:106FE000D96D022F132FAE14BF0499F58091B30110
:106FF000982F907F09F466C60050144063C6D101F3
:10700000ED91FC91119760818091880180FD6195DF
:10701000772767FD7095872F972F63587F4F8F4F86
:107020009F4F20E034E0201B310B442737FD409573
:10703000542F0E94656D20E038E040E050E00E944F
:10704000D96D2030B8E03B07B0E04B07B0E05B07FC
:1070500039F4D101ED91FC912081332727FD309542
:10706000220F331FE889F98931832083AB89BC89DA
:107070000D931D93BC8BAB8B0894E11CF11CE2E0DB
:10708000F0E06E0E7F1E288939892E5F3F4F398BC5
:10709000288B2E0E3F1E4EE050E0440E551E57E04A
:1070A000E516F10409F0EBCD0091B7016B850623DD
:1070B000809154078095802319F088E10E945E6DCD
:1070C0000093540780E094E09093D6068093D50611
:1070D0009093D8068093D706E4EAF4E024E731E001
:1070E000AFEDB6E0BD0181919191D9014D915D91D6
:1070F0009D01841B950B880F991FDB018D939D9338
:10710000BD01B4E0EC3AFB0771F78091AC049091BB
:10711000AD04880F991F9093E8068093E70680914D
:10712000AE049091AF04880F991F9093EA06809364
:10713000E9068091B0049091B104880F991F909353
:10714000EC068093EB068091B2049091B304880F13
:10715000991F9093EE068093ED06EFE0F7E0FC8731
:10716000EB872FEE36E04191519161917191D901F8
:107170004D935D939D01B7E0EF34FB07A1F7C090FD
:10718000BA01CC2009F47AC0E985AE2EBB24AA0C42
:10719000BB1C27EC422E26E0522EA40CB51CD501B8
:1071A0002D903C90442437FC4094542CBD850B2FEB
:1071B00010E0000F111F0953194FF8012081318190
:1071C000442737FD4095542FCA01B9010E94656DCF
:1071D0003B014C01C201B101A20191010E94656D08
:1071E000660E771E881E991EDD24EE24FF248AE099
:1071F000CC0CDD1CEE1CFF1C8A95D1F7C701B60133
:1072000024E630E040E050E00E94D96DB901CA01A7
:107210000E94656D661577058805990578F5C401A6
:10722000B3010E941A32BC0180E090E024E630E015
:1072300040E050E00E94656D3B014C01C201B1018C
:10724000A70196010E94656DA40193010E94D96D6A
:10725000D5012D933C93F80160817181882777FDDA
:107260008095982FA70196010E94656DA401930156
:107270000E94D96DD80111963C932E93E090B801ED
:107280008E2D807E09F4DEC0B9852B2F30E0220FD1
:10729000331FF901E953F94F40815181CE01019625
:1072A000280F391FD901ED91FC91BD856B2F70E03E
:1072B000660F771FDB01A953B94F2D913C91860FC3
:1072C000971FDC018D919C91BA89B1FD05C0E40F37
:1072D000F51F280F391F04C020E030E0E0E0F0E0A7
:1072E000A091B901AA2349F0B0E0AA0FBB1FAB538C
:1072F000B94F0D911C91119702C000E010E0E2FE21
:1073000003C0F095E195FF4FE3FE03C03095219552
:107310003F4FE4FE03C0109501951F4F8091B801C7
:10732000829586958770823071F1833020F48130A8
:1073300009F088C007C0833009F459C0843009F0CF
:1073400081C06CC0C90168E070E00E94A46D7B013F
:10735000C90160E870E00E94A46D29014E185F0821
:107360007201E61AF70AC90160E072E00E94A46D9A
:10737000E61AF70AC8018E1B9F0B9093DA068093DA
:10738000D906CF0120C0CF0168E070E00E94A46D53
:107390007B01CF0160E870E00E94A46D3F016E1890
:1073A0007F087301E61AF70ACF0160E072E00E94DD
:1073B000A46DE61AF70AC801821B930B9093DA06B4
:1073C0008093D906C90162E070E00E94A46D600F4D
:1073D000711FCB018E0D9F1D9093DC068093DB0601
:1073E0006E197F097093DE066093DD062BC0C8011D
:1073F0008E1B9F0B9093DA068093D906E00FF11F46
:10740000CF01820F931F9093DC068093DB06E21B73
:10741000F30BF093DE06E093DD0614C0C8018E1B6B
:107420009F0B9093DA068093D906C801820F931FB1
:107430009093DC068093DB06021B130B1093DE0691
:107440000093DD0680919C04882311F00E94902F08
:1074500080E4EFE0F7E0DF011D928A95E9F7BA8951
:10746000B1FF2DC08091860190E08170907022E084
:1074700030E0281B390B80E090E0ED89FE89AF8970
:10748000B88D2817390729F01182108211961C92A5
:107490001E920196329612968430910591F71092C1
:1074A000E0061092DF061092E2061092E1061092BA
:1074B000E4061092E3061092E6061092E50684E8D0
:1074C00093E090930101809300019C012F5F3F4F57
:1074D00030930301209302019C012E5F3F4F3093B4
:1074E0000501209304010396909307018093060100
:1074F00025E1422E28E0522E95E9692E97E0792E5B
:1075000085E5282E87E0382E19861D8689850E94FC
:10751000840E7C01FC0180818150803108F0ADC275
:10752000838161E040E00E944F10D2019C9188234A
:10753000A1F4292F1C92F7019181892F8850823064
:1075400008F08AC287818E70843009F485C2993030
:1075500009F04BC000E01CEF4AC021E0911120E08F
:1075600081E0D2018C93D7011196EC913E2F3150DE
:10757000832F90E0DC01AA0FBB1FA953B94F0D91D7
:107580001C911197343160F0B9853B1748F4DC0148
:10759000AA0FBB1FAA0FBB1FA15FB84F0D911C9173
:1075A000D70117963C911797832F807381F0832F13
:1075B0008295837090E0019741E050E002C0440F53
:1075C000551F8A95E2F7CA015D85582B5D8736FF06
:1075D0000EC0E53060F4F0E0EE0FFF1FE250FF4F09
:1075E000C70108969183808302C000E010E0D701B4
:1075F0001796CC901797C6FC0BC018968C911897CD
:10760000882331F02AA30E94670E080F191F2AA1B0
:10761000F7018681882321F48581882309F458C1E4
:10762000D3016D917D918D919C911397222389F4C3
:1076300020E031E040E050E00E94D96D5095409547
:10764000309521953F4F4F4F5F4F4801820E931E5B
:107650005AC08C2D8E70843051F5D701EC91F0E03A
:10766000EE0FFF1FE351F94F60817181882777FD8D
:107670008095982F20E034E640E050E00E94656D50
:10768000F3016083718382839383D70112962C91D7
:107690001297222361F0332727FD3095432F532F74
:1076A0000E94D96DF3012083318342835383D30138
:1076B0006D917D918D919C91139720E031E040E098
:1076C00050E00E94D96D50954095309521953F4FDF
:1076D0004F4F5F4F4801820E931E8114910499F021
:1076E000F701258197FE22952F7030E044E650E0A7
:1076F000249FC001259F900D349F900D1124D1012E
:1077000011969C938E93F10180819181009799F05D
:1077100020919C04222319F0019791838083D10149
:107720008D919C911197009731F0F30160817181E7
:1077300082819381B7C08114910409F4C9C0D70133
:1077400016968C911697882309F4B4C080919C04F6
:10775000882309F476C012962C9112972223B1F057
:10776000332727FD309537FF03C0309521953F4FD4
:10777000332727FD3095432F532F60E070E080E2E0
:1077800093E00E94D96D59016A0106C0A12CB12C69
:10779000F0E2CF2EF3E0DF2EF701868118141904F2
:1077A000FCF48F7090E00097F1F144E650E0849F84
:1077B0009001859F300D949F300D1124442737FD93
:1077C0004095542FC601B5010E94D96DF301808107
:1077D0009181A281B381280F391F4A1F5B1F2CC0E2
:1077E00082958F7090E00097F1F044E650E0849F1E
:1077F0009001859F300D949F300D1124442737FD53
:107800004095542FC601B5010E94D96D59016A01F6
:10781000D3012D913D914D915C9113972A193B090C
:107820004C095D0909C09801442737FD4095542F44
:10783000542F432F322F2227F30120833183428399
:107840005383D3016D917D918D919C9120E031E026
:1078500040E050E00E94D96DC801AA2797FDA0958D
:10786000BA2F1814190434F482179307A407B50724
:1078700034F012C0281739074A075B076CF4222737
:1078800017FD2095322F322F212F102F0027F301C3
:107890000083118322833383D3016D917D918D9178
:1078A0009C91139720E031E040E050E00E94D96DB8
:1078B00089010EC0C801AA2797FDA095BA2FBA2F3B
:1078C000A92F982F8827F30180839183A283B38304
:1078D000D70114966C911497633061F1643028F4E9
:1078E000613051F06230A0F444C0653069F1653018
:1078F00038F1663081F52BC0F7018181893029F498
:1079000017FD35C0005012400EC017FF32C02CC00A
:10791000D70111968C911197893041F410161106F8
:1079200004F100501E4F000F111F23C01016110646
:10793000DCF01FC017FF1DC0109501951F4F19C027
:107940001016110674F010C017FF0EC010C01016EC
:1079500011063CF00CC06750C8010E9452328C01E5
:1079600008C000E014E005C000E010E002C000E044
:107970001CEFF701878180FD13C0E181EE2381F0C8
:10798000E53070F4F0E03197EE0FFF1F21E030E0BA
:107990002C0F3D1FE20FF31F80819181080F191FEB
:1079A000B801882777FD8095982FD70112962C91E2
:1079B0001297332727FD3095432F532F0E94656D73
:1079C000F701008110E001501040278126952770B3
:1079D000213071F0F801EE0FFF1FEE0FFF1F223074
:1079E00069F5E15FF84F608371838283938334C0CC
:1079F00024E630E040E050E00E94D96DE22EC32E34
:107A0000DA01000F111F000F111F015F184FF8015D
:107A100020813181428153816E2D7C2DCD010E94C8
:107A2000656D20E034E040E050E00E94D96DD8015F
:107A30002D933D934D935C9313970EC0E15FF84FE8
:107A40002081318142815381260F371F481F591FE2
:107A50002083318342835383B985BF5FB9870894FC
:107A6000411C511CE4E0F0E06E0E7F1E22E030E08D
:107A7000220E331EB03209F049CD0E947C0E8C01DB
:107A8000ED84E0FE05C0882319F48EE10E945E6D4E
:107A9000E1FE0BC0C80190708034910519F0883464
:107AA000910519F48FE10E945E6DE2FE0DC0107029
:107AB0000038110531F00838110519F000391105A9
:107AC00019F480E20E945E6DBDEF4B2EB4E05B2E98
:107AD0003F8D28A1832F922F9A87898722243324D0
:107AE000598A488AAB85BC85ED90FD900D911C911B
:107AF000C801B70124E630E040E050E00E94D96DB3
:107B0000EB85FC852083318342835383A889B9891F
:107B10002D933D93B98BA88BEE85FF85E35AFE4FDD
:107B200080819181EE85FF85E55AFE4F2081BAE084
:107B30002B0260011124E8EEF3E0CE0EDF1EEE858D
:107B4000FF85E65AFE4F20812B0250011124A8E147
:107B50004A2EACEF5A2EA40CB51C96014C2D232FA7
:107B60008C159D0514F4482F292F842E922E8A14EB
:107B70009B040CF44501E114F1040105110569F1C0
:107B80009401442737FD4095542F1E141F041006FE
:107B9000110654F4B601882777FD8095982F621B53
:107BA000730B840B950B0DC0C501AA2797FDA095FB
:107BB000BA2F29013A01481A590A6A0A7B0AC301F5
:107BC000B201A80197010E94656D20EA36E841E004
:107BD00050E00E94D96D79018A01C4010E94D01938
:107BE0003C01882477FC8094982C6E0C7F1C801EAE
:107BF000911EC6010E94D0198C01C5010E94D019A6
:107C0000222717FD2095322F06151705280539055F
:107C100014F438014901AA2797FDA095BA2F8401D1
:107C20007301681679068A069B0614F47C018D019F
:107C3000EE85FF85E45AFE4F8081882341F0109540
:107C40000095F094E094E11CF11C011D111DF2EA75
:107C5000CF2EF1E0DF2EC20CD31CF601E358FD4F0E
:107C60008081882389F060E040E00E944F108823E3
:107C700059F0F601E258FD4F80810E94670E7C01A9
:107C80000027F7FC0095102FF894A985BA85ED928E
:107C9000FD92BA87A9877894EB85FC853496FC879A
:107CA000EB87E2E04E2E512C240C351C2E853F85AF
:107CB0002B5F3F4F3F872E8730E22316310409F0B8
:107CC00011CF04C08F7009F09AC9C3C9A2960FB62C
:107CD000F894DEBF0FBECDBFCF91DF911F910F9102
:107CE000FF90EF90DF90CF90BF90AF909F908F90DC
:107CF0007F906F905F904F903F902F900895EF92FC
:107D0000FF920F931F93DF93CF93CDB7DEB7C0548D
:107D1000D0400FB6F894DEBF0FBECDBF8E010F5F0F
:107D20001F4FC80163E00E941C3581E2E82EF12C50
:107D3000EC0EFD1EC70161E00E941C35EEEFF2E083
:107D4000418152816081D8012D913C91D7018D9163
:107D50009C911197662329F0B901681B790BCB011F
:107D600002C0821B930B840F951F73E0883E970718
:107D70002CF4ACEF89319A0724F005C088EE93E02B
:107D800002C088E19CEF9283818335960E5F1F4F7E
:107D900062E070E0E60EF71E73E0EE34F70781F65E
:107DA0008091860190E08170907022E030E0281B85
:107DB000390B80E090E02817390721F0FC01EC57DF
:107DC000FC4F1082019684309105A9F786E00E944D
:107DD000845781E00E945E6DC05CDF4F0FB6F8945F
:107DE000DEBF0FBECDBFCF91DF911F910F91FF90EE
:107DF000EF9008952F923F924F925F926F927F92F1
:107E00008F929F92AF92BF92CF92DF92EF92FF92AA
:107E10000F931F93DF93CF930F92CDB7DEB71091DF
:107E200084011F70813809F475C0823888F4833268
:107E3000F1F1843230F48032E1F0823209F07CC01A
:107E400045C0813609F45BC0803809F075C01BC09D
:107E50008438F9F0853838F4823809F44AC0833818
:107E600009F06AC040C08538E1F08F3B09F064C07A
:107E700057C0153009F060C08091A00491E08927B7
:107E80008093A0044BC00E94B1140E94F01480E8BB
:107E900005C08AED90E30E94F01484E80E949F617F
:107EA0004BC086E89AE40E94F01485E8F7CF812F52
:107EB0008F5F80938401863010F01092840181E0FE
:107EC0000E94845783E10E945E6D36C0112319F031
:107ED000812F815001C085E08093840181E00E9460
:107EE000845784E1F0CF86EF99E10E94E01483E8A3
:107EF000D5CF81E99AE10E94E01482E8CFCF80914A
:107F00004506823021F483E08093450607C0153092
:107F100099F402C00E9445300E942F1587E1D3CF0B
:107F200081E00E949F6183E00E949F6182E00E9445
:107F30009F6181E0809335088091B60160E040E068
:107F40000E944F10882331F080913508882311F466
:107F50000E947F3E8091B60160E040E00E944F1099
:107F60008093350880918401803108F0D3C09091CE
:107F7000080180917101981710F496E001C094E017
:107F8000B2EAEB2EB1E0FB2E0AE0D7014D917D0164
:107F9000802F60E024E099830E94A05C055F9981B6
:107FA000083799F7492F406884E260E10E941F0F6B
:107FB00084E268E146E50E945F5D80914506882382
:107FC00099F0823011F406E001C004E040914606C9
:107FD000509147068EE560E1202F0E94A00E83E3BA
:107FE00068E140E00E94C40F4091B40183E0480280
:107FF000A00111244051584F84E260E123E000E0E9
:108000000E94635D8091B3018F7031F089E360E17C
:108010004CEE57E00E94C25DAEE0EA2EA1E0FA2EDF
:10802000F0E0CF2EF1E0DF2E66247724EFE19E2EE4
:10803000F70101917F01D601ED91FD916D018081E4
:1080400087FD8D5F85958595843E0CF484EEA82E82
:108050008D3114F07CE1A72E862D81508230F8F40A
:10806000802F64E046E30E94445E2091860130E068
:108070002625372520FD04C08091B3018F7061F45F
:10808000802F81506EE143E00E94445E802F8F5F1D
:108090006EE143E00E94445E992D9A1914C0802F2E
:1080A0008B516BE346E30E94405E802E8A94882DBC
:1080B0006AE343E00E94405E882D6CE343E00E9447
:1080C000405E0A0D9BE36DEF862E800E5DEFA52EC0
:1080D000A90E882D6A2D47E099830E94445E9981FC
:1080E000692F6D5F882D47E00E94405E802F8D5F75
:1080F0006A2D47E00E94445E882D6A2D47E00E9469
:10810000405E0894611C711CB4E06B16710409F0A8
:108110008FCF27C080E060E042EA51E02AE001E131
:108120000E94635D9091080180917101981710F48D
:1081300042E001C040E084E560E00E941F0F8091B2
:108140004506882371F0823011F402E001C000E09E
:1081500040914606509147068FE660E0202F0E942E
:10816000A00E123008F085C043E2E42E45E0F42E64
:1081700000E039E1A32EB12C2BE1922E90E2692E82
:10818000712C80E8482E512CF701219031907F010D
:10819000113011F1802F8370899DC02C1124D02EB5
:1081A000D694D694DD0CDD0CDD0CF8E2DF0EC101B7
:1081B000B3010E94A46D9B01C101B2010E94A46D94
:1081C000AB01421B530B420D531D8C2D8F5D6D2D4A
:1081D00020E20E94D65F48C0043018F4B2E2CB2EF1
:1081E00002C0AEE5CA2E802F8370D82EDD0CDD0CC8
:1081F000D80E26E2D20EC10137FE04C08827992787
:10820000821993098A9DA0018B9D500D9A9D500D56
:10821000112440505E4F452F550F550B4595459500
:10822000842E4A3114F0E9E18E2E8C2D89516D2D6A
:1082300043E325E50E94125E6D2D62508C2D45E0D2
:108240000E94445E1214130414F4C39401C0C818AD
:108250006D2D6F5F8C2D482D0E94405E6D2D6150FD
:108260008C2D482D0E94405E0F5F083009F08CCFA6
:108270008AC0153008F07DC00E946D20123061F078
:10828000812F880F810F880F8950912F9150192FBE
:10829000110F190F110F02C080E016E0C82E9927A8
:1082A00087FD90952C01440C551C480E591E60E228
:1082B000D62EEE24FF2452E0852E912C880E991E96
:1082C0003C011AC00E94C10F5C018C2D60E040E0AF
:1082D0000E944F10082FA501440D551D8AE06D2DF9
:1082E00023E00E94635D0894E11CF11C83E090E0B0
:1082F000480E591E98E0D90EC394C701860D971DEC
:1083000088169906FCF6812F992787FD90952C01F8
:10831000440C551C480E591E30E2D32EEE24FF2487
:1083200022E0822E912C880E991E3C011AC00E94D8
:10833000C10F5C01812F60E040E00E944F10082FC8
:10834000A501440D551D85E66D2D23E00E94635D5A
:108350000894E11CF11CA3E0B0E04A0E5B1EB8E0FB
:10836000DB0E1F5FC701860D971D88169906FCF668
:108370000AC04091A2045091A3048CE368E224E077
:1083800004E00E94A00E0F90CF91DF911F910F91FA
:10839000FF90EF90DF90CF90BF90AF909F908F9025
:1083A0007F906F905F904F903F902F900895181698
:1083B0001CF010921D050895282F332727FD3095B6
:1083C00090911D05291B3109462F50E04217530794
:1083D00024F4861B80931D050895465050402417B1
:1083E000350724F48A5F861B80931D050895AF929C
:1083F000CF92DF92EF92FF920F931F93DF93CF9371
:108400000F92CDB7DEB7182F8FE79BE00E94EF19D0
:108410008FE898E0612F42E02CEC37E00AE07AE840
:10842000E72E7BE0F72ECC2456E0A52E0E94671B9A
:10843000F0908F088F2D67E00E94D74188E064E7B5
:108440007BE00E94BA5D31E08F2D813009F030E091
:108450008091B80182958695877090E0AC01440FB9
:10846000551F480F591F440F551F4B5A544F84E551
:1084700068E026E0032F39830E94635D398133234E
:1084800099F06091B801629566956770812F40E020
:1084900024E00E9493148295880F807E9091B80109
:1084A0009F71982B9093B80180E16AE47BE00E9471
:1084B000BA5D01E0EF2DE23009F000E084E560E113
:1084C0004091B901202F0E94250F002349F0812FF0
:1084D0006091B90140E024E20E9493148093B901B5
:1084E00088E16FE37BE00E94BA5D4091BA01FF2D05
:1084F000F33011F421E401C020E484E568E150E0A8
:108500000E94D65F8F2D833049F4812F6091BA018C
:1085100040E024E60E9493148093BA010091B801D0
:1085200006950695017080E261E37BE00E94BA5DEA
:10853000CF2CDD24C7FCD09421E0E4E0CE16D1049A
:1085400009F020E084E560E2402F0E94321BFF2DFD
:10855000F43079F4812F602F40E021E00E949314E1
:108560008170880F880F9091B8019B7F982B909312
:10857000B8010091B801069506950695017088E24C
:1085800063E27BE00E94BA5D21E085E0C816D10479
:1085900009F020E084E568E2402F0E94321BEF2DB5
:1085A000E53081F4812F602F40E021E00E94931498
:1085B0008170880F880F880F9091B801977F982B52
:1085C0009093B8010091B8010295017080E365E1D4
:1085D0007BE00E94BA5D21E0F6E0CF16D10409F0FD
:1085E00020E084E560E3402F0E94321B8F2D86300F
:1085F00079F4812F602F40E021E00E949314817074
:108600008295807F9091B8019F7E982B9093B801BE
:108610000F90CF91DF911F910F91FF90EF90DF901E
:10862000CF90AF900895AF92BF92CF92DF92EF922A
:10863000FF920F931F93DF93CF930F92CDB7DEB7C7
:10864000D82E8EED9CE00E94EF1981E998E06D2D07
:1086500041E02CEC37E00AE0A4EEEA2EACE0FA2E82
:10866000FBE0CF2EE0E1AE2E0E94671B1091910837
:10867000F0909208812F67E00E94D74120916F010E
:1086800030E02F5F3F4F442737FD4095542F8AE25B
:1086900060E001E172E0E72E0E94A05E2D2D2534FE
:1086A00051F0263418F4243401F511C03D2D343630
:1086B00071F03536D1F41130C1F4FF20B1F0809162
:1086C0001E05882391F08091920881500CC01130D2
:1086D00061F44F2D493048F480911E05882329F01C
:1086E000809192088F5F8093920880911D05882366
:1086F00009F088C088E069ED7CE00E94BA5D113025
:1087000031F481E090E020911E05222311F080E0F9
:1087100090E0082F00618CE368E042EA51E02AE033
:108720000E94635D80911E05882359F48091210584
:1087300087FF07C081E080931E05109221051092EB
:10874000920880911E05882381F02091210533270E
:1087500027FD30958F2D90E08217930734F4109207
:108760001E051092210510929208113009F04DC09B
:1087700080911E05882309F448C080919208909149
:108780002105891B8093920887FF02C010929208EE
:10879000809192088A301CF089E0809392081092B0
:1087A0002105AF2CBB24F501EE55FE4F80810E94C0
:1087B000712D682F20919A0430919B042115310569
:1087C00049F47D2D723631F0733621F0723411F098
:1087D000733431F48D2D40E021E40E949314682F0E
:1087E000862F0E94812D482FF501EE55FE4F808384
:1087F0008F2D880F8F0D880F845C68E021E00E9428
:10880000A05C03C098E0E92E02C080E1E82E8091D0
:108810001D05823008F084C08E2D63ED7CE00E943F
:10882000BA5D4091AF015091B001123099F4FF2030
:1088300039F480911E05882309F01AC421E019C477
:108840008F2D813039F480911E05882329F020E096
:1088500002E004C020E00DC420E001E087E46E2DBA
:108860000E94A00E123009F059C080911E05882385
:1088700039F480919A0490919B04009709F44EC0BA
:10888000FF2029F09F2D913009F048C022C080912F
:10889000AF019091B0010CE3A02EB12CB5010E9464
:1088A000906D8D2D40E02BE30E9493142CE3482F14
:1088B0004203900111248091AF019091B001B50164
:1088C0000E94906D280F391F3093B0012093AF01A3
:1088D00025C08091AF019091B0016CE370E00E94DF
:1088E000906D082F0E5F8D2D602F41E02EE30E94CA
:1088F0009314081B602F772767FD70952091AF01B7
:108900003091B001261B370B3093B0012093AF019B
:1089100037FF04C01092B0011092AF0168E0E60E7C
:1089200080911D058330F8F48E2D6BEC7CE00E9465
:10893000BA5D01E0133009F000E08CE36E2D402FAA
:108940000E94C40F002349F08D2D6091AD0147ECCA
:1089500029E30E9493148093AD0178E0E70E8E2DF9
:10896000893308F088C380911D058430C8F58E2DA9
:1089700064EC7CE00E94BA5D91E0143009F090E074
:108980008091AE01282F217030E0A901440F551FBE
:10899000A3E0220F331FAA95E1F7420F531F415561
:1089A000534F8CE36E2D2AE0092F99830E94635D5B
:1089B0009981992379F06091AE0161708D2D40E02D
:1089C00021E00E94931481709091AE019E7F982BBC
:1089D0009093AE0198E0E90EEE2DE93308F04BC319
:1089E00080911D05853030F50091B3010F708E2DFB
:1089F00068EA7CE00E94BA5D21E0153009F020E0D1
:108A00008CE36E2D402F0E94221B153069F48D2DB2
:108A1000602F40E021E00E9493148F709091B30189
:108A2000907F982B9093B301F8E0EF0E2E2D293311
:108A300008F021C380911D05863040F50091B301F7
:108A400002950F708E2D61EA7CE00E94BA5D21E0F4
:108A5000163009F020E08CE36E2D402F0E94221B7F
:108A6000163071F48D2D602F40E021E00E949314A8
:108A70008295807F9091B3019F70982B9093B30162
:108A800038E0E30E4E2D493308F0F5C280911D0504
:108A9000873050F58E2D68E97CE00E94BA5D91E048
:108AA000173009F090E04091B40186E04802A0013F
:108AB00011244758534F8CE36E2D26E0092F9983DC
:108AC0000E94635D9981992349F08D2D6091B401D5
:108AD00040E024E00E9493148093B40168E0E60E25
:108AE0007E2D793308F0C7C280911D05883008F5C6
:108AF0008E2D61E77CE00E94BA5D01E0183009F03C
:108B000000E086E36E2D4091B601202F0E94710F88
:108B1000002349F08D2D6091B6014AEE26E10E94B6
:108B200093148093B60188E0E80E9E2D993308F0E7
:108B3000A2C280911D05893008F051C08E2D68E6D3
:108B40007CE00E94BA5D9CE3AA24BB24A501405AA4
:108B5000534FFA1411F4193061F02091B70130E04D
:108B60000A2C02C0359527950A94E2F7022F01706E
:108B700001C002E0892F6E2D21E099830E94635D80
:108B80000894A11CB11C99819A5F9636F9F61930A8
:108B900001F5ED2DE03631F080919A0490919B041F
:108BA0000097B9F08D2D0E949F6110921E0581E003
:108BB00090E00F2C02C0880F991F0A94E2F72091D1
:108BC000B70128272093B70182E00E9484570E94B2
:108BD0002058F8E0EF0E2E2D293308F04CC280917A
:108BE0001D058A3008F0E3C08E2D6AE57CE00E9406
:108BF000BA5D4091B10186E0489FA00111244F5B0E
:108C0000534F1A3041F4FF2031F480911E05882320
:108C100021F002E003C000E001C001E084E26E2D1B
:108C200026E00E94635D8091B101882321F08330AA
:108C300009F04DC009C086E66E2D4CE35CE020E0F3
:108C40000E94935D9CE308C082E76E2D49E35CE0DF
:108C500020E00E94935D98E44091B201552747FDC2
:108C60005095440F551F440F551F4C5D534F1A30FC
:108C700049F43F2D313031F480911E05882321F0D5
:108C800002E003C000E001C001E0892F6E2D24E066
:108C900099830E94635D9981892F865D4091B5011A
:108CA00092E34902A0011124445D5E4F1A3049F459
:108CB0006F2D623031F490911E05992321F022E04E
:108CC00003C020E001C021E06E2D0E94D65F80919C
:108CD000B101813001F582E46E2D45E15CE020E0D8
:108CE0000E94935D4091B201552747FD50954F5F1B
:108CF0005F4F1A3049F47F2D713031F480911E0599
:108D0000882321F022E003C020E001C021E08EE7AB
:108D10006E2D0E94D65F1A3009F043C080911E0567
:108D2000882331F480919A0490919B040097C9F1B3
:108D30008F2D813079F0813018F0823091F522C08A
:108D40008D2D6091B10140E023E00E949314809347
:108D5000B10127C08091B101882311F0833031F433
:108D60008D2D6091B2014EEF24E007C08130C9F42F
:108D70008D2D6091B20140E02CE70E949314809306
:108D8000B2010FC08091B101882311F0833049F402
:108D90008D2D6091B5014CEF2AE00E9493148093D1
:108DA000B50198E0E90EEE2DE93308F064C1809139
:108DB0001D058B3008F07AC08091B101882311F035
:108DC000833019F58E2D66E07CE00E94BA5D4091FB
:108DD000BB0185E04802A00111244F515F4F1B30B9
:108DE00011F421E201C020E28EE46E2D0E94D65FD4
:108DF0001B3009F055C08D2D6091BB014CEE24E174
:108E00000E9493148093BB014BC08130B9F401E000
:108E10001B3009F000E080E06E2D40EF5BE0202F7A
:108E20000E94935D0023E1F1FD2DF038C9F581E04A
:108E300080936B0E80E00E945E6D32C08E2D67EED7
:108E40007BE00E94BA5D8091B20187FD03C0833050
:108E50001CF403C080E001C082E08093B20149E0CD
:108E60008402A00111244553544F1B3031F48091EA
:108E70001E05882321F002E003C000E001C001E0EC
:108E80008CE36E2D29E00E94635D1B3049F48D2D2B
:108E90006091B20140E022E00E9493148093B201FD
:108EA00028E0E20E3E2D393308F0E5C080911D0523
:108EB0008C3098F58E2D61EC7BE00E94BA5D31E03C
:108EC0001C3009F030E08091B801817090E0AC0175
:108ED000440F551F480F591F4654544F8CE36E2DB5
:108EE00023E0032F39830E94635D3981332379F0B6
:108EF0006091B80161708D2D40E021E00E949314D3
:108F000081709091B8019E7F982B9093B80148E0B2
:108F1000E40E6E2D693308F0AEC080911D058D30D2
:108F200040F50091B801069501708E2D60EB7BE055
:108F30000E94BA5D21E01D3009F020E08CE36E2D27
:108F4000402F0E94221B1D3071F48D2D602F40E0B8
:108F500021E00E9493148170880F9091B8019D7F49
:108F6000982B9093B80178E0E70E8E2D893308F0A6
:108F700082C080911D058E3040F50091AE010695AE
:108F800001708E2D68EA7BE00E94BA5D21E01E3000
:108F900009F020E08CE36E2D402F0E94221B1E3032
:108FA00071F48D2D602F40E021E00E9493148170B8
:108FB000880F9091AE019D7F982B9093AE0198E021
:108FC000E90EEE2DE93308F056C080911D058F3073
:108FD00048F50091AE010695069501708E2D6FE95A
:108FE0007BE00E94BA5D21E01F3009F020E08CE3B5
:108FF0006E2D402F0E94221B1F3079F48D2D602F83
:1090000040E021E00E9493148170880F880F9091B6
:10901000AE019B7F982B9093AE01F8E0EF0E2E2DC2
:10902000293348F580911D05803128F580911F0571
:10903000882319F421E0103109F020E080E06E2D42
:109040004BE85BE00E94935D1031A9F43D2D303870
:1090500091F410921E0589E180931F0580E80E941B
:109060009F611092390688E590E30E94F01403C0D6
:1090700022E000E0F3CB0F90CF91DF911F910F9191
:10908000FF90EF90DF90CF90BF90AF9008956F92D8
:109090007F928F929F92AF92BF92CF92DF92EF9288
:1090A000FF920F931F93DF93CF930F92CDB7DEB74D
:1090B000B82E89E29FE00E94EF1987EA98E06B2DB5
:1090C00047E02CEC37E00AE079E3E72E7FE0F72E6B
:1090D000CC24C3945CE0A52E0E94671B8090A70857
:1090E0008A94D090A808882D66E00E94D74118E0A5
:1090F000CC24992487FC909490911D059C0D9C3064
:1091000009F44FC1E92EFF248E149F0439F4809195
:109110001E05882329F022E0A22E04C0AA2402C042
:10912000AA24A39480E0612F46E25FE022E000E001
:1091300099830E94635D9981993010F048E301C0E2
:1091400041E3490F8CE0612F0E945F5DF701EE0F54
:10915000FF1FEE0DFF1DE650FC4F408187E0489F4A
:10916000A00111244D53514FDD2011F000E001C04A
:109170000A2D88E1612F27E00E94635DC701880FF7
:10918000991F8E0D9F1D8E559E4FFC01E85AFD4F75
:109190002081253008F4F6C0FC01EA5AFD4F283042
:1091A00008F4F9C040819D2D9130D1F53BC020E0FD
:1091B00001C02A2D88E4612F0E94250FF701EE0FD0
:1091C000FF1FEE0DFF1DE750FC4F4081552747FD67
:1091D0005095ED2DE23011F020E001C02A2D88E7F6
:1091E000612F0E94D65F00E035C020E001C02A2D2B
:1091F00088E4612F0E94710FF701EE0FFF1FEE0D43
:10920000FF1DE750FC4F4081FD2DF23011F020E0B2
:1092100001C02A2D80E6612F0E94710F01E01AC063
:1092200020E001C02A2D88E4612F0E94250FF7015C
:10923000EE0FFF1FEE0DFF1DE750FC4F40818D2DFF
:10924000823011F020E001C02A2D86E6612F0E94B5
:10925000250F02E080911E05882339F480919A043D
:1092600090919B04009709F486C0AA2009F483C05A
:109270009D2D9130D1F1913020F0923009F07BC0DA
:1092800046C03701660C771C6E0C7F1CEAEFF3E0DA
:109290006E0E7F1E8B2DF301608140E02DE00E9459
:1092A0009314F3018083202F30E0853028F088303C
:1092B00030F481E090E005C080E090E002C082E000
:1092C00090E02817390709F456C0C701880F991F85
:1092D0008E0D9F1D8E559E4FFC01EA5AFD4F108248
:1092E000895A9D4FFC01108246C0013041F0C701F0
:1092F000880F991FE80EF91E88EF93E031C03701FF
:10930000660C771C6E0C7F1C88EF93E01AC001304E
:1093100089F0C701880F991F0230F1F0E80EF91E9D
:1093200089EF93E0E80EF91E8B2DF701608143E889
:109330002DE71DC03701660C771C6E0C7F1C89EF72
:1093400093E0680E791E8B2DF30160814AEE26E1D1
:109350000E949314F3010EC0E80EF91E89EF93E00A
:10936000E80EF91E8B2DF701608140E024E20E9497
:109370009314F7018083C394185FFC2DF73009F034
:10938000BBCE0FC08A5A9D4FFC014081FD2DF130AC
:1093900009F00DCF0ECF40818D2D813009F025CF02
:1093A00026CF0F90CF91DF911F910F91FF90EF90FB
:1093B000DF90CF90BF90AF909F908F907F906F90F5
:1093C00008956F927F928F929F92AF92BF92CF92A9
:1093D000DF92EF92FF920F931F93CF93DF93982E1C
:1093E0008BE39FE00E94EF1989EA98E0692D48E03D
:1093F0002CEC37E00AE01BE4E12E1FE0F12ECC2438
:10940000C394B0E1AB2E0E94671B6090A9086A94D8
:109410008090AA08862D66E00E94D741A8E0FA2E27
:10942000DD24772467FC709440911D054D0D40317B
:1094300009F45DC0A42EBB244F5F80E06F2D20E0B7
:109440000E94510FEE24E501CC0FDD1FC05EDB4F03
:109450008501000F111F015E1B4F6A147B0471F41C
:109460008E1461F480911E05882359F480919A042A
:1094700090919B04009739F421E001C020E0CC24B6
:1094800005C022E001C021E0CC24C394EE2091F479
:109490008EE16F2DF80140810E94710FCC20D9F030
:1094A000892DF80160814AEE26E10E949314F801AB
:1094B000808311C04881552747FD509580E66F2D68
:1094C0000E94D65FCC2039F0892D688143E82DE7D2
:1094D0000E9493148883E394FE2DF33009F0BDCFEE
:1094E000D39488E0F80EED2DE73009F09DCFDF91A1
:1094F000CF911F910F91FF90EF90DF90CF90BF9091
:10950000AF909F908F907F906F900895AF92BF9291
:10951000CF92DF92EF92FF920F931F93DF93CF933F
:1095200000D0CDB7DEB7182F80919101813019F0AE
:1095300048E1C42E02C03AE1C32E2BEFB22EBC0C80
:109540008AE19AE00E94EF1986E498E0612F40E0FA
:1095500020EE37E006E0EC2C0E94F01EF09046086A
:10956000D09047088F2D67E00E94D74160911D057C
:109570008C2D90E0462F50E09C0127503040421740
:10958000530761F42F2D30E004972817390714F49E
:109590008FEF01C081E0680F60931D05113629F13E
:1095A000123678F4143409F448C0153420F4123417
:1095B00008F46AC063C0153419F1103609F064C0AC
:1095C00009C0143608F45AC01436B9F1153609F03A
:1095D0005BC016C0FF2009F457C081E090911E05C2
:1095E000911180E080931E054FC080911E05882355
:1095F00009F44AC010921E0581E60E949F6144C092
:109600002F2D213059F4DD2049F080911E0588234B
:1096100029F0809147088150809347082F2D30E032
:109620008B2D992787FD90952817390769F5DD203F
:1096300059F18091470881501EC03F2D313061F4AF
:109640008D2D893048F480911E05882329F0809162
:1096500047088F5F809347082F2D30E08B2D992787
:1096600087FD90952817390779F49D2D973060F480
:10967000809147088F5F8093470806C080911E0540
:10968000882311F41092470880911D05882309F062
:1096900089C088E06FE07AE00E94BA5DEF2DE1308A
:1096A00031F481E090E020911E05222311F080E04A
:1096B00090E0082F006182E468E043E951E02AE08D
:1096C0000E94635D80911E05882359F480912105D5
:1096D00087FF07C081E080931E051092210510923C
:1096E000470880911E05882381F0209121053327AA
:1096F00027FD30958D2D90E08217930734F410925A
:109700001E051092210510924708FF2DF13009F037
:109710004CC080911E05882309F447C080914708FA
:1097200090912105891B8093470887FF02C0109202
:109730004708809147088A301CF089E080934708E9
:1097400010922105AD2CBB24F501ED56FE4F808112
:109750000E94712D682F20919A0430919B0421154D
:10976000310541F4123631F0133621F0123411F084
:10977000133431F4812F40E021E40E94A214682FB9
:10978000862F0E94812D482FF501ED56FE4F8083D4
:109790008D2D880F8D0D880F8E5B68E021E00E9473
:1097A000A05C03C098E0E92E02C080E1E82E809121
:1097B0001D058230A0F5C0908501C694C694C6945C
:1097C00027E0C2228E2D68E07AE00E94BA5D91E027
:1097D0003F2D323009F090E046E08C2D849FA001AF
:1097E00011244352564F8CE56E2D26E0092F9A83A3
:1097F0000E94635D9A81992381F0812F6C2D40E056
:1098000026E00E94A2148770880F880F880F90911D
:109810008501977C982B9093850198E0E90E8091C3
:109820001D05833058F5C09091018E2D62ED79E0D1
:109830000E94BA5D91E0EF2DE33009F090E046E040
:10984000FC2DF49FA00111244B53564F8CE56E2D37
:1098500026E0092F9A830E94635D9A81992341F043
:10986000812F6C2D40E021E00E94A2148093910191
:1098700028E0E20E3E2D393308F0FFC380919101BC
:10988000813041F580911D05843030F58E2D67EBD8
:1098900079E00E94BA5D40918F018F2D843011F4E0
:1098A00021E401C020E486E66E2D50E00E94D65FE0
:1098B0009F2D943049F4812F60918F0141E024E67F
:1098C0000E94A21480938F01E8E0EE0EFE2DF93382
:1098D00018F0D3C304E001C005E0809191018150EC
:1098E000823038F580911D05801710F58E2D67EABE
:1098F00079E00E94BA5D40919001F01611F421E4E4
:1099000001C020E486E66E2D50E00E94D65FF0167E
:1099100049F4812F6091900140E025E00E94A2145B
:109920008093900128E0E20E3E2D393308F0A5C364
:109930000F5F80911D05801720F58E2D6EE979E06F
:109940000E94BA5D40917001F01611F421E401C04B
:1099500020E486E66E2D50E00E94D65FF01659F4A2
:10996000812F609170014AE02DE20E94A214809341
:1099700070010E94366088E0E80E9E2D993308F051
:109980007CC3C02EC39480911D058C1508F58E2DC7
:109990006EE879E00E94BA5D40917101FC1411F407
:1099A00021E401C020E486E66E2D0E940B0FFC141A
:1099B00049F4812F6091710148E228E70E94A214C6
:1099C00080937101E8E0EE0EFE2DF93308F055C3E7
:1099D000C39480911D058C1560F58E2D6DE779E09F
:1099E0000E94BA5D40918701552747FD5095465F1B
:1099F0005F4FFC1411F421E401C020E486E66E2DD3
:109A00000E94D65F8091A70D6E2D4DE60E945F5D8E
:109A1000FC1449F4812F6091870146EF2EE60E94E5
:109A2000A2148093870128E0E20E3E2D393308F01E
:109A300024C3C39480911D058C1550F58E2D62E7CB
:109A400079E00E94BA5D91E0FC1090E040918901BC
:109A500050E0440F551F440F551F4B59564F86E693
:109A60006E2D24E0092F9A830E94635D9A819923C9
:109A700049F0812F6091890140E022E00E94A21408
:109A80008093890188E0E80E9E2D993308F0F5C295
:109A9000C39480911D058C15C8F480918801817054
:109AA00021E0FC1020E06E2D44E559E0012F0E94DA
:109AB0008B2D8170909188019E7F982B90938801C7
:109AC000E8E0EE0EFE2DF93308F0D7C2C394809182
:109AD0001D058C15D8F4809188018695817021E050
:109AE000FC1020E06E2D48E459E0012F0E948B2DE0
:109AF0008170880F909188019D7F982B90938801A9
:109B000028E0E20E3E2D393308F0B7C2C3948091AD
:109B10001D058C15E8F480918801869586958170E5
:109B200021E0FC1020E06E2D49E359E0012F0E9456
:109B30008B2D8170880F880F909188019B7F982BC7
:109B40009093880188E0E80E9E2D993308F095C225
:109B5000C39480911D058C15F8F480918801869539
:109B600086958695817021E0FC1020E06E2D4BE2F9
:109B700059E0012F0E948B2D8170880F880F880F6C
:109B800090918801977F982B90938801E8E0EE0EE2
:109B9000FE2DF93308F071C2C39480911D058C1518
:109BA00000F58E2D6EE179E00E94BA5D01E0FC10B7
:109BB00000E080E66E2D40917301202F0E94710F0E
:109BC000002349F0812F609173014AEE26E10E9443
:109BD000A2148093730128E0E20E3E2D393308F081
:109BE0004CC2C394BB2480911D058C1508F048C05D
:109BF000BB2019F46EE079E002C06EEF78E08E2DA4
:109C00000E94BA5DBB2019F4A0908A0102C0A09006
:109C10009201AA20A9F08A2D95E0899FA001112424
:109C2000FC1411F421E401C020E486E66E2D0E94AC
:109C3000D65F8091A70D6E2D43E70E945F5D0AC03D
:109C400001E0FC1000E086E66E2D4AEF58E023E0CC
:109C50000E94635DFC1439F4812F6A2D40E028E7EF
:109C60000E94A214A82EBB2019F4A0928A0102C05F
:109C7000A0929201E8E0EE0EFE2DF93308F0FDC14E
:109C8000C394B3942B2D223009F0ADCF80911D05E4
:109C90008C15F8F48091880182958F708095817081
:109CA00021E0FC1020E06E2D4CEE58E0012F0E94C8
:109CB0008B2D809581708295807F909188019F7E09
:109CC000982B9093880138E0E30E8E2D893308F0AD
:109CD000D4C1C39480911D058C15F8F480918E0138
:109CE00082958F708095817021E0FC1020E06E2DB0
:109CF00040EE58E0012F0E948B2D80958170829557
:109D0000807F90918E019F7E982B90938E0198E09A
:109D1000E90EEE2DE93308F0B0C1C39480911D0522
:109D20008C15D8F4809185018095817021E0FC101C
:109D300020E06E2D4FEC58E0012F0E948B2D809576
:109D40008170909185019E7F982B90938501F8E01A
:109D5000EF0E2E2D293308F090C1C39480911D057C
:109D60008C15E8F48091850186958095817021E0BD
:109D7000FC1020E06E2D40EC58E0012F0E948B2D4E
:109D800080958170880F909185019D7F982B90938D
:109D9000850138E0E30E8E2D893308F06EC1C3943F
:109DA00080911D058C1508F086C08E2D65EB78E03E
:109DB0000E94BA5D92E4AA24BB24A5014455574FE2
:109DC000E0919D01F0E00A2C02C0F595E7950A9418
:109DD000E2F7E170F070892F6E2D21E00E2F9A834B
:109DE0000E94635D0894A11CB11C9A819A5F92370E
:109DF00021F7FC1409F059C0809147089091210582
:109E0000891B8093470887FF02C010924708809102
:109E100047088A301CF089E080934708109221059A
:109E20008D2D880F8D0D880F4D2D50E04D55574FBE
:109E30008E5B6E2D21E002E00E94635D103631F0F2
:109E400080919A0490919B04009779F1812F0E9450
:109E50009F6110921E0581E090E002C0880F991F5B
:109E6000DA94E2F790919D01982790939D018031BB
:109E700051F0803271F0883099F493FF02C09F7CDA
:109E80000DC098600BC094FF02C0977D07C0906121
:109E900005C095FF02C0977E01C0906290939D011E
:109EA00081E00E9484570E94205898E0E90EEE2D30
:109EB000E93308F0E2C0C39480911D058C15F8F4D5
:109EC00080918501869586958095817021E0FC10B2
:109ED00020E06E2D44E958E0012F0E948B2D8095E3
:109EE0008170880F880F909185019B7F982B9093AC
:109EF0008501F8E0EF0E2E2D293308F0BEC0C39483
:109F000080911D058C1500F590918501991F992769
:109F1000991F81E0891B21E0FC1020E06E2D46E8AE
:109F200058E0012F0E948B2D809587958827879573
:109F3000909185019F77982B9093850138E0E30EEF
:109F40008E2D893308F099C0C39480911D058C151E
:109F500008F580918801829586958770809581703B
:109F600021E0FC1020E06E2D4CE758E0012F0E940C
:109F70008B2D809581708295880F807E90918801CD
:109F80009F7D982B9093880198E0E90EEE2DE933A0
:109F900008F073C0C39480911D058C1518F580914D
:109FA000880182958695869583708095817021E0E1
:109FB000FC1020E06E2D44E758E0012F0E948B2D0D
:109FC000809581708295880F880F807C90918801A0
:109FD0009F7B982B90938801F8E0EF0E2E2D29336C
:109FE00008F04BC0C39480911D058C1508F045C046
:109FF00086E06E2D4FE658E00E94C25D3E2D38335C
:10A0000090F434E290E0832F6E2D41E857E0292F41
:10A0100000E039839A830E94415C9A819F5F398175
:10A02000385E943081F788E0E80E9E2D993328F54C
:10A03000DD24D394FC10DD24409186014F5C82E145
:10A040006E2D2D2D0E94A05C94E200E00F5F892F01
:10A050006E2D402F20E09A830E94250F9A81985EF2
:10A060000430A1F7DD2049F0812F6091860140E0A6
:10A0700023E00E94A214809386010F900F90CF914D
:10A08000DF911F910F91FF90EF90DF90CF90BF90E5
:10A09000AF9008958F929F92AF92BF92CF92DF922E
:10A0A000EF92FF920F931F93DF93CF930F92CDB751
:10A0B000DEB7C82E84E79FE00E94EF198BEA98E094
:10A0C0006C2D49E02CEC37E00AE0FAE0EF2E0E941C
:10A0D000F01E1091AB081150812F66E00E94D7410D
:10A0E0002C2D203899F480E80E949F6189E18093AB
:10A0F0001F05193019F40E945E6205C0183018F46B
:10A10000812F0E94D06281E00E945E6DDD24E8E034
:10A11000FE2EA12EBB24A7FCB09480911D058D0DB1
:10A12000883081F1882E992494012F5F3F4F442776
:10A1300037FD4095542FA814B90411F401E101C072
:10A1400000E182E16F2D72E0E72E0E94A05EF40133
:10A15000EE0FFF1FE850F64E85919491AC0180916F
:10A160001F05882321F421E0A814B90409F020E098
:10A1700088E16F2D0E94935D38E0F30ED3948D2D0E
:10A18000873059F6EF2DE93308F04FC080911F0555
:10A19000882321F4DD24D394183009F0DD2486E0EF
:10A1A0006F2D46E65FE00E94C25D9AE556E0A52E5F
:10A1B000B12CE0918B01F0E0E852FB4F449150E06C
:10A1C0000A2C02C0559547950A94E2F743705070E7
:10A1D0004F59504F892F6F2D21E00D2D99830E94EB
:10A1E000635D2EEF3FEFA20EB31E99819A5F923707
:10A1F00001F7DD2049F08C2D60918B0140E027E1D3
:10A200000E94A21480938B016F2D685F693368F4FC
:10A2100080911F05882319F421E0193009F020E00E
:10A2200086E04DE45FE00E94935D0F90CF91DF9157
:10A230001F910F91FF90EF90DF90CF90BF90AF9064
:10A240009F908F9008954F925F926F927F928F921E
:10A250009F92BF92CF92DF92EF92FF920F931F9344
:10A26000DF93CF9300D0CDB7DEB7182F82EB9FE0FE
:10A270000E94EF198FEB98E0612F46E02CEC37E05D
:10A280000AE050E1E52E0E94F01E6090BF086A943B
:10A29000862D66E00E94D741103611F0143641F445
:10A2A00067FC06C06092A40882EC92E30E94F0145E
:10A2B000CC24DD24EE24E39418E0F12E772467FC0F
:10A2C000709430911D053C0DBB24B394383028F4B4
:10A2D000BB248E2D883028F074C09E2D973008F056
:10A2E00070C0032F10E091E06016710609F090E055
:10A2F000DD2019F0DD24D39401C0D92E80E06F2D2C
:10A300004FEA5FE0292F3A8399830E94935D3A8157
:10A310009981393010F482E101C087E1A8014F5FD3
:10A320005F4F6F2D292F0E94D65FBB2079F0085018
:10A3300010402801B3E0440C551CBA95E1F7400EDB
:10A34000511EE0EBF3E04E0E5F1E0BC02801440CE3
:10A35000551C440C551C400E511E88E893E0480ED5
:10A36000591E42010AE2F40141914F01552747FD70
:10A370005095802F6F2D20E00E94D65F0B5E033931
:10A3800091F7F8E0FF0EE394BB20B1F085E090E098
:10A39000480E591E0AE2F20141912F01552747FD4F
:10A3A0005095802F6F2D20E00E94D65F0B5E0E37F8
:10A3B00091F7F8E0FF0EE394C3948C2D873009F0F9
:10A3C00080CFDD2029F480911D058F5F80931D05CE
:10A3D0000F900F90CF91DF911F910F91FF90EF9011
:10A3E000DF90CF90BF909F908F907F906F905F9005
:10A3F0004F900895AF92BF92CF92DF92EF92FF926B
:10A400000F931F93CF93DF93F82E85EA98E06F2D7B
:10A410004DE00E94612080919D08882319F087EB10
:10A420009EE002C08DEA9EE00E94EF19182F8091F5
:10A430009E080E94840EEC01812F8A5F60E04881B3
:10A4400020E00E94510FA090A5088A2D66E00E948E
:10A45000D74118E0EE24BB24A7FCB09420911D0541
:10A460002E0D822F90E0DD24D394A816B90609F0B2
:10A47000DD24263009F4FAC0273090F4223009F4A4
:10A4800057C0233030F4222309F1213009F0E8C10C
:10A4900034C0243009F499C0253008F0BAC069C02E
:10A4A0002A3009F46BC12B3038F4283009F420C16C
:10A4B000293008F044C1F1C02C3009F49CC12C3083
:10A4C00008F47AC12D3009F0CBC1B2C18CE0612F04
:10A4D00046EA5EE00E94C25D84E5612F49812D2D30
:10A4E0000E94250FDD2009F4BBC18F2D698141E059
:10A4F00024E20E9493148983B3C18CE0612F4FE959
:10A500005EE00E94C25D4A81552747FD50952D2D82
:10A51000206484E5612F0E94D65FDD2009F4A0C18C
:10A520008F2D6A8143E82DE70E9493148A8398C196
:10A530008F8186FF03C045E95EE002C04EE85EE021
:10A540008CE0612F0E94C25D4885552747FD5095DC
:10A550002D2D206484E5612F0E94D65FDD2009F453
:10A560007FC18F2D688543E82DE70E94931488876B
:10A5700077C1CF80C294C694C694E3E0CE2281E036
:10A58000C8228CE0612F43E85EE00E94C25D43E098
:10A590009C2D949FA00111244458514F84E5612FB4
:10A5A00023E00D2D0E94635DDD2009F459C18F2D3C
:10A5B0006C2D40E021E00E94931481708295880FF9
:10A5C000880F807C9F819F7B90C08CE0612F47E744
:10A5D0005EE00E94C25D8F81817090E0AC01440F0B
:10A5E000551F480F591F4059514F84E5612F23E0F3
:10A5F0000D2D0E94635DDD2009F432C16F81617011
:10A600008F2D40E021E00E94931481709F819E7FF6
:10A610006CC08CE0612F49E65EE020E00E94935D13
:10A620004C8183E0489FA00111244352504F84E5A0
:10A63000612F23E00D2D0E94635DDD2009F410C120
:10A640008F2D6C8140E026E10E9493148C8387302B
:10A6500008F406C19F2D903609F002C187508093FF
:10A66000A40882EC92E30E94F014FAC08CE0612FFF
:10A6700042E65EE00E94C25D8EE4612F4B812D2D8B
:10A680000E94710FDD2009F4EBC08F2D6B814AEE23
:10A6900026E10E9493148B83E3C08CE0612F4AE58E
:10A6A0005EE00E94C25D0F810295037049F02D2D7E
:10A6B000206484E5612F402F50E00E94D65F07C0E0
:10A6C00084E5612F46E55EE02D2D0E94935DDD203F
:10A6D00009F4C6C08F2D602F40E023E00E94931440
:10A6E00083708295807F9F819F7C982B9F83B8C0C9
:10A6F0008CE0612F4FE45EE00E94C25D4F81469581
:10A70000477050E063E0440F551F6A95E1F74A5CDB
:10A71000514F84E5612F28E00D2D0E94635DDD20FF
:10A7200009F49EC06F81669567708F2D40E022E02E
:10A730000E9493148770880F9F81917FD6CF8CE001
:10A74000612F4BE25EE00E94C25D4D8142954F70E9
:10A7500080E6612F50E02D2D0E94D65FDD2009F4A8
:10A760007FC06D8162956F708F2D40E02FE00E9459
:10A7700093148295807F9D819F701BC08CE0612F18
:10A7800042E25EE00E94C25D4D814F7080E6612F23
:10A7900050E02D2D0E94D65FDD2009F461C06D814F
:10A7A0006F708F2D40E02FE00E9493148F709D8179
:10A7B000907F982B9D8354C08CE0612F47E15EE031
:10A7C0000E94C25D4E8142954F7080E6612F50E03D
:10A7D0002D2D0E94D65FDD2009F442C06E81629566
:10A7E0006F708F2D40E02FE00E9493148295807F40
:10A7F0009E819F701AC08CE0612F4EE05EE00E9447
:10A80000C25D4E814F7080E6612F50E02D2D0E9479
:10A81000D65FDD2029F16E816F708F2D40E02FE033
:10A820000E9493148F709E81907F982B9E8318C0F6
:10A830008CE0612F4CEF5DE02D2D0E94935DDD20BB
:10A8400079F08F2D803861F40E949F6180919E087D
:10A850000E947E2281E00E945E6D80E00E94BB1417
:10A86000E394185F9E2D973009F0F8CDDF91CF91DA
:10A870001F910F91FF90EF90DF90CF90BF90AF901E
:10A8800008955F926F927F928F929F92AF92BF9244
:10A89000CF92DF92EF92FF920F931F93CF93DF93AC
:10A8A000D82E86E99FE00E94EF198DEB98E06D2D80
:10A8B00045E02CEC37E00AE07DE9E72E7FE0F72E5B
:10A8C00051E1C52E11E1A12E0E94671BF090BD0839
:10A8D000FA948090BE088F2D66E00E94D7418D2D9E
:10A8E000803821F59F2D903108F5EF2DFF27E7FDEA
:10A8F000F09580911D05E81BF109EE0FFF1FED5D3E
:10A90000FA4FC081D1818F2D0E94940EFC018820C6
:10A9100069F48281882319F0D095C195DF4FD483E3
:10A92000C38382E00E9484570E94205818E0992433
:10A93000552453946F2C772467FC709400911D0567
:10A94000090D003109F4E1C0802F0E94940EEC0142
:10A950008A816B817C81882319F0709561957F4F86
:10A96000A02EBB24F501EE0FFF1FED5DFA4F2081F5
:10A970003181261B370B2333310524F0F501E355D4
:10A98000F74F08C09FEF2E3C39072CF4F501E35533
:10A99000F74F85258083402F4F5F80E0612F20E0B7
:10A9A0000E94510FF501E355F74F8081882311F084
:10A9B0004FE701C04EE78BE4612F20E00E94A05CCE
:10A9C000EE246A147B0471F48E1461F480911E05E8
:10A9D000882359F480919A0490919B04009739F44C
:10A9E00001E001C000E0CC2405C002E001C001E0AC
:10A9F000CC24C3948E2D823009F43FC0833009F4F7
:10AA00005DC08130C1F04B815C81202F206280E3EA
:10AA1000612F0E94D65FCC2009F46BC06B817C81D2
:10AA20008D2D48E15CEF28EE33E002E00E94CF1369
:10AA30009C838B835EC048814456552747FD5095C3
:10AA400088E4612F202F0E94D65FCC2009F451C0EA
:10AA50006881645668838091B80181FF04C08D2DA0
:10AA600043E82DE703C08D2D4CE924E60E949314A2
:10AA7000888388818C5988833CC049814C595527EB
:10AA800047FD509586E6612F202F0E94D65FCC208F
:10AA900081F169816C5969838091B80181FF04C09B
:10AAA0008D2D43E82DE703C08D2D4CE924E60E944F
:10AAB000931489838981845689831BC08A8190E09D
:10AAC000AC01440F551F480F591F4157504F8CE69A
:10AAD000612F23E00E94635DCC2059F08D2D6A81A7
:10AAE00040E021E00E94931491E0882309F490E073
:10AAF0009A83E3949E2D943009F063CF9394185F6A
:10AB0000892D873009F01ACF1FC001E09F2D9031A9
:10AB100009F000E080911F05882311F020E001C0BA
:10AB2000202F82E1612F4EE75FE00E94935D0023BA
:10AB300059F08D2D803841F489E180931F0580E81C
:10AB40000E949F610E947F3EDF91CF911F910F91E4
:10AB5000FF90EF90DF90CF90BF90AF909F908F903D
:10AB60007F906F905F900895F8942091D50D30916B
:10AB7000D60D7894C9010895CF93DF93C2E4D1E054
:10AB800080E6FE0111928A95E9F78AE080934201FE
:10AB900089E1809370018AE58093710181E080935F
:10ABA00086012196FE0120E032E080E891E02193C9
:10ABB000319395878487938F828F41E0E135F40745
:10ABC000B1F783E991E06FE770E14AE050E00E945D
:10ABD000FA6D80E090E029913991820F931FE1E0B6
:10ABE000CB35DE07C1F790936E0180936D01DF9145
:10ABF000CF9108951F93CF93DF9388EC98E060E0A6
:10AC00000E94E05962E471E080E6FB0111928A95AE
:10AC1000E9F788EC98E040E650E00E946C5A182F63
:10AC2000C3E9D1E088810E94712D0E94812D899312
:10AC3000F1E0CD39DF07B1F7809142018A3028F485
:10AC400080917F04816080937F048AE08093420139
:10AC50001D3468F0E3E4F1E020E030E0819191916F
:10AC6000280F391F81E0EB35F807C1F702C020E05B
:10AC700030E081E040916D0150916E014217530721
:10AC800009F080E0DF91CF911F9108951F93182F55
:10AC9000E2EAF1E025EA32E0DF01C9011D92019705
:10ACA000E9F7CF0164E770E14AE050E00E94FA6DF5
:10ACB000812F90E001966AE070E00E94A46D605DD3
:10ACC0006093A701805D8093A8018AE08093AC0126
:10ACD00080E00E94D0621F910895CF92DF92EF92A0
:10ACE000FF920F931F93DF93CF930F92CDB7DEB7F1
:10ACF0006B01803160F5682F6F5F88EC98E04983C5
:10AD00000E94E0594981042F10E0C60160E270E022
:10AD100050E00E941B6E88EC98E0B6014AE050E0DB
:10AD20000E946C5A8A30910591F488EC98E00E9458
:10AD3000D259F601E00FF11F2AE030E006C0B90158
:10AD40000E94906D805D8293CB010097C1F70F90B8
:10AD5000CF91DF911F910F91FF90EF90DF90CF90F7
:10AD600008958F5F0E94635908951F93CF93DF93D7
:10AD7000182F803168F5682F6F5F88EC98E00E948B
:10AD8000E05962EA71E025EA32E0FB01C901119263
:10AD90000197E9F788EC98E045EA52E00E946C5A86
:10ADA0008F3F910509F018F4812F0E944656C2EAA0
:10ADB000D1E088810E94712D0E94812D899391E0BC
:10ADC000CC3AD907B1F78AE08093AC010E942F15E5
:10ADD000DF91CF911F9108950F931F93DF93CF932E
:10ADE000CDB7DEB760970FB6F894DEBF0FBECDBF0C
:10ADF000682F6F5F062F0AC0102F1F5F812F688B8F
:10AE00000E9463596889882329F0012F0031A0F33B
:10AE1000003139F188EC98E00E94E059602F6F5FB3
:10AE200081ED98E042E028E532E00E94525B8E011D
:10AE30000F5F1F4F06C081ED98E0B8010E94CD5A08
:10AE4000A89588EC98E0B8014FE050E00E94FB59CB
:10AE5000482F882381F781ED98E00E947B5B81E099
:10AE600001C080E060960FB6F894DEBF0FBECDBF84
:10AE7000CF91DF911F910F910895EF920F931F9340
:10AE80000E944E59882341F00E94B95887FD04C0A2
:10AE90000E94FA55882381F584E690E161E00E94E2
:10AEA0009E1282E590E10E9485120E9428590E941C
:10AEB000BC5588EC98E060E041E022E431E000E637
:10AEC00010E078ECE72E0E94AA5B8036910529F00D
:10AED00083E490E160E00E949E1280E00E9446566A
:10AEE00088EC98E061E042E022EA31E005EA12E015
:10AEF00058ECE52E0E94AA5B80916F010E94B55626
:10AF00001F910F91EF900895882359F09091E408D4
:10AF1000982B9093E4080E947C0E9093E60880930F
:10AF2000E5080895EF920F931F93CF93DF9310914D
:10AF3000E408112309F47EC0882309F076C00E943A
:10AF40007C0E2091E5083091E608AC01421B530BC2
:10AF50004436510508F46EC068C081E08093E30870
:10AF6000812F90E0EC01C470D07012FF03C023E089
:10AF70002093E3081092E40880FF1CC08AED98E05B
:10AF800061E141E022E431E000E610E0F4E1EF2E7F
:10AF90000E94AA5B8036910511F480E020C0809168
:10AFA000E008823021F48091E408816029C083E3C5
:10AFB00090E135C081FF36C08AED98E061E142E062
:10AFC00022EA31E005EA12E0E4E1EE2E0E94AA5BFB
:10AFD00052E0853A950739F480916F018F5F61E106
:10AFE0000E9471591FC08091E0088230A1F48091C5
:10AFF000E408982F92609093E408209719F08660F7
:10B000008093E4080E947C0E845690409093E6085A
:10B010008093E50807C0209729F483E290E160E07F
:10B020000E949E121092E30805C08091E3088823D5
:10B0300009F493CFDF91CF911F910F91EF90089575
:10B040000AC081E00E9492578091690E833019F402
:10B05000A8951092690E8091E408882391F70895CD
:10B06000DF93CF930F92CDB7DEB7682F70E084E007
:10B07000660F771F8A95E1F7CE01019641E050E017
:10B080000E94226E89810F90CF91DF910895DF9306
:10B09000CF930F92CDB7DEB76983682F70E094E04D
:10B0A000660F771F9A95E1F7CE01019641E050E0D7
:10B0B0000E9473600F90CF91DF91089587EE98E022
:10B0C00060E070E040E450E00E947360089589EE13
:10B0D00098E062E070E041E050E00E947360089503
:10B0E0000F931F93182F082F04C0802F0E943058F1
:10B0F000082F802F0E9430588823B9F7802F609145
:10B10000E9080E9447581093E9080E9467581F9168
:10B110000F9108951F931091E908112359F0812F81
:10B120000E9430588093E9080E946758812F60E0A0
:10B130000E944758812F1F910895F8942091D50DB2
:10B140003091D60D7894C9010895EF92FF92CF9374
:10B15000DF938091E908C0E0D0E003C02F960E9401
:10B1600030588823D9F7CE01DF91CF91FF90EF902F
:10B170000895CF92DF92EF92FF920F931F93CF9398
:10B18000DF9380E8E7E2F9E0DF011D928A95E9F7B5
:10B190000BEE18E0C0E0D0E08C2FC43139F4D09031
:10B1A000E90839EEE32E38E0F32E0BC07E01EE0CF9
:10B1B000FF1CEC0EFD1E2BEE38E0E20EF31ED80154
:10B1C000DC9090E0C82EC3941DC08D2D84508C3728
:10B1D00038F4ED2DF0E0E95DF64F8081882361F0D1
:10B1E000992329F0892F60E00E9447580DC0F7018C
:10B1F00010820E945E5808C0C0828D2D0E94305877
:10B200009D2DD82EDD2009F721960D5F1F4FC531EA
:10B21000D10511F604E0E02FF0E0E95DF64F808102
:10B22000882349F4802F6091E9080E9447580093D1
:10B23000E9080E9467580F5F003869F780E0DF91E6
:10B24000CF911F910F91FF90EF90DF90CF900895D5
:10B250001F9380E4E7EEF8E0DF01982F1D929A95A6
:10B26000E9F794E09093E7088093E80880E1809301
:10B27000EA0884E001C0812F182F1F5F612F0E9410
:10B2800047581038C1F78FE760E00E94475884E0C4
:10B290008093E9080E945E581F91089587EE98E018
:10B2A00060E070E040E450E00E94226E8091E70888
:10B2B000843039F481E09091E808903419F080E00E
:10B2C000089580E0089590E0FC01EE0FFF1FE80F65
:10B2D000F91FE951F74F81E09481992309F480E047
:10B2E0000895DF93CF9300D00F92CDB7DEB790E0F3
:10B2F000FC01EE0FFF1FE80FF91FDE011196E5516B
:10B30000F74F23E001900D922150E1F770E0DC014E
:10B31000AA0FBB1FA80FB91FFB01EE0FFF1FE60FFF
:10B32000F71FA551B74FE551F74F83E001900D92FC
:10B330008150E1F7FB01EE0FFF1FE60FF71FE5510C
:10B34000F74FDE01119683E00D9001928150E1F7F5
:10B350000E945E580F900F900F90CF91DF9108954B
:10B36000DF93CF930F92CDB7DEB790E09C01220F11
:10B37000331F280F391FF901E951F74F84812551F7
:10B38000374F93E0D9011D929A95E9F789830E947E
:10B390005E588981882311F00E9470580F90CF91D8
:10B3A000DF910895FC01808190E0FC01EE0FFF1F0A
:10B3B000E80FF91FE451F74F918180819F70089544
:10B3C000FC0160831282118270E0CB01880F991F0B
:10B3D000860F971FDC01A951B74F14962C91149733
:10B3E00023831482158216828351974FFC0180813A
:10B3F00082958F7008958F929F92AF92BF92CF9255
:10B40000DF92EF92FF920F931F93DF93CF930F92F0
:10B41000CDB7DEB78C015B01FC01808190E0FC01BF
:10B42000EE0FFF1FE80FF91FE451F74F80812181D4
:10B43000922F9F70F80121813281821B930BE42EA1
:10B44000F52E8E159F0508F47C0167014E010894C6
:10B45000811C911C25C0F8016381662321F1848140
:10B460008F5F848370E0B4E0660F771FBA95E1F7D1
:10B47000680F711DC40141E050E00E94226E898175
:10B48000F50181935F01F80184818F3030F01482DF
:10B4900083810E943058F80183830894C108D10841
:10B4A000C114D104C1F6F801818192818E0D9F1DD6
:10B4B0008C199D09928381838E2D8C190F90CF91C9
:10B4C000DF911F910F91FF90EF90DF90CF90BF9091
:10B4D000AF909F908F9008958F929F92AF92BF925E
:10B4E000DF92EF92FF920F931F93CF93DF938C0124
:10B4F0005B017A01C0E0D0E045E0842E912C880EFB
:10B50000991E3BC0F801858190E08F77907000977D
:10B5100041F4C801B40141E050E00E94FB59813080
:10B5200079F5F80145813FE7D32ED4222D2D30E067
:10B53000C7018C1B9D0B8217930710F4DE2CDC1ABD
:10B54000B5016C0F7D1F47FF08C0CB0160E070E0C4
:10B550004D2D50E00E941B6E0AC0C8014D2D50E0D9
:10B560000E94FB598D1519F0C80FD11D09C0CD0DD2
:10B57000D11DF80185818D198583CE15DF0510F267
:10B58000CE01DF91CF911F910F91FF90EF90DF904F
:10B59000BF90AF909F908F9008959F92AF92BF926F
:10B5A000CF92DF92EF92FF920F931F93CF93DF938F
:10B5B000EC018B01C42E8B81882389F489819A81C7
:10B5C000009769F4E880FF240E948A588B83F70172
:10B5D000EE0FFF1FEE0DFF1DE951F74F8483DC2CAA
:10B5E0006FE0962E44C0EF80F8840E947C0EE81A2B
:10B5F000F90AF7FE02C082E004C08B81882319F4A7
:10B6000081E08E8337C09C819F3080F01C820E9435
:10B610003058882339F4EB800E948A58682F8E2D89
:10B620000E9447588B810E9430588B838B818823DE
:10B6300039F36C81992D961BED2C9D1508F4E92E9C
:10B64000AE2CBB2470E06F5F7F4F90E054E0880F1A
:10B65000991F5A95E1F7680F791FC801A5010E944B
:10B6600073600A0D1B1D8C818E0D8C83DE18DD200E
:10B6700009F0B9CF2C2D30E02D19310989819A813B
:10B68000820F931F9A8389838C2D8D19DF91CF911F
:10B690001F910F91FF90EF90DF90CF90BF90AF90F0
:10B6A0009F9008950F931F93CF93DF93EC0189012F
:10B6B00068831A82198270E0CB01880F991F860F68
:10B6C000971FFC01E951F74F24812B831C821D82B7
:10B6D0001E82FC01E451F74F10824295407F418366
:10B6E0000E947C0E080F191F18870F83DF91CF91DE
:10B6F0001F910F9108951F93CF93DF93EC018881E1
:10B7000090E0FC01EE0FFF1FE80FF91FE451F74F27
:10B71000898180839A819F708181807F892B818339
:10B720008B81882389F00E943058182F882361F07C
:10B730008B8160E00E9447580E945E58112331F0CF
:10B74000812F0E94705802C010E0F6CFDF91CF9198
:10B750001F9108954F925F926F927F929F92AF9246
:10B76000BF92CF92DF92EF92FF920F931F93DF93DE
:10B77000CF930F92CDB7DEB75C01290168012E2D62
:10B7800030E00E94525B1982720100E010E081E01B
:10B790003E010894611C711CF70191917F0199236E
:10B7A00041F4882349F49081992349F4992493948E
:10B7B0001EC0882371F403C09924939401C0992476
:10B7C00099819F3718F40C151D0561F5882379F0D0
:10B7D00001C099248981882321F180688983C5016A
:10B7E000B30141E00E94CD5A8130D1F025C089815A
:10B7F0008823B9F0C501B30141E00E94CD5A8130E0
:10B80000D9F44981B801641B7109640D751DC50126
:10B810000E94CD5A9981891719F0981B99830CC001
:10B820001982892D99819F5F99830F5F1F4FC016E1
:10B83000D10608F0B1CF05C089818F776801C81A99
:10B84000D108C5010E947B5BC6010F90CF91DF91AB
:10B850001F910F91FF90EF90DF90CF90BF90AF902E
:10B860009F907F906F905F904F90089580E094E05C
:10B87000E7EAF9E0DF019C011D9221503040E1F739
:10B8800008950F931F93CF93DF93DA011196FA0176
:10B890004491ED012196FD01A491B0E0179613E0CB
:10B8A000B595A7951A95E1F71A2FDE011196FE01BD
:10B8B0009491929FE0011124AC0FBD1F00FD08C0C0
:10B8C00001FF08C09091D70D51E096FD04C002C061
:10B8D00051E001C050E066956695669570E09B0169
:10B8E0003695322F22273795279590E0280F391F5C
:10B8F000610F711D7695762F662777956795680F8E
:10B90000791F042F10E014C0E901C955D64F80E01B
:10B9100090E008C0FD01E80FF91FE4915111E09596
:10B92000E99301968417B0F3A00FB11F20583F4F41
:10B930002617370749F7DF91CF911F910F9108958F
:10B94000FF920F931F93CF93DF93942F46313CF4D4
:10B95000440F490F440F22FFABC0440FA9C0482F2A
:10B960004A5F092F112707FD109520FD09C021FF0F
:10B970000AC03091D70DFF24F39436FD05C003C0F3
:10B98000FF24F39401C0FF2466956695669570E0E8
:10B990007695762F662777956795680F711DEB0171
:10B9A000C955D64F22FF4FC09E3209F04A5FC801E9
:10B9B000809760E170E00E94A46D80EA90E0689F4B
:10B9C0009001699F300D789F300D1124C801880FB8
:10B9D000991F53E0000F111F5A95E1F7800F911F37
:10B9E000280F391F205D3E4E85E0882369F0F9015C
:10B9F0009491E056FF4F54912F5F3F4FF9016491AE
:10BA0000E056FF4F749104C060E050E090E070E0B9
:10BA1000FF2021F09095609550957095DE01AF570D
:10BA2000BF4FFDE0A73ABF0740F498836983FE014A
:10BA3000E058FF4F50837C93229681508F3FC1F195
:10BA40002F5F3F4FD2CF23FF0DC0FF2011F08FEFAC
:10BA500001C080E06955764FFB01808321964F5FDE
:10BA600091E001C090E09801220F331F220F331F95
:10BA7000200F311F2351304F85E0F9012F5F3F4FD9
:10BA8000E491992311F0843039F0FDE0C73ADF07E3
:10BA900018F4F110E095E993815079F75DE0C73A29
:10BAA000D50730F4FF2011F08FEF01C080E08883CC
:10BAB000842FDF91CF911F910F91FF90089520E087
:10BAC0000E94A05C0895CF92DF92EF92FF920F93B5
:10BAD0001F93CF93DF93162FF22EF0E1EF2EE0228B
:10BAE000C42EE6016E01D52EE6010CC0EE2011F049
:10BAF000488102C0FE014491612F202F0E94A05C6A
:10BB0000FA942196FF2091F7DF91CF911F910F9129
:10BB1000FF90EF90DF90CF9008950F9300E00E9488
:10BB2000635D0F910895CF92DF92FF920F931F9361
:10BB3000CF93DF93162F022FA0E1FA2EF222C42E0C
:10BB4000E6016E01D52EE601FF2011F0488102C00A
:10BB5000FE0144912196442329F0612F202F0E9459
:10BB6000A05CF2CFDF91CF911F910F91FF90DF90FA
:10BB7000CF900895982FAB0180E0692F20E00E94BC
:10BB8000935D089520E00E94935D0895EF92FF92E7
:10BB90000F931F93DF93CF930F92CDB7DEB7182F7C
:10BBA000062F7A01982F9C5E95504E2D4F704A308B
:10BBB0001CF0495C28E002C0405D20E0892F602F26
:10BBC00099830E94A05C9981911731F0B4E0F694BA
:10BBD000E794BA95E1F7E8CF0F90CF91DF911F91ED
:10BBE0000F91FF90EF900895E62FE695E695E69584
:10BBF000F0E0F695FE2FEE27F795E795E80FF11D9B
:10BC0000E955F64F8DE0E73AF80758F4677081E0A0
:10BC100090E002C0880F991F6A95E2F720812827DB
:10BC20002083089547FF02C0840F4195E62FE695D3
:10BC3000E695E695F0E0F695FE2FEE27F795E79569
:10BC4000E80FF11DE955F64F6770A1E0B0E001C0C3
:10BC5000AA0F6A95EAF711C08DE0E73AF80778F481
:10BC6000822F90E09C013595279580FF04C080814C
:10BC70008A278083206841503196442369F70895CC
:10BC80002FEF0E94125E08950F931F93CF93DF93BF
:10BC9000C82FD0E0E62FE695E695E695F0E0F6951C
:10BCA000FE2FEE27F795E795EC0FFD1FE955F64FB0
:10BCB000062F10E0242F332727FD3095200F311F4A
:10BCC000C90168E070E00E94A46D7695762F662722
:10BCD000779567956C0F7D1F6955764F07701070CB
:10BCE00081E090E002C0880F991F0A95E2F78195E4
:10BCF0009081892708C0E058FF4F8DE0E73AF807A8
:10BD0000D0F4808180958083E617F707A0F38DE05B
:10BD1000E73AF80780F4C90168E070E00E94A46D7A
:10BD200021E030E002C0220F331F8A95E2F721950F
:10BD3000808182278083DF91CF911F910F91089599
:10BD40002F923F924F925F926F927F928F929F922B
:10BD5000AF92BF92CF92DF92EF92FF920F931F9319
:10BD6000DF93CF9300D00F92CDB7DEB7182F662E9A
:10BD700059016A01F02E802F05FF04C004FF04C0A2
:10BD800002E003C000E001C001E0E7FE04C0E1946E
:10BD90002224239401C02224D7FE0BC0D094C09447
:10BDA000B094A094A11CB11CC11CD11C4424439488
:10BDB00001C0442482FF06C09CE09093A70D3AE0A6
:10BDC000932E05C096E09093A70D25E0922E86FF56
:10BDD0002FC04110190D28EEA21623E0B20620E074
:10BDE000C20620E0D20614F0190D06C034E6A316F0
:10BDF000B104C104D10414F0190D06C08AE0A816DC
:10BE0000B104C104D1040CF0190D002391F00230EB
:10BE100039F4E4E6AE16B104C104D10454F4190DAA
:10BE2000FAE0AF16B104C104D1041CF4190D01C02D
:10BE3000191B8091A70D810F8093A70D023011F47B
:10BE400020EFF20E5524539492E0792E88242E2D63
:10BE5000332727FD3095862D8A5F89833B832A838C
:10BE600070C0C601B5012AE030E040E050E00E9419
:10BE7000D96DE62E80E3382E3E0C812F662D432DA2
:10BE80002F2D0E94A05C0515D9F5F2FE23C08E2D42
:10BE90008150833008F47394C601B5012AE030E084
:10BEA00040E050E00E94D96DCA01B9012AE030E0BB
:10BEB00040E050E00E94D96D623011F06430C1F46E
:10BEC000E32DE43319F4812E839413C0812E8A94D8
:10BED00073940FC01250812F8F5FF0FE05C0662D46
:10BEE00047E00E94445E05C069810E94F45D01C084
:10BEF000812EFAE0AF16B104C104D1040CF000E0C9
:10BF0000C601B5012AE030E040E050E00E94D96D62
:10BF100059016A01211531054105510581F40023BC
:10BF200031F0023059F4252D223040F408C0F4FEDF
:10BF300010C0222021F430EFF30E01C000E01919E7
:10BF40005394852D90E0EA81FB81E817F9070CF006
:10BF500088CF882061F0662D645F882D472D0E9470
:10BF6000405E662D635F882D472D0E94405E442011
:10BF700039F0812F8919662D4DE22F2D0E94A05C8A
:10BF80000F900F900F90CF91DF911F910F91FF9025
:10BF9000EF90DF90CF90BF90AF909F908F907F9069
:10BFA0006F905F904F903F902F900895EF920F9376
:10BFB000022FFA019F01442737FD4095542F75E069
:10BFC000E72E0E94A05E0F91EF90089520E00E945E
:10BFD000D65F0895A998AB98AC988BBBAD9AAD98F5
:10BFE000AB9AA99A089520E030E006C045E04A9552
:10BFF000F1F700002F5F3F4F28173907BCF3089572
:10C00000AA9885E08A95F1F7000085E08A95F1F716
:10C010000000AA9A8CED95E00E94F35F82EE0E94E8
:10C02000EA5F8EEA0E94EA5F81EA0E94EA5F86EA9E
:10C030000E94EA5F84EA0E94EA5F82EA0E94EA5F65
:10C0400080EC0E94EA5F8FE20E94EA5F85E20E9434
:10C05000EA5F81E80E94EA5F82E20E94EA5F8FEA7B
:10C060000E94EA5F82E28093700108951F93182F67
:10C0700081E80E94EA5F812F0E94EA5F1F91089584
:10C080001F93CF93DF9310E0C7EAD9E084E00E94CA
:10C09000EA5F80E10E94EA5F812F806B0E94EA5F85
:10C0A000A998AB9AAC98FE0180E290819BBBAD9AB7
:10C0B000AD9891819BBBAD9AAD9892819BBBAD9A97
:10C0C000AD9893819BBB3496AD9AAD98815069F73A
:10C0D000C058DF4FAB9AA99A1F5F1830B9F6DF91AD
:10C0E000CF911F910895BF92CF92DF92EF92FF926E
:10C0F0000F931F93CF93DF93EA01E82EF92E062FBB
:10C10000172F21C0F701B1907F0168010894C11C6D
:10C11000D11C04C0009739F00E94B6188091E30842
:10C1200090E082709070E199F5CF1FBB0EBBE09A52
:10C130008DB3B81631F0BDBA8FB7F894E29AE19A90
:10C140008FBF219786012097E9F6DF91CF911F914C
:10C150000F91FF90EF90DF90CF90BF900895809364
:10C16000D80D08958091D80D1092D80D0895FC0136
:10C170008081982F990F9E70807F892B8083662302
:10C1800021F09160807F892B808381818F5F818303
:10C190009281992391F020812F7079F4933659F090
:10C1A000242F20622093D80D903111F4803118F0A3
:10C1B00080818F7C8083118212828281883009F491
:10C1C00043C0893058F4813009F446C08130A0F072
:10C1D0008230D1F1843009F052C036C08F3549F138
:10C1E000803620F4803109F04AC02EC0813689F0B3
:10C1F000823609F044C03DC08081982F9F709F30E7
:10C20000F1F591E6928391819131E0F08F7C80830A
:10C2100019C040664093D80D9081892F82958F7008
:10C220008F5F83708295807F9F7C982B90838FE5B2
:10C2300008C08181883111F4406818C08832F9F44F
:10C2400080E18283118208959181903328F090E0FB
:10C250009595879582831182828190E00197218153
:10C2600030E082239323009751F440644093D80D2B
:10C2700008958181803418F088E0828311820895C6
:10C280008E3091056CF4FC01EE0FFF1FE80FF91FD3
:10C29000E555F24F90819F7081E09F30E9F53FC0F6
:10C2A000823129F1833160F48F30C9F0803118F484
:10C2B0008E3091F529C0803161F0813169F512C06D
:10C2C000843151F08431C8F08531D9F0863121F5BF
:10C2D0001EC091B194701DC091B192701AC090911E
:10C2E000630013C0909163009095987012C0809184
:10C2F000630083FF13C091B102C091B19095907417
:10C3000008C091B1907105C091B1917002C091B116
:10C31000907281E0992319F480E0089580E00895F7
:10C320008F708E3058F490E0FC01EE0FFF1FE80F85
:10C33000F91FE555F24F82E68283118208958F70CE
:10C340008E3068F490E0FC01EE0FFF1FE80FF91F3C
:10C35000E555F24F83E6828380818F7C8083089548
:10C360000F931F93CF93DF938091D50D9091D60DAE
:10C3700001969093D60D8093D50D8091D70D8F5F48
:10C380008093D70D06B3009540E050E010E001C067
:10C39000AE01EA012196CA01880F991F840F951FEB
:10C3A000B8010C2E02C0759567950A94E2F761708A
:10C3B00070708555924F50E00E94B760C630D1052D
:10C3C00039F700B30095C0E0D0E0FE01E051F64E31
:10C3D000E4919E012A5F3F4FC901880F991F820F88
:10C3E000931F8555924FE02361E009F460E09E01C0
:10C3F0002A5F422F50E00E94B7602196C830D105D5
:10C4000021F7DF91CF911F910F910895FF920F9324
:10C410001F93CF93DF93F82EECEBF1E080E090E0F8
:10C42000582F9C014081F41638F0442329F00196DE
:10C430003A9681329105A1F75032B9F1E901CC0F5A
:10C44000DD1FC901A3E0880F991FAA95E1F7C80F66
:10C45000D91F8E0104541E4FA9014F5F5F4FCA01BF
:10C46000880F991FE3E0440F551FEA95E1F7840F09
:10C47000951F20953095205E3F4FA901440F551F11
:10C4800063E0220F331F6A95E1F7420F531F845474
:10C490009E4FB8010E94096E8AE0D8011D928A95CC
:10C4A000E9F7CE55DE4FFA8E02C00CEB11E0C80161
:10C4B000DF91CF911F910F91FF90089580E491E05B
:10C4C000ECEBF1E0DF019C011D9221503040E1F7DF
:10C4D0000895E8E8F3E088E2DF011D928A95E9F724
:10C4E000B89688E4DF011D928A95E9F70895282F10
:10C4F00030E08830C0F4462F572FDA01F901EE0FF3
:10C50000FF1FEE0FFF1FE20FF31FE857FC4F95E0F0
:10C51000899FC001112483579C4F2D912193E817C7
:10C52000F907D9F70895462F572FDA0128503040E0
:10C53000F90193E0EE0FFF1F9A95E1F7E20FF31F69
:10C54000E055FC4F99E0899FC00111248F589C4F02
:10C550002D912193E817F907D9F7089590E00197F5
:10C56000FC01EE0FFF1FE80FF91FEE55FE4FDF0134
:10C57000A85ABD4F6C93DF01AA5ABD4F4C93E95A9C
:10C58000FD4F20830895E0918601F0E0EE0FFF1F3C
:10C59000EE0FFF1FE80FF11DE151FB4F849108954D
:10C5A0008F929F92AF92BF92CF92DF92EF92FF92C3
:10C5B0000F931F93DF93CF93CDB7DEB76D970FB671
:10C5C000F894DEBF0FBECDBFF82EDE011596E6E271
:10C5D000F1E085E001900D928150E1F7DE011A96BD
:10C5E000E1E2F1E085E001900D928150E1F7DE019A
:10C5F0001F96ECE1F1E085E001900D928150E1F7AA
:10C60000DE015496E7E1F1E085E001900D92815062
:10C61000E1F7DE015996E2E1F1E085E001900D924B
:10C620008150E1F719821A821B821C82E0918B01F2
:10C63000F0E0E852FB4F26E030E011E0E491CE2E2E
:10C64000DD24BE016F5F7F4F0FC04F5F5F4FA417A8
:10C65000B50711F4FC01108344305105B1F71F5F99
:10C6600022503040153081F040E050E0C601022EEB
:10C6700002C0959587950A94E2F783709070DC016B
:10C680001196860F971FE1CFFF2041F50E945E6251
:10C6900089810E9406628C0181E00E94C362F801D8
:10C6A000818374E6F72EF2828A810E9406628C01F1
:10C6B00082E00E94C362F8018183F2828B810E9432
:10C6C00006628C0183E00E94C362F8018183F282DA
:10C6D0008C810E9406628C0184E07EC0FF2DF130C7
:10C6E00071F48B810E940662FC0188E081838CE9F1
:10C6F0008283F3828781817F84608783D7C18F2D76
:10C700008230E9F58B810E940662FC0108E001831A
:10C710006CE9F62EF28285E183838781817F8460D4
:10C7200087838EE00E940662FC0182E2818314E628
:10C7300012838EE00E940662FC010183F28284E192
:10C7400083838781817F846087838EE00E94066275
:10C75000FC010183128381E083838781817F846070
:10C76000878383E00E94C362482F8BE062E02DE95B
:10C770000E94AE628CE061E042E220E095C1EF2DC4
:10C78000E33081F50E945E62E9808E2D0E94066290
:10C790008C0181E00E94C362F801818354E6F52E8A
:10C7A000F2828E2D0E9406628C0182E00E94C3629A
:10C7B000F80181838CE98283EA808E2D0E940662D3
:10C7C0008C0181E00E94C362F8018183F2828E2D88
:10C7D0000E9406628C0182E00E94C362F80181839C
:10C7E000F28264C1FF2DF43081F50E945E62EA801E
:10C7F0008E2D0E9406628C0182E00E94C362F801C5
:10C80000818344E6F42EF2828E2D0E9406628C0112
:10C8100084E00E94C362F8018183F282EC808E2D55
:10C820000E9406628C0182E00E94C362F80181834B
:10C83000F2828E2D0E9406628C0184E00E94C36207
:10C84000F80181838CE9828331C1FF2DF53009F035
:10C85000D0C00E945E620E94696281E00E9406620E
:10C86000FC013AE0C32EC18224E6B22EB28282E0FD
:10C870000E940662FC019BE0D92ED182B28283E045
:10C880000E940662FC018CE0E82EE182B28284E024
:10C890000E9406628C0181E00E94C362F8018183DC
:10C8A000B28285E00E9406628C0183E00E94C3622E
:10C8B000F8018183B28204E0A02EA38287E0848302
:10C8C00087818160878385E00E9406628C0183E016
:10C8D0000E94C362F8018183B282F38218E0812E44
:10C8E000848287818160878385E00E9406628C0153
:10C8F00083E00E94C362F8018183B282B6E0BB2E5E
:10C90000B382A9E09A2E948287818160878385E033
:10C910000E940662FC0181828CE9828381E083832C
:10C920008781817F8460878386E00E940662FC01A4
:10C9300091828EE1828388EF83838BE00E9406627E
:10C940008C0183E00E94C362F801818376E4972E14
:10C950009282A382C4828781816087838BE00E9458
:10C9600006628C0183E00E94C362F8018183928297
:10C97000F382D4828781816087838BE00E94066284
:10C980008C0183E00E94C362F80181839282B382AA
:10C99000E4828781816087838091B8018F71806292
:10C9A0008093B8018FE18093B90180E0BE016B5F95
:10C9B0007F4F0E94776281E0BE01665F7F4F0E94D9
:10C9C000776282E0BE01615F7F4F0E94776283E001
:10C9D000BE016C5E7F4F0E9477628E01075E1F4F23
:10C9E00084E0B8010E94776285E0B8010E94776216
:10C9F0005DC0FF2DF630B1F486E00E940662FC01B6
:10CA0000F18282E3828388EF838314E6108786E0D5
:10CA10000E940662FC01F1828EEC828388E08383AF
:10CA2000108744C08F2D873009F040C08FE00E94EE
:10CA30000662FC0184E2818384E6828388E886833F
:10CA400080E10E940662FC0189E081830EE6028398
:10CA50008AE0838380E10E940662FC0118E0118372
:10CA600082E982838BE083838781817F84608783EF
:10CA700080E10E940662FC01118302838CE08383C3
:10CA80008781817F8460878381E06BE043E224E2D9
:10CA90000E94AE6282E061E043E229E60E94AE625B
:10CAA00083E062E043E227E90E94AE6282E00E94F6
:10CAB00084570E9420586D960FB6F894DEBF0FBEC3
:10CAC000CDBFCF91DF911F910F91FF90EF90DF903D
:10CAD000CF90BF90AF909F908F9008956F927F926C
:10CAE0008F929F92AF92BF92CF92DF92EF92FF927E
:10CAF0000F931F93CF93DF938091B80181FF03C001
:10CB000060E075E002C060E074E09091B50184E6F9
:10CB10009802C0011124885A9D4FE091BB01FF2764
:10CB2000E7FDF09548EE53E0E49F9001E59F300D5E
:10CB3000F49F300D112428533045AA24BB24A81A91
:10CB4000B90A281B390BF3E2EF2EF5E0FF2E4091D6
:10CB5000B201440F485F50E0440F551F440F551F6A
:10CB60004752524FE9EDFDE0CC24DD24C61AD70A26
:10CB7000A8E5B2E0A81BB90B1CC0E7016990799049
:10CB80007E014B01661677060CF4430184018C1478
:10CB90009D040CF48601005A164FE501C01BD10B11
:10CBA0002C0F3D1F0A0F1B1F118300839383828369
:10CBB0003496E417F50709F7318320839383828342
:10CBC00015821482DF91CF911F910F91FF90EF900A
:10CBD000DF90CF90BF90AF909F908F907F906F909D
:10CBE0000895E0912B01F0912C018193F0932C0199
:10CBF000E0932B010895FF920F931F93CF93DF9340
:10CC0000B9E0FB2E90E120E0C82FD0E08E0101704A
:10CC10001070201711F4905F07C0892F90E00197E2
:10CC20000E94F165202F90E1FA9431F0D595C795D7
:10CC3000AE014068842FE8CF892F90E00F960E94C4
:10CC4000F165DF91CF911F910F91FF9008951F9390
:10CC5000CF93DF93182F29ED3DE030932C012093E3
:10CC60002B0180913101877471F08091B20188238A
:10CC700019F0813029F402C080E803C080E901C0C6
:10CC800088E9809331018091310187FF0BC086E1F3
:10CC900090E00E944061882329F4809131018F77D0
:10CCA000809331018091310187FD5AC085E160E0B8
:10CCB00040E00E944F10882309F452C08091310156
:10CCC00080628093310180916F018F5F8093320188
:10CCD000E3E3F1E0A3E2B5E080E01CC02D913D91DB
:10CCE0003595279520503E4F37FD05C093E02F3FE7
:10CCF000390724F405C020E030E002C02FEF33E014
:10CD0000932F9370482F440F440F942B90832183CB
:10CD10008F5F3296811711F7C1E3D1E089910E94AC
:10CD2000FB6581E0CF33D807C9F780912B01909143
:10CD30002C01019790932C0180932B018FEF90E0B1
:10CD40000E94F16580E090E00E94F16589ED9DE030
:10CD50009093300180932F01DF91CF911F9108951F
:10CD6000809131018F7DADCF1F920F920FB60F9240
:10CD700011242F938F939F93EF93FF9388B391E0A8
:10CD8000892788BBE0912F01F09130012191F09328
:10CD90003001E0932F01822F90E097BD86BD293CA2
:10CDA00008F0C09A8091690E81608093690EFF91AE
:10CDB000EF919F918F912F910F900FBE0F901F9029
:10CDC00018951F920F920FB60F9211242F933F9335
:10CDD0008F939F93EF93FF9388B391E0892788BB4C
:10CDE000E0912B01F0912C01208130E020FD04C066
:10CDF00088B599B5809603C088B599B5409699BD18
:10CE000088BDC90195958795009791F4CF0101964A
:10CE100090932C0180932B018181882351F4809180
:10CE20007800909179008053984F99BD88BD01C0DA
:10CE300080838091690E81608093690EFF91EF91EC
:10CE40009F918F913F912F910F900FBE0F901F9048
:10CE50001895EDE7F0E08081857E808317981F9A12
:10CE6000AAE8B0E01C9210928B0082E88C9380813B
:10CE7000806280830895EDE7F0E080818F7D80837C
:10CE8000179AAAE8B0E01C9210928B008AE08C936B
:10CE900080818861808308951F920F920FB60F9250
:10CEA00011248F939F93AF93BF93EF93FF93809140
:10CEB000750E882321F01F9A1092750E04C01F98DA
:10CEC00081E08093750EA0912D01B0912E01FD019E
:10CED000819191919093870080938600F0932E0129
:10CEE000E0932D0180916C0E90916D0E90938500D2
:10CEF0008093840012968D919C911397009759F41A
:10CF000081E29EE090932E0180932D018091B801E3
:10CF100081708093750E8091690E81608093690E97
:10CF2000FF91EF91BF91AF919F918F910F900FBEA5
:10CF30000F901F901895AF92BF92CF92DF92EF9211
:10CF4000FF920F931F93CF93DF938091B80181FFDE
:10CF500003C040E055E002C040E054E0F090B20170
:10CF6000FF0C80E1F80E2091B50184E628029001C3
:10CF70001124285A3D4FE091BB01FF27E7FDF095B2
:10CF800068EE73E0E69FC001E79F900DF69F900D5D
:10CF9000112488539045CC24DD24C21AD30A821B65
:10CFA000930B68EFE62EEF0CE1E2FEE0002711277D
:10CFB000041B150B68E572E0621B730B21C0AE2DDC
:10CFC000B0E0AA0FBB1FAD5DBA4FAC901196BC90FC
:10CFD000D5014A175B070CF4DA01A017B1070CF46E
:10CFE000D801A05AB64FE601CA1BDB0B8C0F9D1F60
:10CFF00031832083A60FB71FB383A2833496E394B3
:10D00000EF14E8F23183208393838283885E934018
:10D0100090936D0E80936C0E15821482DF91CF91E8
:10D020001F910F91FF90EF90DF90CF90BF90AF9046
:10D0300008951F920F920FB60F9211242F933F93D2
:10D040004F935F936F937F938F939F93AF93BF9310
:10D05000EF93FF9378940E949B67FF91EF91BF91AC
:10D06000AF919F918F917F916F915F914F913F9180
:10D070002F910F900FBE0F901F9018952091720E58
:10D080003091730E90E0822793279070880F991F3C
:10D09000845A954EFC0145915491232F3327422702
:10D0A00053275093730E4093720E089590916E0E15
:10D0B00096959695982B90936E0E80916F0E8F5F3C
:10D0C00080936F0E843068F0E091700EF091710ED5
:10D0D0009193F093710EE093700E10926E0E109279
:10D0E0006F0E089503C080E00E94566880916F0E15
:10D0F0008823C9F7E091700EF091710E10820895A7
:10D10000882339F08091740E8F5F8093740E80E8CD
:10D1100003C01092740E80EC0E9456688091740EC9
:10D120008530B8F708950F931F93182F0E943E681B
:10D1300008E0812F81700E94806816950150C9F720
:10D140001F910F91089580EC0E94566880E80E941C
:10D15000566880E80E94566880E80E94566880E819
:10D160000E94566880E80E94566880E80E945668CF
:10D1700080EC0E9456680895AF92BF92CF92DF92E2
:10D18000EF92FF920F931F93CF93DF9389ED9DE072
:10D1900090932C0180932B019093710E8093700ECD
:10D1A0001092730E1092720E10926E0E10926F0EFD
:10D1B0001092740E0E94A3688091B2010E9493683D
:10D1C00080916B0E0E94936880E00E949368109299
:10D1D0006B0E03E215E054E0C52ED12CF80120813E
:10D1E0003181C901880F991F820F931FB6010E94D8
:10D1F000A46DEB0122813381C901880F991F820F31
:10D20000931FB6010E94A46D60507C4FC050DC4F4C
:10D21000F8E0C030DF0710F0CFEFD7E07B0128E067
:10D220006030720720F0AFEFEA2EA7E0FA2E8C2FC5
:10D230000E9493685E019B2D9F708E2D8295807F4A
:10D24000892B0E949368C701F4E096958795FA951B
:10D25000E1F70E9493680C5F1F4F25E0033312072C
:10D2600009F0BCCF0091730E8091720E0E949368FA
:10D27000802F0E9493680E94A3680E947268809128
:10D28000780090917900805C934690937900809328
:10D290007800C09ADF91CF911F910F91FF90EF908E
:10D2A000DF90CF90BF90AF9008958091B1019091A1
:10D2B0006A0E981709F494C080936A0E8130F9F0D1
:10D2C000813030F08230F1F1833009F089C05EC0E6
:10D2D0000E9429671EBC80E49CE99BBD8ABD1DBCE1
:10D2E0001CBC87B7837C87BF8CE386BF8FE38093AA
:10D2F0007C0087B7806187BF1FBC8AE021C00E9485
:10D3000029671EBC1DBC1CBC80E797E199BD88BD88
:10D3100080EA9FE0909379008093780087B7837CC0
:10D3200087BF8CE386BF8FE380937C0087B78860DC
:10D3300087BF80917D00816080937D001FBC82E06B
:10D340008EBD4EC00E9429671EBC88EC90E0909371
:10D350007900809378008CE291E09DBD8CBD80EED9
:10D360009BEA97BD86BD87B7837C87BF8CE386BF6A
:10D370008FE380937C0087B7806287BF80917D00B8
:10D38000816080937D001FBC8AE1DACF1EBC80E4FF
:10D390009CE99BBD8ABD1DBC1CBC87B7837C87BF35
:10D3A00080917D008E7F80937D008CE386BF8FE32C
:10D3B00080937C0087B7806187BF1FBC8AE08EBDE9
:10D3C0000E949B6780E593EC909387008093860092
:10D3D00088E893E190938500809384000E943B67E6
:10D3E0008091B101813051F0813028F0823051F0CC
:10D3F000833079F40CC00E946E65089578940E9481
:10D40000BC680895789486E00E94276608950E947B
:10D410006E6508951F920F920FB60F9211242F93ED
:10D420003F934F935F936F937F938F939F93AF93AC
:10D43000BF93EF93FF938091B1018230C1F480E4F8
:10D4400092EA97BD86BD80917800909179008F3FD8
:10D45000910538F488E598E99093790080937800F5
:10D4600008C088EC90E090937900809378000E9447
:10D470005569FF91EF91BF91AF919F918F917F91EE
:10D480006F915F914F913F912F910F900FBE0F9031
:10D490001F9018951F920F920FB60F9211242F9381
:10D4A0003F934F935F936F937F938F939F93AF932C
:10D4B000BF93EF93FF938CB59DB52091760E2223F9
:10D4C00021F0C09A1092760E04C0C09821E02093FB
:10D4D000760EA0913F01B0914001FD012191319163
:10D4E0003BBD2ABDF0934001E0933F012091C3066C
:10D4F0003091C4062817390720F49093C40680930E
:10D50000C30620910C0130910D018217930720F47E
:10D5100090930D0180930C0112968D919C9113971D
:10D520000097D9F489ED9DE09093400180933F01ED
:10D530008091B801809581708093760E87B78F7E39
:10D5400087BF0E9455698091B101882311F0833013
:10D5500021F487B7806187BF78948091690E8160DC
:10D560008093690EFF91EF91BF91AF919F918F9141
:10D570007F916F915F914F913F912F910F900FBECF
:10D580000F901F901895909185019873903121F418
:10D5900063E00E94846D0895983111F48695089592
:10D5A000983211F4880F0895903319F4982F990F39
:10D5B000890F0895FC01A5E6B0E08C918B7F8C93D8
:10D5C000148215821082118216A617A608950E9451
:10D5D000DA6A089521E0FC018481882309F420E0BF
:10D5E000822F0895FC0181819081891B877098E0CA
:10D5F000981B81E0933008F480E00895FC01848159
:10D600008823F9F08150848382819381890F8283FA
:10D6100086A5882309F44CC087A5982F915097A719
:10D62000882331F0809165008460809365000895BF
:10D63000809165008B7F809365008091900187A722
:10D6400008951B98809165008B7F8093650085818C
:10D65000882319F0815085830895808191818917ED
:10D6600039F190E0DF01A80FB91F16962C9116979B
:10D67000228356962C91569724831E962C911E97A2
:10D6800023835E962C915E972583D0962C91D0971C
:10D6900026A717A696962C919697322F31509696DC
:10D6A0003C939697222321F4019687709070808393
:10D6B00008958F929F92AF92BF92CF92EF92FF9276
:10D6C0000F931F93DF93CF9300D0CDB7DEB74C01FC
:10D6D000122F4A8369830E94F26A4A8169818823F2
:10D6E00031F180918501887311F1F401A180BB248F
:10D6F000C501019697E0F92EF8228081F816B9F05D
:10D70000662329F080918F01865F860F01C080E03B
:10D71000A80CB91CF5018683842F0E94C36AF50109
:10D72000868B168FE0AA06A3C686F401F1820F90BD
:10D730000F90CF91DF911F910F91FF90EF90CF90BD
:10D74000BF90AF909F908F900895AF92BF92CF926D
:10D75000EF920F93DF93CF9300D00F92CDB7DEB748
:10D760005C012B834A8369830E94F26A2B814A8180
:10D770006981882329F180918501887309F16623E5
:10D7800029F080918F01865F860F01C080E0F5014E
:10D790008283842F2B834A8369830E94C36AF501A5
:10D7A00084832B812583E6A617A6C382808181838B
:10D7B0004A816981002321F00150C5010E94596B03
:10D7C0000F900F900F90CF91DF910F91EF90CF902E
:10D7D000BF90AF900895CF92EF920F93CF93DF93C6
:10D7E000EC018091850186958695869587702881C4
:10D7F0009981291709F05CC1E62FF0E0E132F105CB
:10D8000008F056C1EA5BFF4FEE0FFF1F0590F49141
:10D81000E02D0994CE0166E44AE0DEC0CE0166E464
:10D8200044E1DAC0CE0166E44EE1D6C0CE0164E642
:10D830004AE022E002E0EE24E39452E0C52E36C135
:10D84000CE016FE545E022E00AE0EE24E394CC242B
:10D850000E94596BCE016FE545E02AE001E00E948D
:10D86000596BCE016FE545E022E00AE01FC1CE0111
:10D8700060E54AE023E002E0EE24CC24CA940E9452
:10D88000596BCE016CE34AE023E0CC24C3940E94A0
:10D89000596BCE0166E44AE021E000E032E0E32E7D
:10D8A00096C0CE0166E445E021E001E0EE24E39479
:10D8B000CC240E94596BCE0162E34FE022E00E942B
:10D8C000596BCE0160E54FE022E0F0C0CE016EE67C
:10D8D00045E021E002E0EE24E394CC240E94596B61
:10D8E000CE016CE745E021E02AC0CE0162E345E0CD
:10D8F00025E000E0EE24CC240E94596BCE016AE5BD
:10D9000045E025E00E94596BCE016EE643E024E03D
:10D9100002E0CCC0CE0160E545E02AE003E0EE2461
:10D92000E394CC240E94596BCE0160E545E024E1EC
:10D9300001E00E94596BCE0160E545E02AE003E07A
:10D94000B5C0CE016AE044E125E002E0EE24E394B4
:10D95000CC24C394ABC0CE0162E344E02AE002E0F1
:10D96000EE24E394CC240E94596BCE0166E448E097
:10D9700024E101E00E94596BCE0162E348E02AE015
:10D9800002E00E94596BCE0166E444E024E101E02C
:10D990008DC0CE0168E745E02AE00AE016C0CE015E
:10D9A00068E745E022E30AC0CE0160E044E12AE0F6
:10D9B00001E00BC0CE0160E044E12AE002E005C0D6
:10D9C000CE0160E044E12AE003E0EE24E394CC24BD
:10D9D0006DC0CE0166E448E221E000E048C081303D
:10D9E00009F466C0CE016BE405C0813009F460C063
:10D9F000CE0161E44AE021E000E041C0CE01642FA5
:10DA000046E0F9CFCE0166E44AE022E0E6CF81307D
:10DA100009F44EC0CE0166E44AE022E0EDCFCE012B
:10DA200068E7E8CFCE0168E74AE021E01FC0CE01F9
:10DA30006AE74AE021E00FC0CE016CE74AE021E04E
:10DA400004C0CE0168E74FE023E003E010C0CE0140
:10DA500068E74FE023E002E00AC0CE0168E74FE04C
:10DA600023E004C0CE0166E444E129E101E0EE24B4
:10DA7000E39406C0CE0166E44AE022E002E0EE2430
:10DA8000CC240E94A56B14C0CE016CE344E123E0DA
:10DA900002E0EE24CC24C3940E94596BCE0160E5D1
:10DAA00044E123E0EE24E394CC24CA940E94596B11
:10DAB000DF91CF910F91EF90CF900895682F87E479
:10DAC00094E046E40E94EB6B0895629FD001739F3F
:10DAD000F001829FE00DF11D649FE00DF11D929F0A
:10DAE000F00D839FF00D749FF00D659FF00D992749
:10DAF000729FB00DE11DF91F639FB00DE11DF91F6D
:10DB0000BD01CF0111240895991B79E004C0991F2C
:10DB1000961708F0961B881F7A95C9F78095089587
:10DB2000AA1BBB1B51E107C0AA1FBB1FA617B70743
:10DB300010F0A61BB70B881F991F5A95A9F780955F
:10DB40009095BC01CD01089597FB092E07260AD0B8
:10DB500077FD04D0E5DF06D000201AF470956195BA
:10DB60007F4F0895F6F7909581959F4F0895A1E214
:10DB70001A2EAA1BBB1BFD010DC0AA1FBB1FEE1F47
:10DB8000FF1FA217B307E407F50720F0A21BB30B92
:10DB9000E40BF50B661F771F881F991F1A9469F70E
:10DBA00060957095809590959B01AC01BD01CF016A
:10DBB000089597FB092E05260ED057FD04D0D7DF18
:10DBC0000AD0001C38F450954095309521953F4F70
:10DBD0004F4F5F4F0895F6F790958095709561953A
:10DBE0007F4F8F4F9F4F0895EE0FFF1F0590F491C9
:10DBF000E02D0994FB01DC014150504048F00590B4
:10DC00000D920020C9F701C01D9241505040E0F72D
:10DC100008956817790768F4FB01DC01E40FF51F2C
:10DC2000A40FB51F02C002900E9241505040D8F789
:10DC300008950C94326EDC0101C06D934150504048
:10DC4000E0F70895DC01CB01FC01E199FECF06C0AD
:10DC5000FFBBEEBBE09A31960DB20D9241505040A1
:10DC6000B8F70895FB01DC0102C001900D9241500C
:0ADC70005040D8F70895F894FFCF54
:10DC7A0084038503860387034AF0004DFF072204C5
:10DC8A007C5E9CCE003264E2F1003264645A505ADF
:10DC9A006450463C46649CEC1E465AD90D210ED966
:10DCAA000DFF0000AA05FF09FF0DFF135414AAD99E
:02DCBA000D005B
:00000001FF
